:020000040800F2
:1000000000000120C9EC040865ED0408B9BB010833
:1000100009BA010865ED040865ED04080000000058
:1000200000000000000000000000000065ED040872
:1000300065ED04080000000065ED04084980010832
:1000400065ED040865ED040865ED040865ED040838
:1000500065ED040865ED0408B17B0108B97B010872
:10006000C17B0108C97B0108D17B01087998000890
:100070008998000899980008A9980008B99800087C
:10008000CD980008E198000865ED040865ED0408C6
:1000900065ED040865ED040865ED0408D97B0108E9
:1000A00015B5000801B4000825B50008F1B3000833
:1000B00029B4000839B4000849B400085594000870
:1000C00049940008899400087D94000865ED0408AF
:1000D00065ED0408957F0108A17F0108AD7F010847
:1000E000E17B010865ED040865ED040835B50008FD
:1000F000EDB4000865ED0408DDB40008F5980008CB
:1001000065ED040859D3000859B4000865ED0408EA
:10011000B97F0108C57F010869B400089DA10408E2
:10012000099900081D9900083199000845990008AF
:1001300059990008000000000000000000000000C5
:100140000000000000000000000000001DAE0408D8
:100150006D9900088199000895990008D17F0108E0
:10016000BD940008B194000865ED040865ED04082D
:1001700065ED040865ED04080000000000000000C3
:1001800065ED040865ED040865ED040865ED0408F7
:1001900065ED040865ED04080000000065ED040845
:1001A00000000000000000000000000065ED0408F1
:1001B00065ED040865ED0408000000000000000083
:1001C000000000000000000000000000000000002F
:1001D00000000000000000000000000065ED0408C1
:0801E000D4E704000100000057
:1001E800FF21010005000000CC280120F431012086
:1001F8000000000025DC0008F03101200530010076
:1002080008000000E8310120003201200000000051
:10021800CC380608FC31012013020100040000005C
:10022800342F01200C32012000000000D4380608C9
:10023800083201200A9001002400000078190120EA
:10024800143201200000000099A002081032012099
:100258001402010005000000C42501203C320120E1
:1002680000000000D8380608383201201F020800B4
:100278001000000024240120483201200000000062
:1002880035DC000844320120061001002600000079
:10029800C41B01205C320120000000005DDB000867
:1002A8005832012021020100F0000000A449012079
:1002B800184B01200000000059550308144B012079
:1002C8002C00040010000000944901200C4C01206F
:1002D80000000000CD9D0208084C012025201E00CA
:1002E8002C01000068480120204C0120000000007B
:1002F800000000001C4C01202B001200240000000C
:1003080020480120504D012000000000E99D02080E
:100318004C4D012016200100060000005C3A012027
:10032800784D012000000000E0380608744D0120D7
:100338002700010004000000503A0120844D0120EC
:1003480000000000E6380608804D01200C5004002B
:1003580080000000783301208C4D0120000000004F
:1003680005430208884D0120031101000A0000001E
:10037800FC380120104E0120000000000DA10308E8
:100388000C4E01202920140078000000E8370120D5
:10039800204E012000000000000000001C4E01203B
:1003A800012001000C000000DC3701209C4E0120D8
:1003B80000000000EA380608984E012023200100BA
:1003C80010000000CC370120AC4E012000000000D6
:1003D80085A00208A84E01200B3001001A00000079
:1003E80094370120C04E012000000000F6380608AE
:1003F800BC4E01200E50040058020000F8330120C2
:10040800E04E0120000000007D9B0208DC4E012028
:100418001E10010009000000143701203C51012082
:100428000000000010390608385101200D100100A5
:1004380070000000A03601204C510120000000008F
:100448001DC8010848510120220201001C010000BA
:1004580008390120C05101200000000025EF0008E4
:10046800BC510120160215003F000000D44A0120AB
:10047800E0520120000000007DDC0008DC52012071
:10048800184001003800000068360120245301207C
:100498000000000061E10008205301201B02010058
:1004A800100000007053012060530120000000007C
:1004B80011DC00085C53012028020400040000003D
:1004C80088530120845301200000000005DC000847
:1004D80080530120270204000400000094530120E7
:1004E8009053012000000000F9DB00088C53012024
:1004F8001A0201003C000000944A01209C5301208C
:100508000000000001E100089853012004000800E1
:10051800800000001C3B0120DC530120000000008B
:1005280000000000D85301201C0202001C0000003B
:10053800B03701206054012000000000A9E0000845
:100548005C5401202630010008000000C83B01204F
:100558008054012000000000999E03087C5401206B
:100568000812040014000000B43B01208C54012040
:1005780000000000D9DA00088854012003120100A5
:100588003D0000002C3C0120A45401200000000084
:100598001A390608A0540120010201000A000000CF
:1005A800343F0120E8540120000000003DDB000832
:1005B800E45401200C02010004000000D03B01209B
:1005C800F8540120000000004DDB0008F45401201D
:1005D800FD1701009A000000443F0120005501204A
:1005E80000000000A59C0308FC5401201310010022
:1005F800040000008C370120A055012000000000F5
:10060800583906089C550120020201000300000029
:10061800303F0120A8550120000000000000000024
:10062800A4550120F5C1010074000000883801209C
:10063800B05501200000000061A60308AC55012058
:10064800F62101000C0000007C380120285601200A
:10065800000000005C39060824560120121201002F
:1006680004000000706F01203856012000000000CF
:1006780068390608345601201102010008000000FC
:10068800746F012040560120000000006C390608F4
:100698003C560120F83101000600000050360120C8
:1006A8004C56012000000000743906084856012005
:1006B800020001000C000000EC3B0120585601200C
:1006C800000000000000000054560120FE01010057
:1006D8001400000060380120685601200000000066
:1006E800C1DA000864560120061204001800000050
:1006F800D43B0120805601200000000035E00008AE
:100708007C560120F7010100060000007438012022
:100718009C560120000000007A39060898560120EE
:100728001A0001000E0000009C3B0120A856012081
:100738000000000080390608A456012014000100BA
:100748000500000060360120BC56012000000000B2
:100758008E390608B8560120FD010100240000006A
:10076800F63A0120C856012000000000C3560108CF
:10077800C45601201D02020006000000F03A0120C4
:10078800F05601200000000000000000EC56012097
:10079800F9010100040000007C6F0120FC560120D3
:1007A800000000007D560108F856012012300100B3
:1007B80010000000903201200457012000000000C2
:1007C8009439060800570120373001002600000040
:1007D800DC7401202076012000000000A4390608FE
:1007E8001C7601201B2001000C000000DC73012096
:1007F8004C760120000000002138030848760120CB
:100808001010010002000000A87101205C76012090
:1008180000000000CA390608587601200E020100BF
:100828000200000098760120647601200000000094
:10083800CC390608607601202F2001002200000034
:100848006C760120846F012000000000CE39060874
:100858006876012001010100040000001C790120D4
:10086800407F012000000000000000003C7F0120C4
:10087800000101000400000018790120487F0120D0
:1008880000000000F0390608447F01200201010041
:100898000300000014790120507F012000000000AF
:1008A800F54202084C7F01202902010040000000A7
:1008B800787E0120587F012000000000F4390608E6
:1008C800547F0120205201000800000020780120F8
:1008D8009C7F012000000000343A0608987F012020
:1008E8002A1201000800000018780120A87F0120C2
:1008F800000000003C3A0608A47F0120190001000E
:100908000500000010780120B47F012000000000DD
:10091800443A0608B07F01201F500100240000005F
:10092800547E0120C07F0120000000004C3A0608D8
:10093800BC7F01203840010006000000B876012085
:10094800E87F012000000000703A0608E47F0120DB
:100958002332010014000000C485012068870120AB
:1009680000000000783A06086487012005020100AB
:10097800040000007C860120808701200000000020
:100988008C3A06087C8701202C0201000400000034
:10099800CC800120A887012000000000903A0608BA
:1009A800A48701202D020100010000001080012011
:1009B800B08701200000000000000000AC87012083
:1009C800001201000A000000C8910120FC960120D5
:0C09D8000000000000000000F896012064
:08280000082800080040000850
:1080000030B5FAB18E464FEA014C034600F1C00587
:10801000002419680C3353F8042C43F8084C41EA47
:108020000C0142EA0E02AB4243F80C1C43F8042C4C
:10803000EFD1D0F8C03043EA0E03C0E93144C0F8B4
:10804000C03030BD4FEA014E8C46DEE7836930B464
:108050005C6999682268096822F0010222601C8A22
:10806000CA6822EA0402CA60027D00681F2A06D993
:10807000203A082144689140214216D0FEE70821A9
:10808000046891402142F9D1202101FA02F2826074
:10809000204A12783AB11A7F012A0BD1D3F8042171
:1080A0000132C3F8042130BC7047202101FA02F2EA
:1080B000C260EDE7D3F800210132C3F80021EFF3ED
:1080C0001181502282F312885868C9B29D6C0268EF
:1080D000DC6C22EA05022243026081F311885A69AE
:1080E0009968D3E90D40096814605061D3E90F40E5
:1080F000546090605C6CB3F8B400D4600124C86232
:108100001068204310601A8A1C77CB68134330BC78
:10811000CB6070478001002070B50E4E7368002B55
:1081200016DD06F10804002503E073682034AB4235
:108130000EDD237F0135002BF7D0E06800220028F8
:10814000F3D0217D20340FF09DFD7368AB42F0DC4D
:10815000012070BD80010020704700BF024B03EB7F
:10816000401090F825007047800100204368426D60
:1081700030B49A61EFF31182502383F3128841687F
:10818000D2B2856C0B68046D23EA050323430B60B0
:1081900082F31188436981681A68096822F0010234
:1081A000D0E908541A60826A1D605C615A60D0E9A7
:1081B0000B429C60DA600023B0F86C2030BCCA62CD
:1081C00003777047084A0346D0F8E4005268D3F8B2
:1081D000F010121A00209142B8BFC3F8F02001221B
:1081E00083F81C21704700BF001000E04FF40063CB
:1081F00083817047704701207047012070472DE947
:10820000F047DFF880810E460746D8F80050B8F8EE
:108210000420B8F80A90C2EB25135200C2EBE50225
:10822000B8F906506A4303FB03F5B8F908302D137B
:108230005D43B8F90E30AD134FEAE37E05EBE2255E
:10824000A5F5FA31C8F81C5081FB010C03FB0CF2B8
:1082500000FB0E22A3FB003E9644B8F90C201B0A3B
:1082600082FB014243EA0E63120342EA14522403E2
:108270001B194FF0000442EB2E22A3FB093E02F52E
:10828000004209FB02EE4FEAEE734FEA6E0253EA38
:108290006E0E6BD0B8F914904FEAE97E09FB0CFC26
:1082A00000FB0ECCA9FB00908444B8F9120080FBBF
:1082B00001E148044FEA4E4140EADE3011EB090982
:1082C000D8F820104CEB0000C1F5801C14EB090419
:1082D000B8F910100CF0004A40F6354900EBC10126
:1082E0004AEA5C0A4FEACC7CBCEB04006AEB010A68
:1082F000A0FB090109FB0A1146F0AAFAB8F91A40D5
:108300004FEA613E8146430B04FB0EF24FEAE47CE8
:1083100043EAC14303FB0C2CA4FB0342624404FB6D
:108320000EFE03FB02EEB8F91820A4FB03439E44A3
:10833000640E02FB01F344EACE1414EB000C4FEA86
:10834000E274A2FB092941EB6E6E04FB0031D40CF0
:10835000B8F91630494444EA41341CEB04044EEBAE
:10836000E141240A44EA016404EB03140FB1240A36
:108370003C6026B105EB850580352D123560BDE8E2
:10838000F08700BF7818012008B5006840F0A2FE11
:10839000D8B90F4A0F4992F8093192F808011B0128
:1083A00043EA003392F80A0143EA101392F80B01F2
:1083B0000B6292F80C3192F80D211B0143EA003355
:1083C000012043EA12130B6008BD0020FCE700BF48
:1083D00080010020781801203B4BDFED3C3A93F8F8
:1083E000251093F82400090293F8262093F827C05B
:1083F00001EB004193F8280093ED0D6A0A4409024D
:108400004FEA002093F8291048BF02F17F42B8EEEE
:10841000C66A00EB0C4007EE902AB3F940200144F5
:10842000000205EE902AB3F93C20F8EEE77A48BF47
:1084300001F17F4104EE902AB3F93E20F8EEE55AAF
:1084400007EE101A67EEA37A06EE902AF8EEE44AD9
:10845000B3F93A20F8EEE66A012005EE102AB3F9E6
:108460003820E7EEA54AB8EEC55A04EE102AB8EE59
:10847000C77AB3F92E20B8EEC44AA7EEA65AD3EDB8
:108480000C6A27EE237A05EE902AA4EEA76AB3F9C8
:108490002C20F8EEE66AF8EEE55A04EE902AF6EEA5
:1084A000003AE7EE046AF8EEE44AA5EE076A65EEE4
:1084B000875AB0EE667AE4EEA35AA7EE867AC3ED49
:1084C000125A83ED117A70477818012008218436FA
:1084D00030B10A4BD3ED117AFDEEE77AC0ED007AA8
:1084E00051B1064B9FED067AD3ED127A67EE877A8B
:1084F000FDEEE77AC1ED007A704700BF78180120E1
:108500000000C842704700BF01207047012070473B
:10851000704700BF002070470020704738B5074BF8
:1085200014460D46DB6C1B6A984702464FF40073F5
:10853000002012682A60238038BD00BF781801200F
:1085400008B5064BDB6C33B15B69984780F00100DE
:10855000404240B208BD4FF0FF3008BD78180120FE
:10856000002070472DE9F041FBB1164688469F1860
:10857000114DEC6C002341463046A4681A46A047D2
:108580000028F6D0EB6C2BB15B69984718B9EB6CFF
:10859000002BF9D1FEE7013608F50078B742E8D1A3
:1085A0002B6D00206B65BDE8F081034D00202B6D25
:1085B0006B65BDE8F08100BF781801202DE9F0411E
:1085C0002BB316460F4603EB0208144C03E0E16C94
:1085D00011B14B699847E16C00230D69304639466B
:1085E0001A46A8470028F2D1E36C2BB15B69984783
:1085F00018B9E36C002BF9D1FEE7013607F50077D7
:10860000B045E8D1236D00206365BDE8F081034CDF
:108610000020236D6365BDE8F08100BF781801205C
:1086200000207047836910B5074C04EB8303986FF3
:108630003BF0A6F80021B4F8980040F047FC002376
:1086400084F89A3010BD00BF7818012080699C30F2
:108650003BF096B82DE9F0412E4F07EB401898F803
:1086600024300BB9BDE8F08100EB80030E460021F9
:10867000044607EB4313450193F8122183F81211C6
:1086800088F80A2047F074FF98BB3D4422482E81A9
:1086900000EB441047F090FF3B782A6A9BB1E968F1
:1086A0000124D2F8AC308C4003F1C001420010F438
:1086B000004F90B202D15A6822435A600C3399425B
:1086C000F4D1BDE8F081E9680124D2F8AC3001F1C1
:1086D000100203F1C0019440420010F4004F90B228
:1086E00002D15A6822435A600C339942F4D1BDE852
:1086F000F0810A4B93F8FC2002EB420203EBC20329
:10870000234493F8A960002EBFD0012388F80A30D3
:10871000BBE700BF800100208801002078180120FD
:1087200010B5044647F0D4F80146204689B2BDE8AA
:1087300010408FE72DE9F04147F036FF98B31D4E0A
:10874000D6F81056002D12DD0024377806F21C6092
:10875000A046013417B1037F012B1FD04269AC4200
:1087600000F58670136843F001031360F1D10FF038
:10877000BDFCD6F81846C6F81406002C0CDD0E4BCE
:1087800003EBC4041968083333F8042CC868A34207
:1087900042EA0002CA60F5D1BDE8F08180F8FC80B1
:1087A000FFF7E4FCDAE73FF0D1FC0028C7D1BDE8D1
:1087B000F08100BF80010020CC0B00200269C3685B
:1087C0002DE9F04712EA03092AD005460E464FF07C
:1087D00000474FF00008B9FA89F327FA03F21B3B70
:1087E000D24309EA02092A61042B16D8DFE803F014
:1087F000352C231A0300B36A002B37D003F1FF3A5C
:10880000C6F828801FFA8AFA746A34B123682046B1
:10881000514698476468002CF8D1B9F1000FDAD1BD
:10882000BDE8F0877068696B036889B29847B9F151
:10883000000FD0D1F4E7B068A96B036889B29847FC
:10884000B9F1000FC7D1EBE7F068E96B036889B2B3
:108850009847B9F1000FBED1E2E73069296C03688F
:1088600089B29847B9F1000FB5D1D9E7E96A1FFA83
:1088700081FAC9E72DE9F04F4D4C83B02378F3B965
:10888000D4F81036002B16DD00264A4831464769D9
:10889000D0F8AC303D6803F1C00225F001053D6021
:1088A00059600C339342FBD10136D4F8103600F5F1
:1088B0008670B342EBDC012003B0BDE8F08F3E4B85
:1088C000DFF80091D3F850B00FF010FC59F8C42C29
:1088D000D4F814161432401AB0EB420F64DBA9F13D
:1088E000C00704F108060025DFF8DCA0019718E0B6
:1088F000B0F5606F48D0019B98814FF6FF712F4B08
:108900005A46411A4FF05C0018BF012100FB0530A8
:108910000EF032FC019B013520361433082D0193F3
:108920002ED06368AB422BDDB3694FF6FF78244F3E
:10893000D3F814C07268D3E93D015FFA8CF32CF0D0
:10894000FF0C103BA7FB03731B091AF803309C4470
:10895000DCF804309BB2C91A47F056FE4FF6FE739E
:108960009842D7D059F8B83C404503F1010349F883
:10897000B83CBDD159F8BC3C013349F8BC3CBCE71C
:10898000012289F846207BE70B4A92F8FC3003EB82
:10899000430302EBC3032B4493F8A9300D2BAAD158
:1089A0008023019A9377A8E7002003B0BDE8F08FF9
:1089B000800100209C07002078180120C0120020B0
:1089C000ABAAAAAA78120020387B0508836810B5E4
:1089D000044682B01BB19A88196812048A6101208A
:1089E00012F0D4FCA36813B11A689B8893610A2023
:1089F00012F0CCFC236800201B6AADF804005BB9C0
:108A00002046022301AA80210EF02EFE9DF805309B
:108A1000242B14BF00200F2002B010BD10B5104B46
:108A200004465868D4F8E410D4F8D83094F8D0202C
:108A30000B44C4F8D800012AC4F8DC3005D0D4F8BF
:108A4000D4300133C4F8D43010BD04F1E801201D46
:108A50000EF0B0FDD4F8D4300133C4F8D43010BDDA
:108A6000001000E070B586698AB0054696F8DC30E3
:108A7000012B23D0023B012B2BD8D6F89C308C2223
:108A8000154CEC461A700FCCACE80F00D6F89C30B1
:108A90000093D6F8A03001930FCCACE80F0094E817
:108AA0000300AB698CE8030003F1100069460EF087
:108AB00081FDAB691A69136A002BFCD1D6F8A0308E
:108AC000B3F90220EA81B3F904202A82B3F906300F
:108AD0006B8201200AB070BD90060508F0B590F8D1
:108AE0001E318DB00546032B55D090F8DC30D0F800
:108AF000A060012B00F0908016D8D0F89C300022A6
:108B000005211A605A609A609A81D0F8E030C0F866
:108B1000F010B3F57A7F00F28F800323012480F8F0
:108B2000DC3020460DB0F0BD023B012B2FD8D0F831
:108B30009C309222544F0DF1080C1A70D0F8A040CE
:108B40000FCFACE80F000FCFACE80F0097E80300A1
:108B5000D5F89C308CE8030002A905F11000CDE99E
:108B600002340EF027FD2A69136A002BFCD1B6F9F6
:108B700002300124A5F8D0302046B6F90430A5F81B
:108B8000D230B6F90630A5F8D4300DB0F0BD0124CE
:108B900020460DB0F0BD3D4E00230122103006F1FD
:108BA0000C010B938DF814208DF828200190CDE94D
:108BB0000633CDE908330A23CDE9026102A9049303
:108BC0000EF0F8FC2A690198146A002CFCD1F28995
:108BD000052A18DD338AB6F91240B6F9141014F5D7
:108BE000004F08BFB3F5004F376914BF01230023BE
:108BF00011F5004418BF01241C4303D0C5F8D07000
:108C0000A5F8D410063A002AC2D0B0227E210EF078
:108C100003FD20460DB0F0BDB6F908201C46A0F8B3
:108C2000D020B6F90A30A0F8D230B6F90C30A0F84E
:108C3000D43020460DB0F0BD03691A7BF2B15B69F8
:108C4000E3B190F89840CCB1D0F89C1001230E22EB
:108C50008C20C5F8A45008700D49C5F8FC2085F893
:108C60000031D5F89C2085F8DC30D5F8A030C5F867
:108C70000411C5F8F420C5F8F83089E7022301246F
:108C800085F8DC3084E700BF90060508000000206E
:108C9000C58100082DE9F04100F1100590B0B62221
:108CA0007E21064690F81E7128460EF0B5FC642021
:108CB00012F06CFBB3691BB11A689B881B049361AB
:108CC000012012F063FBB36913B11A689B889361AA
:108CD0000A2012F05BFB00227C2128460EF09CFC4F
:108CE000012012F053FB0022592128460EF094FC7B
:108CF000012012F04BFB002301225E218DF8103081
:108D00002846059307930F938DF8031001A98DF85A
:108D100024208DF83820CDE90232CDE90A33CDE99F
:108D20000C330DF103030193B24B06934FF4A4737C
:108D300008930EF03FFC33691C6A002CFCD10A201A
:108D400012F024FB2846012259210EF065FC012077
:108D500012F01CFB032F00F0AD809B22402128461F
:108D6000A54C0EF059FC012012F010FB032241210A
:108D700028460EF051FC012012F008FB94F8013156
:108D8000013BDBB2022B40F28B80CD2242212846F0
:108D90000EF042FC012012F0F9FA08224321284685
:108DA0000EF03AFC012012F0F1FA04225821284674
:108DB0000EF032FC012012F0E9FA0A225321284673
:108DC0000EF02AFC012012F0E1FA02227C21284652
:108DD0000EF022FC012012F0D9FA28460E227D2145
:108DE0000EF01AFC012012F0D1FA96F821010028A9
:108DF00042D00EF021FF0546002800F0F780262320
:108E00008188C3807D4BF360B1FA81F3202BC3F1DD
:108E10001F0231D07A48104404EB820290F8F071BE
:108E200006F10C00C2F824014FF0004232FA03F3BD
:108E300005D0744A106820EA0300106053610023D3
:108E40000191286801A90593CDE903336E4B029384
:108E50003AF086FDE31993F86421F02A00F2AC8021
:108E6000AB884FF00042B3FA83F332FA03F303D036
:108E700064490A6813430B60D4F86C3163499A085B
:108E8000B1EB930F4FF0020306D252085B008A4207
:108E90009BB201D9FF2BF8D9B38210B0BDE8F081A5
:108EA000574A134493F80022120162F0320202F092
:108EB000FD026BE72246482128460EF0ADFB01205B
:108EC00012F064FA4921802228460EF0A5FB012009
:108ED00012F05CFA2246452128460EF09DFB012047
:108EE00012F054FA4621062228460EF095FB012086
:108EF00012F04CFA2246472128460EF08DFB012045
:108F000012F044FA9B22402128460EF085FB0120F6
:108F100012F03CFA384C3A46412128460EF07CFBD0
:108F2000012012F033FA94F80131013BDBB2022B3D
:108F300040D8334A134493F80022120162F03202FF
:108F400002F0FD02422128460EF066FB012012F0DD
:108F50001DFA0822284643210EF05EFB012012F084
:108F600015FA0222582128460EF056FB012012F075
:108F70000DFA0A22532128460EF04EFB012012F072
:108F800005FA02227C2128460EF046FB012012F051
:108F9000FDF90E227D2128460EF03EFB012012F045
:108FA000F5F92846B0227E210EF036FB012012F0A2
:108FB000EDF91AE7CD22C5E7154AF02112F907802D
:108FC00083F8641103214046D75D3FF0CBFEB8F132
:108FD000000FFFF645AF012307F01F074FEA5818AF
:108FE00003FA07F70B4B43F8287039E7034BF3609C
:108FF00042E700BFB8060508781801201D8A00085E
:1090000010060508003C01400000111080969800F1
:10901000207B050800E100E003682DE9F3411E789C
:109020000146012E0BD0022E66D11B6A002B63D1A4
:109030003122742102B0BDE8F0410EF0EDBA3123C7
:10904000424D85F87031036893F90420531C53D0C6
:10905000032A51DC602303FB0253D3F88801002864
:109060004AD093F8C941202C46D1846914F40044B5
:1090700042D193F8C80101283ED091F80480212103
:10908000D5F8F4C283F8C911402183F8C86183F888
:10909000CA1105F5B871C3F8CC41C3F8AC112C491D
:1090A000A3F8B261C3F8B4112A49C3F8BC11B3F8EC
:1090B000B21189B2FF2922D8B3F8B2114FF000776C
:1090C00089B260204FEA480819235043F4222E1831
:1090D000A6F8B0114146CDF800C0DFF884C0604466
:1090E0003FF038FA78B1002386F8C831B5F8F83285
:1090F00001339BB2A5F8F83202B0BDE8F081FF2140
:109100004FF08077DDE7D6F8882196F8B0115368E4
:1091100023F07F7323F4583323F47F7323F0030386
:1091200043EA080343EA01430B493B435360D6F843
:10913000BC3186F8C8018B4203D008498B4218BF66
:10914000F22413681C431460D6E700BF781801208E
:109150000000FFFF190404088D0504088D0E0408A3
:10916000001A012010B5044600683FF0B3FF30B983
:109170002046044AF7213FF00DFF012010BD0020DA
:10918000FCE700BF8802002008B503681A78012AAE
:1091900005D00C4A00213FF0FDFE012008BD93F9E7
:1091A0000430094A03EB430302EB431393F8C9214C
:1091B000202A01D0002008BDD3F888319B691B0408
:1091C000F8D4E6E79C1801207818012010B50E4C61
:1091D000D4F8FC2294F8FA322AB103F001031168A2
:1091E000928873B98A6142F03DFE02E05B6998475C
:1091F00018B9E36C002BF9D1FEE7236D00206365FD
:1092000010BD1204EEE700BF78180120BFF34F8FA6
:109210000549064BCA6802F4E0621343CB60BFF312
:109220004F8F00BFFDE700BF00ED00E00400FA052E
:109230002DE9F041CB781BB900273846BDE8F08115
:1092400000F110040D460646897820460DF0FAFF1D
:1092500007460028F0D0E8780EF0EEFCB0612B78DD
:109260000133DBB210B1C371222383710D21DFF80A
:109270008C800EF04DFDB0690DF0DEFFD8F8503057
:10928000632BFBD9D8F86C311B499A08B1EB930FCB
:109290004FF0020306D252085B008A429BB201D90A
:1092A000FF2BF8D92046B382FFF790FB0446E0B9C4
:1092B000E8780EF0C1FCD8F808730646002FBBDD35
:1092C000DFF83C8002E00134BC42B5D004EB440539
:1092D00018F805000EF0B0FC8642F4D1214608EBE8
:1092E000050000270EF018FDA7E7306986F8D84082
:1092F00044F060FAA1E700BF40420F007818012057
:10930000841B012030B490F8443000F10801474A32
:10931000012BC2F83C136ED083684549DC68454D8B
:1093200024F46004AB42DC60DC6844F46004DC607C
:109330009C6B24F440149C639C6B44F480149C63E9
:109340009C6B24F4F8449C639C6B44F488449C63B9
:109350009C6824F470249C609C689C609C6824F445
:1093600040149C609C689C605C6824F480645C6031
:109370005C6824F480545C605C6901EA0401596112
:109380005969596145D0DC68294924F0E064DC6002
:10939000DC6844F0E064DC609C6B24F440149C6363
:1093A0009C6B44F480149C639C6B24F478249C6331
:1093B0009C6B44F410249C639C6824F470249C608F
:1093C0009C689C609C6824F440149C609C689C6031
:1093D0005C6824F480645C605C6824F480545C60A5
:1093E0009C692140134C9961A3429969996116D0F7
:1093F000002380F844301048104B848DC18D408D7F
:10940000091B93FBF1F3C2E9D004C2F8483330BC26
:1094100070470B4C616841F400016160B3E7084993
:109420004B6843F400034B60E2E700BF781801206B
:1094300000F0FFFF00200140007AF01F803801009B
:1094400000230140704700BF01483AF0A9BB00BFAC
:10945000001A0120084810B4D0F88831D0F8BC4177
:1094600099691A682CB1234600F5C4705DF8044B65
:1094700018475DF8044B70477818012001483AF00E
:109480008FBB00BF601A0120084810B4D0F8E83143
:10949000D0F81C4299691A682CB1234600F5F47083
:1094A0005DF8044B18475DF8044B704778180120AD
:1094B00001483AF075BB00BFC01A0120084810B43B
:1094C000D0F84832D0F87C4299691A682CB123460A
:1094D00000F512705DF8044B18475DF8044B7047B7
:1094E000781801202DE9F84FD54F6023044603FB7F
:1094F0000073D3F87451002D00F0A081D3F87C6183
:109500001EB1B379002B40F09981602303FB0473F3
:10951000D3F88091B9F1000F04D099F80630002BF0
:1095200040F08C81631CDBB216B11522F371B2716D
:10953000B9F1000F04D0162289F8073089F8062007
:10954000287C4FF009083FF029F930460DF074FEF1
:1095500048460DF071FE112130460EF0D9FB112165
:1095600048460EF0D5FB4FF0330A02E00A2011F016
:109570005FFC26B13368B2881B691A4202D1BAF186
:10958000010AF3D130460DF051FE052011F050FCD8
:1095900030460DF051FE052011F04AFCB8F10108EB
:1095A000E1D130464FF0600B0DF040FE052011F088
:1095B0003FFC48460DF03AFE0BFB04FB052011F082
:1095C00037FC30460DF038FE07EB0B0A052011F092
:1095D0002FFC48460DF030FE9AF8843130460422C4
:1095E000002B984E14BF3E211E210EF071FB9AF8FD
:1095F00084315E444846002B4FF00402C14614BF3C
:109600003E211E210EF064FB4C224146304646F0BE
:109610004BFEDAF874319FED8C7AB0EE084A5B6845
:10962000F7EE003ABAF886B1CAF88831874B9FED59
:10963000885A9A68874BC2F38222134493F8042213
:10964000D7F86C31D34007EE903AF8EE677AC7EE60
:10965000275A07EE90BA9FED807AF8EEE77AC7EEC8
:10966000274ADFED7E7AB0EE007AE5EE877AA5EE46
:10967000875A25EE844A37EE856A74EEE72ABBF5F1
:10968000C87F40F2145309F1010ED7BF19463223A7
:1096900064234FF49670C8BF782007EE90EAD4BFD9
:1096A0004FF4167C4FF4827C0344B8EEE77AC8BFCF
:1096B0004FF4FA7107EE903A27EE257A01EB0C038E
:1096C000F8EEE76A86EE873A73EE636AFCEEE67AB6
:1096D00017EE902A07EE90CAB8EEE73A07EE903AF6
:1096E000F8EEE77A23EE243AC3EE276A36EEC53A5F
:1096F00072EEE66AC3EE077A77EEE37AFCEEE77A7B
:1097000017EE901AC6EE877A77EEE37AFCEEE77AE8
:1097100017EE903A03F1020C0CEB010AF0EE466AE8
:1097200007EE90AAF8EE677AE7EE276AF4EEE64ACB
:10973000F1EE10FA00F398805FFA82FCBCF10F0F93
:1097400000F29480323807EE900AF8EEE77A77EE6E
:10975000C47AC7EE876AFCEEE67A17EE90CA5FFA23
:109760008CF00F2800F2828088B2FF287ED898B251
:10977000FF287BD840EA097310054FEA0C4200F03D
:109780007F6002F47F0203431343354A02EA01215A
:1097900043EA01086020012300FB047400273046DF
:1097A000C4F88C81C4E96473C4E96677C4E9697755
:1097B00043F0A8FC94F8C931202BD9B21AD194F8FF
:1097C000C831012B16D0242384F8C931D4F888314C
:1097D0001A6822F001021A601A6822F480521A6094
:1097E0001A681A601A6842F001021A6084F8C911F6
:1097F00084F8C871002195F912003FF0B3FA95F989
:109800001230AA7C002B07DB02F01F0101225B094A
:109810008A40144941F82320002195F911003FF0B6
:10982000A1FA95F911306A7C002B07DB02F01F01C9
:1098300001225B098A400B4941F82320BDE8F88FDB
:1098400078180120001A0120286B6E4E0038024063
:1098500000001643100605080024744900007042F9
:1098600000FFFF0000E100E0013155E7BEF10F0FFE
:1098700090D0F14603E700BF0248036903B11847DF
:10988000704700BF000001200248436B0BB1243039
:1098900018477047000001200248836D0BB1483023
:1098A00018477047000001200248C36F0BB16C30AD
:1098B00018477047000001200348D0F8A0300BB1D2
:1098C00090301847704700BF000001200348D0F8CF
:1098D000C4300BB1B4301847704700BF00000120FE
:1098E0000348D0F8E8300BB1D8301847704700BFB4
:1098F000000001200348D0F80C310BB1FC301847B0
:10990000704700BF000001200348D0F8303113B188
:1099100000F5907018477047000001200348D0F808
:10992000543113B100F5A2701847704700000120B0
:109930000348D0F8783113B100F5B4701847704778
:10994000000001200348D0F89C3113B100F5C67027
:1099500018477047000001200348D0F8C03113B108
:1099600000F5D87018477047000001200348D0F870
:10997000E43113B100F5EA70184770470000012088
:109980000348D0F8083213B100F5FC70184770474F
:10999000000001200348D0F82C3213B100F5077005
:1099A00018477047000001200138064A064B00EBBB
:1099B000C00052F8200098420CBF952096203EF03F
:1099C000EDBE00BF0000012000600240013800EB46
:1099D000C000F8B54FEA800C104C1D46104B54F8EF
:1099E0000C00174664440E4698420CBF9520962002
:1099F0003EF0D4FE94F91500B9092661A5613FF047
:109A0000B1F994F91530002B07DB03F01F00012298
:109A10005B090449824041F82320F8BD0000012081
:109A20000060024000E100E0AA4B2DE9F04F97B042
:109A300093F85E83A84B0025A84F0093A84BA3F290
:109A4000547ADFF8B092DFF8B0B24E46B30AA3F50D
:109A50008013522B55D8534493F80C320D2B50D809
:109A6000B8F1010FFC5640F01C81012C3FD14FF0A2
:109A700000094946204611F04BFE11F0D1FE90F846
:109A800000C0BCF1000F18BFBCF1540F14BF4FF061
:109A9000010C4FF0000C40F0008109F104091FFA9D
:109AA00089F9B9F1100FE4D1002D00F0B9808A4A8C
:109AB00000210DE0534493F80C320D2B0FD8FB56C8
:109AC000A3420FD0013102F58672A94280F2A48030
:109AD000906803689B0AA3F58013522BEAD90023F0
:109AE000A342EFD143799BF805009842EAD17C4B21
:109AF0005B4513D05BF8206FB30AA3F58013522B9C
:109B0000A9D9B8F1010FF2D001230024B8F1020F56
:109B1000ADD1002BABD0724B5B45EBD1009B013537
:109B200003F58673042D00938BD16E4B4FF0010823
:109B3000DFF8C8B1009303F57C73ABF1080A059315
:109B400008F1FF33DAF804209A4262DDDBF80C609A
:109B5000002E00F0D4833168B78801F13F41B7FA95
:109B600087F701F57E01C7F11F07890ADAF8105659
:109B7000002D40F3C780584B002405E0013403F565
:109B80008673AC4200F0BC801A688A42F6D14FF46A
:109B90008673514ACBF8047003FB04245FFA88F300
:109BA000CBF8184016B1F3710323B3717A00032187
:109BB000012301FA02F0A16C03FA02F20143A1644D
:109BC000216D0A4322659AF80020002A6ED0626D4A
:109BD000BB401A43626516B13268B188916199B28F
:109BE0000122D4F8AC00FEF70BFA204608F1010878
:109BF000FEF7BCFA0123009AB8F1090F8BF81C306C
:109C00000BF1200B0BF8033C537402F11803009383
:109C100096D117B0BDE8F08FBCF1000F7FF467AFAD
:109C200058460DF089FF9BF80540C3B2022B00F2A5
:109C30006E83431C2C4A5BB203EB430398002B4B0F
:109C400003F5727104E0994200F0618353F82C2F00
:109C5000B242F8D11A79A242F5D11A58002AF2D0AC
:109C600094460023224A51680133614512D0102BDB
:109C700002F12402F7D14FF0FF3303EBC3031C4A78
:109C800002EB83031B7F002B7FF431AF009BC3F8F3
:109C900008B043E7DBB2013BEFE7002D7FF407AFED
:109CA00025E7B4F1080318BF01232FE707F11002DD
:109CB0009340626D134363651EB1B38832681B0421
:109CC000936101210022D4F8AC00B94089B2FEF7BB
:109CD00097F98AE7781801209C070020287B05085F
:109CE000640D0508E015002000000140700805081B
:109CF0000000012000040140640C050888010020D8
:109D0000032C6CDC4FF4867303FB05A3D3F8240605
:109D1000002800F0EA82C3F81C160131CAB283F8A9
:109D200025270292542283F824276B1C0268CAF864
:109D30001036447901920DF0FFFEA84B864693F849
:109D4000733303939BF810300493C3B2022B00F2D9
:109D5000DE8200F1010CA249A24800234FFA8CFCDC
:109D6000019A0CEB4C0C4FEA8C0C05E00133172BDD
:109D700000F0CD8251F82C0F8242F7D10879A04231
:109D8000F4D151F80C000028F0D02C210EEB4E0E2F
:109D9000DFF8589201FB03F393494C4603EB8E0323
:109DA0000B44D3F870124FF4867303FB05A3C3F87A
:109DB00034160021C3F83006636898421ED0013182
:109DC00024341029F8D1894B13F8083C5BB9874A31
:109DD0005423029902F8083C02F8071C03E003230D
:109DE0007E4A82F87233824B82488349834AC3E9B0
:109DF000D310C3F8582317B0BDE8F08F4B1C7B4934
:109E0000DBB2013B03EBC30301EB8303197F069134
:109E10000029E8D1029959774FF4867101FB05F0CA
:109E20008C210446542018772046A310744C0190CE
:109E3000504404FB03F33468C0F81417C0F82046FC
:109E400003FB01F1059C03EB430304EB410103EB2E
:109E50000313C0F810176B4901EB8303C0F8C83631
:109E60003323C0F8CC36684B01981C185B4BD3F8F1
:109E70006C11039B062B00F03382072BDFF898C18F
:109E8000624B634814BF4FF0710C1846614B04BF1E
:109E900063464FF01C0CB1FBF3F3B1FBF0F1013B57
:109EA000104601399AB24FF4867303FB05A3A3F859
:109EB000D016A3F888260293019B2266002203F1A4
:109EC0005801514BA4F8582062661944E265484A8B
:109ED00042F8C4CC41F060FE029BD3F824261068FF
:109EE0000292036843F08003036053790C2B08D877
:109EF000DFE803F06C070707640707075B0707073E
:109F000052004FF4867303FB05A3D3F828164FF0D5
:109F1000600C026800234FF0020ECDF838C04FF4F9
:109F2000807C22F001021093CDF850C04FF0010C5C
:109F30001393CDF83CC04FF00A0C1593CDE911CE28
:109F400002600EAA41F0E6FC4FF48672029B02FB0F
:109F500005A2D2F828161A680023012900F088818A
:109F6000042900F08581102900F0C481402900F007
:109F70007F81B1F5807F51D0B1F5806F4ED0B1F5C2
:109F8000805F00F0C081B1F5803F4FF03C030CBF13
:109F900008214FF4006143E04FF486734FF4805181
:109FA00003FB05A3C3F82816B1E74FF486734FF4FB
:109FB000807103FB05A3C3F82816A8E74FF4867346
:109FC000102103FB05A3C3F82816A0E74FF48673FE
:109FD000012103FB05A3C3F8281698E77818012090
:109FE0007008050800000140100605080000012067
:109FF000781200209D56010899560108A5560108BF
:10A000006B4CA407A01600209C07002010552200CE
:10A0100044950800D0DD060040771B00082104238A
:10A0200002F1180050F803C041EA0C01C150029B34
:10A030001879002840F025814FF48672002302FB36
:10A0400005A2D2F82406D2F830160068026842F061
:10A0500001020260D9F804200133914200F00D8121
:10A06000102B09F12409F5D14FF0FF33AB4A03EB74
:10A07000C30352F82300AA4B98420CBF95209620A8
:10A080003EF08CFB4FF4867303FB05A3D3F8242624
:10A0900053790C2B00F2EE80A24901EB4303B3F895
:10A0A0007CC74FF4867310689F4903FB05A3A3F890
:10A0B0002CC6002306E0904200F01F810133042BE0
:10A0C00000F0288151F83320002AF4D1DAF818265C
:10A0D0000132CAF818260AEBC302DB00C2F84C0AA8
:10A0E0001944069823469022B1F804E0DFF8509214
:10A0F0004CEA0E0CA1F804C08C49FFF767FC6069BC
:10A100004FF486734FF4804C03FB05A5036843F0BE
:10A1100010030360036843F0140303600023C4E9E1
:10A120001F33C4E92833C4F8A8300423D5F83426F3
:10A13000C4F89C304FF48063C4F894204FF440324C
:10A14000C4F88430C4F898204022A267D5F8CC2601
:10A15000C4F89020C2B2D5F8201620F0FF00103AC3
:10A1600018312167A9FB0231019B4FF48052090984
:10A17000C4F8882003F170026D4B1A44D5F8C83634
:10A18000C4F88CC0636742F015F8D5F83006019B1F
:10A190004FF40031D0F800E04FF4006C03F1B80246
:10A1A000634BC4F820E0D0F814E01A440023C4F84C
:10A1B00024E0D0F804E0C4F828E0D0F808E0C4F8BF
:10A1C0002CE0D0F80CE0C4F8C830C4F830E0C4F893
:10A1D000F030C4E93033C4E93A33D5F8343601936A
:10A1E0000423C4F8E4304FF48063C4F8CC30019BFE
:10A1F000C4E93731D5F81437C4F8D830C3B220F0E9
:10A20000FF00103BA9FB0331D5F82036C4F8D0C0BD
:10A2100010330909C4F8B830D5F8103701934FF45A
:10A220008043C4F8D430019BC4F8BC3041F0C2FF75
:10A23000D5F830265FFA88F3116861635169A1632C
:10A240005168E16391682164D1686164116841F0EB
:10A2500010011160116841F014011160049ACBF8EB
:10A2600004708BF81020CBF80C60CBF818409AE4FF
:10A270000821D5E64FF0000C13E7DBB20693013B53
:10A28000F4E603920DF0D8FC039A20B30268254B44
:10A2900002F13F42079002F57E0203EB9222029BFD
:10A2A00092F874071A7A03923EF078FA079B039AA1
:10A2B00099880D92002218680C92089108A90393BE
:10A2C000CDE90A220222099241F0EAFC5422039BC2
:10A2D000DA80029B1A68536C43F400435364ABE684
:10A2E00014484FF0380C144BD5E50223134A82F87A
:10A2F000723378E54FF4006192E6DB00F0E64FF050
:10A30000FF37394632E44FF40061042388E6002326
:10A310005B68FFDE00239B88FFDE00BF000001209A
:10A320000060024010060508CC0B00204D8000089C
:10A330009C070020882A1100A0BB0D00781801207E
:10A34000ABAAAAAA2DE9F041834DC0EB001605EB9C
:10A35000C606D6F87433002B00F0BC800446070113
:10A3600096F8E4033EF01AFA96F8E433012203F07B
:10A370001F015B09013B8A40032B0AD8DFE813F079
:10A38000E0000400E600DA0074494B6A23EA0202A6
:10A390004A623B1B04F1010805EBC3035FFA88F82E
:10A3A00093F878030DF048FC18B1122380F8078069
:10A3B00083713B1B05EBC30393F879030DF03CFC61
:10A3C000064618B1132380F8078083713B1B05EB09
:10A3D000C30393F87A030DF02FFC18B1142380F80F
:10A3E000078083713C1B2E21304605EBC40494F892
:10A3F0007C230DF06DFC94F87A030DF01DFC94F8AD
:10A400007D230E210DF064FC94F878030DF014FC0C
:10A4100094F87B232E210DF05BFCD4F87433504963
:10A420001A688B4222F040021A6055D04D4A93427E
:10A4300069D002F58062934258D1484A116A41F4CA
:10A4400000411162116A21F4004111625A6842F41C
:10A4500080525A601A68520634D443491E68D1F8B3
:10A460005442D1F86002D1E99025B0F5005F42EA8C
:10A470000502D1F84C5242EA0502D1F8505242EAA4
:10A480000502D1F8585242EA040242EA0502D1F824
:10A490005C5242EA0502354D42EA000205EA060531
:10A4A00042EA05021A60D1F848225D6842EA144285
:10A4B0002F4C04EA050442EA04025A6002D1B1F8C2
:10A4C00064221A61DA6922F40062DA611A6842F0E1
:10A4D00040021A60BDE8F081204A516A41F480517F
:10A4E0005162516A21F480515162AFE7214A93428F
:10A4F00013D11A4A516A41F400515162516A21F450
:10A5000000515162A2E7154A116A41F4804111627B
:10A51000116A21F48041116298E7174A934295D15C
:10A520000E4A516A41F480115162516A21F480113E
:10A5300051628BE709490B6923EA02020A6128E7A5
:10A5400006494B6923EA02024A6122E703490B6A82
:10A5500023EA02020A621CE7781801200038024050
:10A560000030014000380040000001204000FFFFA3
:10A57000FBF0FFFF003401400050014030B404699B
:10A58000002341684025E46882690C3154624469C3
:10A590009560536093631160C2E90333C2E90533E8
:10A5A000C2E90733C2E90A33C2E90C3384B1C26994
:10A5B000E068936350621160C2E90133C2E903337A
:10A5C000C2E90533C2E90733C2E90A33C2E90C33F1
:10A5D00030BC7047114A037A0168D35C10B4CC5880
:10A5E000CA1824F00104CC501368DB07FCD4037DA7
:10A5F0001F2B09D9203B20225DF8044B02FA03F3FC
:10A6000043F01803CB60704720225DF8044B02FA38
:10A6100003F343F018038B60704700BF387B0508D5
:10A62000F0B50668356A00295CD12F68AC68D6F8A9
:10A6300018E0002F5FD0364B3B40B3F1005F61D094
:10A6400007F01F0104F11F0327F01F02194421F036
:10A650001F01BFF34F8F00290BDD114402F12003CE
:10A66000DFF8B0C08B42CCF868221A4603F1200311
:10A67000F8D1BFF34F8FBFF36F8F03684FF4806241
:10A68000CEF80470CEF814205B69CEF8204043B3B6
:10A690006868F669002837D01D4B0340B3F1005FAE
:10A6A0001AD000F01F0220F01F011F32224422F0B6
:10A6B0001F02BFF34F8F002A0ADD0A4401F1200375
:10A6C000144D9A42C5F87012194603F12003F8D1CF
:10A6D000BFF34F8FBFF36F8F4FF480637060736170
:10A6E0003462F0BDEC69002CFBD06F691435D6F8EC
:10A6F00018E0002F9FD1084A3346CEF81470CEF8E8
:10A700000420C1E73346B9E7044B70617360E7E7A3
:10A710000000FFFF00ED00E0180000201C000020FA
:10A72000F8B507680646D7E90454002C50D0A0615C
:10A730002B7D1F2B39D82022286802FA03F343F01F
:10A7400018038360237D1F2B3AD92022203B02FA75
:10A7500003F3226843F01803D3606368002269683A
:10A760000A601A601A6842F010021A60BA69297AFF
:10A7700041F020FDFA69217A206841F01BFD2A7A18
:10A780002A492F6833688D5C5A687B59206843F0EA
:10A7900001037B51237AC95C435843F001034350C2
:10A7A000536843F003035360F8BD203B2022286820
:10A7B00002FA03F343F01803C360237D1F2BC4D8B0
:10A7C000202202FA03F3226843F018039360C4E7DF
:10A7D0002A7D6B681F2AA8611FD82021286801FAEA
:10A7E00002F242F0180282600021BA691960196809
:10A7F00041F010011960297A41F0DCFC2A7A0B49FA
:10A8000033682868895C5A68435843F00103435011
:10A81000536843F002035360F8BD203A20212868B2
:10A8200001FA02F242F01802C260DDE7387B050847
:10A83000014B43F82010704750280040F0B5A24C5F
:10A84000A5B0E368022B00F03A82A048A04AA149D3
:10A85000121A45F0B5FCA048A04AA149121A45F0C9
:10A86000AFFCA368012B00F2C28003EB43039D4AB7
:10A870009D4D02EB430032F8132041888388C5E9DF
:10A880009A21C5F87032994C994E9A4BB2FBF1F26D
:10A89000994901FB02F20021C6F86C21D4F8882006
:10A8A00042F47002C4F888201A6842F001021A606B
:10A8B0009960924A1868024091481A60C0F30807EC
:10A8C000904A5A601A6822F480221A60D96007B14F
:10A8D000FEE78D49A0604FF6FF000A688B4B42F4FB
:10A8E00000720A60E26802401343E3603EF0CEFA71
:10A8F000BFF34F8FBFF36F8FC4F85072BFF34F8F0A
:10A90000BFF36F8F636943F400336361BFF34F8F0D
:10A91000BFF36F8FC4F88470BFF34F8FD4F88030CB
:10A9200043F6E07CC3F3C90EC3F34E33580100EA8B
:10A930000C01734641EA8372013B5F1CC4F860223C
:10A94000F8D1203810F1200FF1D1BFF34F8F636998
:10A9500043F480336361BFF34F8FBFF36F8F6A4956
:10A96000644B0A6842F480720A60196C684A41F0CC
:10A9700080511964196C01F080510291029911689B
:10A9800041F4404111601268D5F8680202F4404277
:10A99000D5F86C42D5F870120192019A9A6802F0CB
:10A9A0000C02042A00F08D809A6802F00C02082A3A
:10A9B00000F083804F4A136843F480331360D6F865
:10A9C000F47204E0D6F8F432DB1B642B74D81368FD
:10A9D0009B03F7D5474A936803F00C03082B6BD011
:10A9E000136823F080731360D6F8F47208E03E4DCC
:10A9F000D5E99A2147E7D6F8F432DB1B022B5BD866
:10AA000013689B01F7D40B06640843EA8013611EA8
:10AA100043EA01433F491943364B5160116841F005
:10AA200080711160D6F8F41204E0D6F8F422521ABC
:10AA3000022A41D81A689201F7D5196C344A41F0BC
:10AA4000805119641B6C03F080530393039B1368BC
:10AA500043F480331360D6F8F41206E0D6F8F432EB
:10AA60005B1AB3F57A7F00F2CB805368DF03F5D52C
:10AA70001368274943F400331360D6F8F42206E044
:10AA8000D6F8F4329B1AB3F57A7F00F2B9804B689E
:10AA90009C03F5D54FF400124FF0006304A8049214
:10AAA0004FF4C07221930723CDE9082303230A93AF
:10AAB00039F060F980B3FEE7FEE75B685A027FF584
:10AAC00079AF0C4B1B6885E7502800400000000060
:10AAD00088370000440106080000002080010020A3
:10AAE0000C530608A80D05080000012000ED00E049
:10AAF000781801200038024040420F00FFFFF6FEA8
:10AB00000000000810300024003C02400003FA0559
:10AB100000700040080040206C4A136803F00F03E7
:10AB2000062B0AD8136823F00F0343F007031360C2
:10AB3000136803F00F03072B63D1654B9A6842F447
:10AB4000E0529A609A6842F460429A609A6822F0F1
:10AB5000F0029A601A68900153D59A6841F28831E0
:10AB600022F0030242F002029A60D6F8F40204E0F6
:10AB7000D6F8F422121A8A4243D89A6802F00C02DC
:10AB8000082AF5D1514A136819070AD5136823F02A
:10AB90000F0343F007031360136803F00F03072B41
:10ABA0002FD14B4C4B4FA36823F4E05343F4A053F5
:10ABB000A360A36823F4604343F40043A36039F027
:10ABC000A5F8A368C3F303133B4493F8A437D84014
:10ABD000C6F86C013EF05AF9002304A8CDE91333FE
:10ABE000CDE91533CDE91733CDE91933CDE91B3361
:10ABF000CDE91D33384B049339F0BCF810B1FEE7B2
:10AC0000FEE7FEE702234FF0007204A8CDE9063309
:10AC1000D823CDE9042301230B9339F0ABF800B11D
:10AC2000FEE7D4F88C3023F08073C4F88C30D4F86D
:10AC30008C3043F08073C4F88C30A36803F00C03AD
:10AC4000042B36D0082B18D0244BC6F86C31204A80
:10AC5000D5E99A31B3FBF1F39168D6F86C21C1F3D1
:10AC600003110F4497F8A417CA401D4901FB03F3D1
:10AC7000C6F86C21934220D0FEE76368626813F443
:10AC8000800F636802F03F0218BF1649C3F38813B0
:10AC900008BF1249B1FBF2F202FB03F30C4A5268FF
:10ACA000C2F3014201325200B3FBF2F3C6F86C3139
:10ACB000CDE70C4BC6F86C31C9E725B0F0BD0021DB
:10ACC0000320FFF7B5FDFEF7A1FA00BF003C0240EC
:10ACD0000038024010060508C0FF03000024F400FD
:10ACE00040420F0000127A001D4B1E48196C1E4A8C
:10ACF00041F0805130B4196482B0196CFF2401F026
:10AD0000805101910199016841F480710160CA206C
:10AD1000196C41F480611964196C01F4806100912F
:10AD20005321009D5462506251625B6FDB000DD471
:10AD30000E4B00210E4A43F8041B9342FBD10D4BEE
:10AD40000D4AC3F8502802B030BC7047094A0A4B7C
:10AD5000D2F850289A42EBD102B030BC704700BF05
:10AD60000038024000700040002800405428004095
:10AD70006C2800400020004031666542800AA0F542
:10AD80008010522808D8054B184490F80C320D2B2F
:10AD900002D8034AD05670470020704710060508B5
:10ADA000287B0508F0B50446D0F89400434B83B0E7
:10ADB000A16804F1640204F118070E68C1B220F022
:10ADC000FF0001921039A3FB0131090941F03CFA5F
:10ADD000616D0023019A012984F8583018D00429A4
:10ADE00016D0102955D0402912D0B1F5807F53D00C
:10ADF000B1F5806F50D0B1F5805F55D0B1F5803F8F
:10AE00004FF03C030CBF6FF0080C6FF4006C01E0D6
:10AE10006FF0080C06F118053046E95801EA0C01FC
:10AE2000E950616D40F076FD636D012B16D0042B67
:10AE300014D0102B0FD0402B10D0B3F5807F2FD023
:10AE4000B3F5806F2CD0B3F5805F31D0B3F5803F80
:10AE500006F1540502D04FF4006100E008212B6890
:10AE60003A46D4F894000B4340212B602162C1B2D2
:10AE7000124B20F0FF001039A3FB0131090941F00A
:10AE800099F9D4F89420136843F01003136003B0C9
:10AE9000F0BD6FF4006CBDE76FF0080C0423B9E758
:10AEA00006F11C050821DAE76FF4006C0423B1E712
:10AEB00006F11C054FF40061D1E700BFABAAAAAAB6
:10AEC000934B2DE9F04F1C782DED028B85B034B9F2
:10AED0000124204605B0BDEC028BBDE8F08F8D4B00
:10AEE0008D4F1B6D08EE103A0DF000F997F8E43B1A
:10AEF0000190002B00F00681854B07F1480AA7F16D
:10AF0000C004002603F5887B5D46CDF80CB0D7F869
:10AF10003033019AD31A03D4EA6D9A4200F3D580F4
:10AF20007B4A06EB860302EB431393F8683103F088
:10AF3000FF020092002B00F08E80D5F89410AB68D1
:10AF400076481A68CBB221F0FF01103BA0FB030347
:10AF500073481B09C35C19444B68A9891FFA83FE17
:10AF6000D368CEF1160E23EA0103BEF1070FD360BA
:10AF700071D957F8B83C00220121013390468B4625
:10AF800047F8B83CD5F89C309C4602935CF8049B8B
:10AF900048461DE0DCF80090B8F1140FA9EB00035F
:10AFA00048461EDC13F1080948BF03F117094FEAB0
:10AFB000291308EB291803F1FF39013102FA03F3D1
:10AFC0000CF1040C0BFA09F28E4542EA030208D395
:10AFD0008E45DFD8C8F11503DCF800004FF01508E6
:10AFE000E9E7B8F1150F67D14E49C2F38423C2F3E4
:10AFF000441001EB830301EB8000D3F8B437D0F8A1
:10B00000B4071B0243EA001302F01F00C2F3C4326C
:10B0100001EB800001EB8202D0F8B417D2F8B4271C
:10B020000B4343EA023383EA132282EA121202F04C
:10B030000F020F2A40D1C3F30F134FF6FF72934252
:10B040003AD0B3F5606F47D0A381009918EE102A6B
:10B0500050460CF091F828460136FFF7A3FE97F80A
:10B06000E43B0AF15C0A1434B34205F1A0053FF752
:10B070004EAF01210022DDF80CB087F84610C7F86A
:10B080003023002B3FF424AF03EB83030BEB43137C
:10B090009BF810200BF1A00B5BF84C0C12F0020F88
:10B0A0005BF8982C11680A6A14BF42EA80020243D6
:10B0B0005B450A62ECD10BE757F8BC3C013347F81B
:10B0C000BC3CC6B100230093BFE70024204605B076
:10B0D000BDEC028BBDE8F08F0E4991F8FC2002EB2D
:10B0E000420201EBC202324492F8A9200D2AABD1F0
:10B0F0008023A377A9E7029958220B4845F060F80E
:10B100000096A2E70122C7F8303387F84620E0E630
:10B11000800100207818012078120020ABAAAAAA8A
:10B12000387B05081006050864120020830AA3F581
:10B130008013522B45D8F0B50446624885B00344CD
:10B1400093F80C020D283AD85F4D860105EB801369
:10B15000D3F85475A74232D00139C3F8544589B2A7
:10B16000C3F86015D5F86C11B1FBF2F2013AC3F8DF
:10B17000582505F2545202EB80100022C3F86425D2
:10B18000C3F85C25C3F8682539F05AF84F4B9C4248
:10B1900018D0B4F1804F15D0A3F57C439C4272D0F7
:10B1A00003F580639C426ED0494A03F57C439C4280
:10B1B00018BF944246D003F570539C4242D005B06C
:10B1C000F0BD704700234FF48051AA19CDE9001358
:10B1D00092F890150129CDE90233F0D00221D2F87E
:10B1E0005405012482F891153A49876839408160F5
:10B1F00082F8914582F890350023AA19CDE90033F1
:10B20000029392F89035012BD9D0D2F8543502210F
:10B210002E4882F8911583425A6899684ED000F5FD
:10B22000806083424AD022F0700221F080013544D0
:10B2300001205A609960002385F8910585F89035C2
:10B2400005B0F0BD00214FF48053CDE90031AB19BA
:10B2500093F89025012ACDE90211B0D0D3F8540516
:10B26000022283F891251B4A87683A4082601A4A75
:10B2700083F890150121944283F89115BCD0144BAA
:10B280009C429CD1B8E700224FF48051AB19CDE924
:10B29000001293F890150129CDE902228FD00221E6
:10B2A000D3F85405012483F891150A498768394079
:10B2B000816083F8914583F890259DE722F4700220
:10B2C000B1E700BF10060508781801200000014012
:10B2D000000C00408800FEFF0004014003689B0A48
:10B2E000A3F58013522B58D8F0B53D4C234493F866
:10B2F0000C320D2B50D84479A608002952D003EB0C
:10B300008300384D4FF0020CA40803EB40000CFA08
:10B3100004F4304405EB8316D6F8546505EB800C35
:10B32000F768CCF818193C43CCF82829F4609C0144
:10B33000EFF3118C502282F312882C2203FB02F2CD
:10B34000A818D0F8141949B30A1DC0F838192649AD
:10B350002C20264E03FB00F006EB000E14300144B7
:10B3600051F8040B18B1106051F8042C04328E45CA
:10B37000F6D100215FFA8CFC11608CF311882C222D
:10B380002C4402FB0353D4F85425D3F8383913B3B3
:10B39000D36843F00103D360F0BD704724321249F3
:10B3A0000A44D5E703EB83000E4D344603EB40001F
:10B3B000304405EB8316D6F854750226A640FC6887
:10B3C00024EA0604FC6005EB8004C4F81819C4F8EC
:10B3D00028299C01ACE7D36823F00103D360F0BDBA
:10B3E00010060508781801208C210120B0210120C9
:10B3F00001490248FDF7E2B98C210120000001401B
:10B4000010B5064C064804F61411FDF7D7F904F5FB
:10B410002A610448BDE81040FDF7D0B97818012032
:10B42000000001400044014002494FF08040FDF718
:10B43000C5B900BFB821012001490248FDF7BEB9D6
:10B44000E42101200004004001490248FDF7B6B99B
:10B45000102201200008004001490248FDF7AEB962
:10B460003C220120000C00402DE9F843194E3569BB
:10B47000F3681D4010D04FF00047DFF85C80B5FA4C
:10B4800085F227FA02F31F2A6FEA030305EA030590
:10B49000336103D0002DF2D1BDE8F883D8F8183A13
:10B4A000A3B103F1FF3900231FFA89F9C8F8183A4C
:10B4B000D8F8144A002CEDD0236820464946984716
:10B4C0006468002CF8D1002DD9D1E5E7F16A1FFAA4
:10B4D00081F9EDE700100040781801200149024889
:10B4E000FDF76CB9C02201200004014010B5064CE4
:10B4F000064804F64821FDF761F904F624310448B2
:10B50000BDE81040FDF75AB9781801200004014049
:10B51000001C004001490248FDF750B9EC2201200F
:10B520000040014001490248FDF748B94423012089
:10B530000048014001490248FDF740B9702301204D
:10B54000001800402DE9F04F4FF4257295B000210E
:10B55000804844F0A9FE804B804F4FF080415A6CE8
:10B5600007F12004B94642F0010207F51E65A24624
:10B57000DFF8F4815A645A6C794E02F001020092AD
:10B58000009A1A6C42F001021A641A6C02F001026D
:10B590000192019A1A6C42F002021A641A6C02F0CB
:10B5A00002020292029A1A6C42F004021A641A6CA5
:10B5B00002F004020392039A1A6C42F008021A6421
:10B5C0001A6C02F008020492049A1A6C42F01002FB
:10B5D0001A641A6C02F010020592059A1A6C42F075
:10B5E00020021A641A6C02F020020692069A5A6C23
:10B5F00042F002025A645A6C02F002020792079A61
:10B600005A6C42F480325A645A6C02F480320892C6
:10B61000089A5A6C42F400325A645A6C02F40032AE
:10B620000992099A5A6C42F480225A645A6C02F4C4
:10B6300080220A920A9A1A6C42F040021A641A6C2A
:10B6400002F040020B920B9A1A6C42F080021A64CC
:10B650001A6C02F080020C920C9A1A6C42F48072FE
:10B660001A641B6C03F480730D930D9B42460023F8
:10B6700001E056F833208A420CD001330E2BF8D16A
:10B680000AF1200A00203DF089F855450DD05AF8FE
:10B69000201CEBE7334A0AF1200A02EBC30393F8BC
:10B6A00000013DF07BF85545F1D107F51C67DFF847
:10B6B000BCB0DFF8BCA009F120094F4526D099F8AD
:10B6C0000630002BF7D099F804000CF0B5FA0646C6
:10B6D0000028F0D0036809F1200919F8188C5344A8
:10B6E0000BEB932393F874073DF058F8B288306859
:10B6F00000230E9202220EA9CDF84C80CDE90F2333
:10B70000CDE9113340F0CCFA4F45D8D14FF080410C
:10B71000154F134E3A46002301E056F833208A4273
:10B720000BD001330E2BF8D1203400203DF036F839
:10B73000AC420CD054F8201CECE70A4A203402EB4F
:10B74000C30393F800013DF029F8AC42F2D115B0E3
:10B75000BDE8F08F8C21012000380240440E05081E
:10B760000418050808170508000001401006050820
:10B770000000FEBF08B572B6FDF748FD344BDB682C
:10B78000012B30B583B04BD0324C0025324A052313
:10B79000C4F89850C4F89C50C4F8A020C4F8943061
:10B7A000BFF34F8FBFF36F8F4FF6FF01E2682B4B54
:10B7B0000A4013432A4AE360536F38F0A7FA294B33
:10B7C0002949A3FB0023D4F8FC209B0C42F0807293
:10B7D000C4F8FC20C1F8A83BD1F86C312349244AB5
:10B7E000A1FB031323499B09C2F8B01F5560013B1D
:10B7F0001168B3F1807F41F00101116008D24FF070
:10B80000E022F0215361072384F82310956113612E
:10B810004FF0E022136943F00403136103B030BD1D
:10B8200002210320FFF704F80D4B13485A6C13490B
:10B8300042F480425A645B6C03F480430193019AA2
:10B8400002680B68026083F308884B689847FEE73C
:10B850005028004000ED00E01B0000060005FA053E
:10B860000038024083DE1B4378180120D34D62105C
:10B87000001000E055CEACC5003801400000F01FBC
:10B88000D0F82011242200232DE9F041C0F89421A2
:10B8900004460A68806804F5907522F001020A6087
:10B8A0000B604B608B6094F805C0C4F89C314FEA84
:10B8B0008C22C4F8943184F8903102F48052C4F898
:10B8C0009831C4F83831C4F828214FEA0C32C4F852
:10B8D000403102F40052C4F834312379C4F82C21E9
:10B8E0004FEA0C22C4F8240113F0010002F4806234
:10B8F000C4F8302102D00422C4F8342113F002032A
:10B9000005D0D4F8342142F00802C4F834211CF0E8
:10B91000010F0DD048B1D4F8442142F00202C4F81E
:10B9200044214FF48032C4F84C21002B40F0FF80BA
:10B93000A64B03F1200053F8042F944200F0BD8081
:10B940009842F8D11CF0080F40F0CD80D4F8943123
:10B95000002B00F0128124232846C4F894310B6890
:10B9600023F001030B6038F059FD012815D0D4F8FD
:10B970004431002B40F01481D4F8203128465A6815
:10B9800022F490425A609A6822F02A029A601A6859
:10B9900042F001021A6041F089FB2379DA0761D590
:10B9A000D4F8FC20002A00F0D5800023D4F804113C
:10B9B00004F13C06E263A3644FF480623046E26423
:10B9C000C4E91013C4E91433C4E91833C4E91A33C1
:10B9D0004FF48033E3654FF48073A36541F0E0FBDF
:10B9E000304637F0E7FDD4F89881C4F88C61B8F19F
:10B9F000200F656731D1E368626999B26AB3B1FA21
:10BA000081F77F0949B394F89001012825D0304689
:10BA10000126C4F89C710B4684F890612226A4F894
:10BA20007811C4F898616A4ED4F82011A667694E5F
:10BA30002431C4F87421E667674EC4F88C70C4F8EA
:10BA4000886037F055FE002800F0AE80102384F89F
:10BA50009071C4F89C31C4F89481E26B23795268E8
:10BA6000C4F814219B0773D5D4F80021002A69D0AB
:10BA70000023D4F8081104F19C06C4F89C20C4F8F3
:10BA8000A8304022C4F8B8303046C4E92C33C4E9A9
:10BA90003033C4E932334FF48033C4F8BC304FF450
:10BAA0008063C4E92812C4F8AC3041F079FB304619
:10BAB00037F080FD002863D0FEE7002C3FF442AF52
:10BAC00094F8B831002B3FF43DAFD4F844311CF06A
:10BAD000080F43F00803C4F844314FF40043C4F89E
:10BAE00054313FF433AFD4F89431002B51D0242398
:10BAF0002846C4F894310B6823F001030B6038F03A
:10BB00008DFC01283FF449AFD4F84431002B43D1D8
:10BB1000D4F8203128465A6822F490425A609A6834
:10BB200022F022029A609A6842F008022EE7D4F8C6
:10BB3000443143F00103C4F844314FF40033C4F8F6
:10BB40004831F5E6D4F8A021136843F08003136070
:10BB5000BDE8F081D4F8A021116841F48071116032
:10BB6000916841F001019160116841F0200111607C
:10BB7000116841F01001116074E784F89031EAE631
:10BB8000D4F89C30C4F88861C4F8D4505860BDE83B
:10BB9000F08184F89031AAE7284638F0F9FDB7E73C
:10BBA000284638F0F5FDE7E6D4F8203184F8900116
:10BBB0001A6842F480721A609A6842F001029A6030
:10BBC0009A6842F040029A6047E700BF641E002076
:10BBD000310804086108040865080408F8B5EFF3A3
:10BBE0001185502383F31288D0F800311B6813F0BD
:10BBF000010303D0EDB285F31188F8BDD0F894218C
:10BC00000446D0F898110A4302F02102212AF1D00B
:10BC1000D0E90901884253D043D822691846531A03
:10BC20009BB2D4F894710022A062202F84F8A42142
:10BC3000E0D1A2695118DDD0B3FA83F67609002B62
:10BC4000D8D094F89021012AD4D00122D4F88801C8
:10BC5000A4F8723184F890212122C4F89C61C4F8C0
:10BC60006C11A4F87031C4F89421E8B1DFF858C021
:10BC7000D4F82021C0F83CC0DFF850C02832066557
:10BC8000C0F840C0DFF848C0C0F84CC037F030FD05
:10BC900050B1102384F89061C4F89C31C4F89471B9
:10BCA000A8E7431A9BB2BCE7D4F820310022402118
:10BCB000196284F890219A6842F080029A6099E7AC
:10BCC000012384F8A43195E7090804082D08040825
:10BCD00065080408F8B5D0F820310446DA69910601
:10BCE00015D5586AE36AC0B2002B00F0D580216BED
:10BCF0009847D4F820311A6822F480721A609A6842
:10BD000022F001029A609A6942F008029A61DA69A7
:10BD1000D20701D501221A62DA69970701D50222FA
:10BD20001A62DA69560701D504221A62DA69150720
:10BD300001D508221A62D4F8002152B3D969490604
:10BD40000AD4DA69D20606D5626B12B19047D4F8EC
:10BD5000203110221A62F8BDD96904F590701E686E
:10BD60000F079D682DD18F0602D5B50600F1C8805A
:10BD70000F0602D5350600F1B380480602D57106DC
:10BD800000F1A38012B12046FFF728FFD4F820313C
:10BD9000D7E7D9690806D1D5D4F894112129CDD097
:10BDA000D4E90901814200F0A480A069405C01311E
:10BDB000C0B298622069B1FBF0F500FB1511A162D9
:10BDC000BCE705F0010506F4907C5CEA0507CFD0DE
:10BDD000CF0709D5F70507D501271F62D4F89C7155
:10BDE00047F00107C4F89C718F0761D44F0708D54D
:10BDF0003DB104271F62D4F89C7147F00207C4F8D4
:10BE00009C710F070CD506F0200C5CEA050507D0E5
:10BE100008251D62D4F89C5145F00805C4F89C51D2
:10BE2000D4F89C51002DADD08D0607D5B10605D5AF
:10BE3000D4F8802112B19047D4F82031D4F89C1165
:10BE40009A6801F0080102F04002114368D01A68B4
:10BE50002020002122F490721A609A6822F00102D8
:10BE60009A60C4F898019A68C4F88011520610D5F7
:10BE70009A68D4F88C0122F040029A6048B190F898
:10BE800035302A4A022B02653FD08023436534F0C7
:10BE900019FDD4F8002175E7E3696269D054E369BC
:10BEA000E2680133B3FBF2F102FB1133E36120E7F7
:10BEB000002DA6D002271F62D4F89C7147F004071A
:10BEC000C4F89C714F079CD593E71968202021F096
:10BED000400119600023C4F89401C4F8843151E78B
:10BEE000D4F88431002B3FF44DAF9847D4F80021AB
:10BEF00048E7A4F87221196821F0800119601DE754
:10BF0000D4F88031002BF0D13CE70168052380F89C
:10BF100035300B68D4F8002123F001030B6031E7C2
:10BF2000D4F80021C4F89C112CE700BFC508040810
:10BF30002DE9F04FAC4C89B004EB8004D4F8F04B01
:10BF4000002C6CD0D4F8A8511F46DFF8B0B2904650
:10BF50006B680646DFF8A892C4F8A0316B6BA1604D
:10BF600063612B6BA3616B8FE3600BF5B67323608A
:10BF70002B8F23612A7809EB420393F9AC0B530012
:10BF80000193C3B2012B40F2B480D4F800319BB1CD
:10BF900096494FF0000C9E46084643680CF1010C90
:10BFA00024309E4500F02E81BCF1100FF5D111F820
:10BFB000083C002B00F07781D4F8FCE0BEF1000FC4
:10BFC00040F0EB806B68C4F8203195F82800002819
:10BFD00040F0FB8094F8AE010BF02EFE17F0080B3A
:10BFE000814694F8ACA11ED0002841D017F0510F23
:10BFF0004FF00B0306F1010614BF0A211A2117F0B6
:10C00000410F8371C67114BF4023202394F8AF21E0
:10C0100019430BF037FED4F8FC30002B52D02046E9
:10C0200009B0BDE8F08F18F0020F21D000B302680C
:10C030006F49704B114403EB912393F874070B2362
:10C0400089F80630731C89F8073094F8AF713CF01A
:10C05000A5FBB9F8043002A9D9F800000293022325
:10C060000797CDF818B00393CDE904BB3FF018FE55
:10C0700050460BF0E1FD07460028CCD018F0010F28
:10C08000C9D001680C235A4A013683710A44594BBE
:10C09000C67103EB922394F8AD6193F874073CF0FA
:10C0A0007DFBBB88386802220293002302A9079611
:10C0B000CDE90323CDE905333FF0F2FDD4F8FC30A0
:10C0C000002BACD195F82C1095F92A0089093CF089
:10C0D00049FE95F92A3095F82A20002B9FDB02F0C3
:10C0E0001F0201215B09444801FA02F240F82320B3
:10C0F00095E708234FF00C0A0BF5CE7C1AFB003AAB
:10C100000023E64619460131182961D01EF81C3F6C
:10C11000042BF8D19EF801309342F4D15EF80A3036
:10C12000002BF0D08E460199C4F800318944CEEB43
:10C13000CE0199F9ADEB890000EB4009BEF1FF3F5C
:10C1400001EB89015944D1F8A811C4F808113FF452
:10C150001FAF0021013118293FF419AF1CF81CEF63
:10C16000BEF1050FF6D19CF801E09645F2D15CF8DE
:10C170000AE0BEF1000FEDD0C1EBC101C4F8FCE054
:10C1800000EB4000890001EB80008344DBF8A8113C
:10C19000C4F80411002B7FF4FBAE144900230A46B7
:10C1A00050680133243286455BD0102BF8D111F84A
:10C1B000083C002B7FF406AF2B78013301F8073CD5
:10C1C0000C2301F8083C6B68FDE63CF0E7FA01E758
:10C1D000019B9944D4F8003199F9AD1B0131B8D1D4
:10C1E000002B7FF4D5AEE7E6781200200000012096
:10C1F0000000FEBF1006050800E100E00817050872
:10C20000781801205FFA8CF9013209F1FF33D2B2BC
:10C2100003EBC30301EB830C9B009CF81C0000287C
:10C220007FF4CAAEC858234B8CF81D2098420CBF2F
:10C23000952096200B238CF81C303CF0AFFA234657
:10C24000484695F82B201C49FDF7C0FB6B68D4F8D5
:10C25000FCE02833C4F81831BEF1000F3FF4B2AE51
:10C260009BE7DBB22A78013B013203EBC303D2B276
:10C2700001EB830C9B009CF81C0000287FF4A2AE0D
:10C28000C8580C4B8CF81D2098420CBF9520962066
:10C290000C238CF81C303CF081FA6B6803F124020B
:10C2A000C4F81C218FE601320B2301F8072C01F89A
:10C2B000083C81E6006002404D8600084A1C4FF4AD
:10C2C000003310B408BF4FF0800C4C4C18BF4FF037
:10C2D000450C00E0FBB1626B013B12EA0C0FF9D098
:10C2E000002923DD626B52071CD403291ED0434A68
:10C2F000536B13F0010320D1022908D01369DBB27C
:10C3000083421ED1012953692BD006291BD000205E
:10C310005DF8044B7047002904DD636B5C0701D4B2
:10C320000329E4D103205DF8044B7047002B5DF82E
:10C33000044B14BF00200320704701205DF8044B1C
:10C3400070471020EFE713F4604F02D12C4AC2F877
:10C35000BC3B990431D45A04F3D41B04D7D50F2025
:10C36000E1E7284818400028DDD0002B29DB5C00DD
:10C3700025D4980029D4D90025D41A0129D45C01E8
:10C3800025D4D8012FD41902E9D45A02D9D49C0259
:10C3900027D4D8022FD419030FD45A0329D49C03CD
:10C3A00025D4D80321D4190419D45A0415D49C04D3
:10C3B00011D41807ABD51A20B5E71320B3E709202D
:10C3C000B1E71C20AFE70B20ADE70A20ABE70D205B
:10C3D000A9E70C20A7E71920A5E71820A3E7172055
:10C3E000A1E711209FE70E209DE716209BE715206F
:10C3F00099E7142097E7122095E700BF002C014031
:10C400007818012008E0FFFDF8B5164DD5F8E83B97
:10C41000A3B1D5F8F01B0446012915D0124B40F208
:10C42000FF500021DA6A22F00802DA629863C5F848
:10C43000E81B236823F001032360F8BD0A4AD36B8D
:10C4400043F48073D363F8BD074E40F2FF570023D7
:10C450000C20B763B36040F24C43F360FFF72EFF4C
:10C46000B763DBE778180120002C01402F4B1A68D6
:10C47000910102D59A6D52074BD42C4B1A68500289
:10C4800002D5DA6E11063CD4284B1A68D20102D5C7
:10C490009A6D90072DD4254B1A68510102D59A6DDB
:10C4A000120717D4214B1A68120112D59A6DD006C3
:10C4B0000FD59A6D510334D49A6DD20503D49A6D79
:10C4C00022F010029A65194B4FF0006218489A60EA
:10C4D0009AE770479A6D500307D49A6DD10503D43B
:10C4E0009A6D22F008029A65104B4FF080629A60B4
:10C4F000D8E79A6D4FF0807122F002029A65996038
:10C50000C9E7DA6E4FF4800122F08002DA669960A2
:10C51000BAE79A6D4FF0007122F004029A659960B3
:10C52000ABE74FF000629A60704700BF00640240C2
:10C5300058640240384B5A68110303D5D3F8A02041
:10C5400052075BD4344B5A68D00303D5D3F8B420D8
:10C55000110649D4304B5A68520303D5D3F8A020B2
:10C56000900737D42C4B5A68D10203D5D3F8A020BA
:10C5700012071CD4284B5A68920217D5D3F8A02072
:10C58000D00613D5D3F8A020510341D4D3F8A0206E
:10C59000D20505D4D3F8A02022F01002C3F8A020C1
:10C5A0001D4B4FF400121D48DA602DE77047D3F899
:10C5B000A02050030AD4D3F8A020D10505D4D3F885
:10C5C000A02022F00802C3F8A020134B4FF48012E1
:10C5D000DA60CFE7D3F8A0204FF4802122F00202E6
:10C5E000C3F8A020D960BDE7D3F8B4204FF4803160
:10C5F00022F08002C3F8B420D960ABE7D3F8A020C2
:10C600004FF4002122F00402C3F8A020D96099E77A
:10C610004FF40012DA60704700640240A0640240E8
:10C620002DE9F041564E82B096F8F43B022B00F211
:10C630009380544D6B6913F0007303D00E2002B049
:10C64000BDE8F081CDE9003340F2FF574FF48A6333
:10C650004FF008080446AF630121C5F80880102098
:10C66000EB60FFF72BFEAF630028E8D1AF63012139
:10C67000D6F8BC3B3720AB6040F27743EB60FFF766
:10C680001DFEAF630028DAD13F4A40F27343012117
:10C690006A62C5F82880EA6A42F03302EA62AF6350
:10C6A000A8603320EB60FFF709FEAF630028C6D116
:10C6B000694640F22A4201E09B0253D46B6B13425D
:10C6C0006B6BF9D01F0752D46B6B980751D46B6B0F
:10C6D000990650D46B6B9B024FD4B4F5006F009B4E
:10C6E00008BF4FF480221BBA18BF4FF480321A42A1
:10C6F00036D0D6F8BC2B40F27743224D40F2FF569D
:10C7000001213720AE63AA60EB60FFF7D7FDAE636F
:10C71000002894D1B4F5006F40F24643AE634FF069
:10C72000010108BF0220A8600620EB60FFF7C6FDEC
:10C73000AE63002883D16B6803F400639C423FF42E
:10C740007EAF124A6B68134023436B606B6803F43F
:10C750000063A342F6D172E7282002B0BDE8F08161
:10C7600026206CE7D5F8803041F8043BA6E704208A
:10C7700065E7022063E7062061E722205FE700BF4C
:10C7800078180120002C014000E1F5050081FFFF31
:10C7900070B5184D40F2FF56174C40F24D43D5F896
:10C7A000BC2B0121A6630D20A260E360FFF786FD8C
:10C7B000A66320B96369C3F34323042B02D04FF06F
:10C7C000FF3070BDD5F84C0C0028FAD00168838882
:10C7D000096995F8492C0B402AB1002B0CBF0020A9
:10C7E0004FF0FF3070BD002B14BF00204FF0FF3022
:10C7F00070BD00BF78180120002C014070B51A4DA3
:10C800001046D5F84C4C3CB12668A28834692240C9
:10C8100095F8494C14B31ABB0A4600213BF072FB51
:10C82000F0B9D5F8E83B002BFBD1104C40F2FF5695
:10C83000D5F8BC2B40F24D43A6630121A2600D2028
:10C84000E360FFF73BFDA6630028F1D16369C3F302
:10C850004323042BECD12B6D6B6570BD002ADBD11B
:10C860004FF0FF3070BD00BF78180120002C014050
:10C8700070B51A4D1046D5F84C4C3CB12668A288CC
:10C880003469224095F8494C14B31ABB0A4600217A
:10C890003BF0D2FAF0B9D5F8EC3B002BFBD1104CB1
:10C8A00040F2FF56D5F8BC2B40F24D43A663012160
:10C8B000A2600D20E360FFF701FDA6630028F1D11F
:10C8C0006369C3F34323042BECD12B6D6B6570BDFF
:10C8D000002ADBD14FF0FF3070BD00BF7818012077
:10C8E000002C0140C94BD3F8C01BD3F8C42B70B542
:10C8F0008C0FC2F3072C100E83F8F04CC1F3836445
:10C90000000183F8F14CC1F3016483F8F24CC1F3E8
:10C91000074483F8F34CC1F30724C9B283F8F44CFD
:10C92000C2F3035483F8F51CA3F8F60CC2F3C0302D
:10C93000B3F8F61C89B22143C2F30344A3F8F61CF2
:10C94000C2F3403183F8F84CC2F3803483F8F90C19
:10C95000002083F8FA4C83F8FB1CC2F3003183F803
:10C96000FC1C93F8F41B83F8FD0C012940F2F380C2
:10C97000022900F0C580D3F8C81B2A204FEA4C0CCE
:10C9800083F8094DC1F3C01201F07F010CF07E0C59
:10C9900083F80ACD4FF0010C93F80A4D1443D3F8F5
:10C9A000CC2B83F80A4DD40F83F80B1D910D83F81F
:10C9B0000C4DC2F3417401F00C01C2F3815583F8B0
:10C9C0000D4DC2F3826483F80E4D83F80F1D93F86A
:10C9D0000F1DD3F8D04B294383F80F1DC2F34051EC
:10C9E00083F8101D002183F8111DC2F3004183F864
:10C9F000121DC2F3C03183F8131DC2F3803183F8D6
:10CA0000141DC2F3403183F8151DC2F3003183F8C1
:10CA1000161DC2F3812183F8171DC2F30121C2F351
:10CA2000460283F8181DC4F3074183F8192D220E1E
:10CA3000090283F81ACD83F81C2DC4F30722A3F84A
:10CA40001E1D2406B3F81E1D89B21143A3F81E1D36
:10CA5000D3F8D41BC3F8204D0C0ED3F8202D42EA96
:10CA60000442C3F8202D0A0AD3F8204D02F47F4275
:10CA70002243C1F30724C9B2C3F8202DD3F8205DA7
:10CA8000D3F8D82B2C43C3F8204D83F8241D110E66
:10CA900083F8251D110C0906C3F8281D1102D3F8CF
:10CAA000284D0A4601F47F01214392B2D3F8DC4BB2
:10CAB000C3F8281DD3F8281D0A43C3F8282DC4F352
:10CAC0000352D3F8281D41EA1461C3F8281D93F8D6
:10CAD0002C1D1143C4F3072283F82C1D210A01F4F5
:10CAE0007061A3F82E1DB3F82E1D89B21143C4F353
:10CAF0004602A3F82E1D83F8302D83F831CD70BD8A
:10CB00001204D3F8C81B02F47C12C1F3072CC3F83B
:10CB1000002D0A0ED3F8004D44EA0224C1F3074267
:10CB2000C3F8004DD3F8004D22434FF40074C3F80E
:10CB3000002DD3F8002DC3F8404D013240F1000420
:10CB4000A40244EA92549202C3F83C4DC1F38034EB
:10CB5000C3F8382D12E74FEA8C2CD3F8C81B92008B
:10CB60004FF0010E0CF44064C1F3C26502F47F7211
:10CB7000C1F3072CC3F8004DD3F8004D2243CC0B72
:10CB8000C3F8002D04F00602D3F8004D44EA917476
:10CB9000C3F8004DC1F3026483F8045D83F8054DCA
:10CBA000C1F3425483F8064DC1F3824483F8074D24
:10CBB000C1F3C03483F8082D93F8082D224383F87D
:10CBC000082DD3F8004D93F8082D93F8F85C023245
:10CBD0000EFA05F50EFA02F2C3F8405DD617A2FB75
:10CBE000052E05FB06EE04FB0EEE0134A2FB042429
:10CBF000A644520AC1F3803442EACE52C3F8382D1B
:10CC00004FEA5E22C3F83C2DB8E600BF7818012039
:10CC10000E4838B5D0F84C3C0D4614463BB1196867
:10CC200090F8492C9B8809690B4052B15BB9FFF71A
:10CC300059FE074A4FF400730020926C2A6023804B
:10CC400038BD002BF3D14FF0FF3038BD78180120EC
:10CC5000682501202DE9F04FB74D89B0B74F00246A
:10CC60000646D5F8481D3B465A68013424339142A4
:10CC700000F00381102CF7D10024B14B9E4206D066
:10CC800048339E4203D0002009B0BDE8F08F04F184
:10CC9000FF3808EBC8034FEAC80207EB8303009292
:10CCA0001A7F002AEFD14FF0170AA3F81CA0002C1E
:10CCB000E9D0DFF8A0920120D9F8243043F40063D2
:10CCC000C9F824300EF062FBD9F82430012023F497
:10CCD0000063C9F824300EF059FBA5F89AAED9F8D4
:10CCE000443043F40063C9F84430D9F8303043F499
:10CCF0008003C9F83030D9F8303043F00C03C9F85C
:10CD0000303095F84E3D002B40F00A81D5F8942E36
:10CD10004FF00209DFF830A24FF0000B01935244AC
:10CD2000884B03EB922292F874071722A5F8BA2ECB
:10CD3000A5F8EA2E3BF032FD0323B5F8982E02A9A0
:10CD4000D5F8940E0292CDE903930C23CDE905BBEF
:10CD500007933EF0A5FF019B002B40F09080D5F893
:10CD6000B43E4FF00009784A4FF0030B4FF00C0A25
:10CD70001344744A02EB932393F874073BF00EFDBF
:10CD8000B5F8B83E02A9D5F8B40E02930223CDF847
:10CD90001CA0CDE90599CDE9033B3EF081FFD5F814
:10CDA000E41E694A674B0A4403EB922292F8740727
:10CDB0003BF0F4FC022302A9D5F8E40ECDF81CA048
:10CDC000CDE9033BB5F8E83ECDE9059902933EF085
:10CDD00067FF5E4BDB68C5F8486DC3F30223C3F100
:10CDE0000702191D042A28BF04220629584988BFB2
:10CDF000A3F103094FF0FF339340564ADB4303F09E
:10CE0000010303FA09F31B01DBB281F831334FF45C
:10CE100000334B60136B43F48003136300233360D0
:10CE20004D4BB36003F59B3303F5EC739E427ED00C
:10CE30004A4B4FF47412DA60009B434457F82300C6
:10CE4000474B336007237361464B98420CBF9520D4
:10CE500096203BF0A3FCD5F8482D394B20469A424A
:10CE60004FF000034FF001020CBF3F493F49FCF770
:10CE7000ADFD012009B0BDE8F08FE4B2FDE6D5F8C4
:10CE80009C3E304A534402EB932393F874073BF0E3
:10CE900085FC032302A9D5F89C0ECDF80C90CDF8A3
:10CEA00018B0CDE9043B0C230793B5F8A03E0293DC
:10CEB0003EF0F6FED5F8A43E224A534402EB9323FB
:10CEC00093F874073BF06AFC032302A9D5F8A40E7B
:10CED000CDF80C90CDF818B0CDE9043B0C230793A6
:10CEE000B5F8A83E02933EF0DBFED5F8AC3E154AFD
:10CEF000534402EB932393F874073BF04FFC032356
:10CF000002A9D5F8AC0E04930C23CDF80C9007932E
:10CF1000B5F8B03ECDE905BB02933EF0C1FE1EE779
:10CF2000A5F8A2AEA5F8AAAEA5F8B2AEEEE64FF00F
:10CF3000746243F8502C7FE778180120000001202C
:10CF400058640240100605080000FEBF00ED00E036
:10CF500000E100E000380240802C01400064024003
:10CF60006054A308006002406DC4000835C5000885
:10CF70000E4A01210D20D2F8BC2B38B50C4C40F2E2
:10CF8000FF5540F24D43A563A260E360FFF796F9B9
:10CF9000A56340B96069C0F34320A0F10400B0FA72
:10CFA00080F0400938BD002038BD00BF781801204E
:10CFB000002C0140A34A0220A34B516C41F40061B4
:10CFC0002DE9F043516483B0526C03259F4C02F469
:10CFD00000620192019A6268134043F07603636035
:10CFE000636823F48073636025600EF0CFF9636893
:10CFF00040F2FF50002143F480734FF4806263607D
:10D000004FF40033A063A160E26001E0002B60D028
:10D01000626B013B1706F9D5002B5AD040F2FF5541
:10D020004FF4D5724FF489630721A5630820A563E7
:10D03000A260E360FFF742F9A563002842D04FF0F9
:10D040000009824F40F2774340F2FF58002201214D
:10D050003720C7F83880BA60FB60FFF72FF9C7F8B0
:10D060003880034650BB7A4D0446064649EA05051A
:10D0700010E0C7F83880BD60FA60FFF71FF94FF67F
:10D08000FE720346C7F83880C0B97B69002B29DBE4
:10D09000944227D840F27743C7F838800121BE6018
:10D0A0003720FB60FFF70AF9034640F2694203218B
:10D0B00029200134C7F83880002BDAD0184603B095
:10D0C000BDE8F083634B01224FF0804983F8F42BD5
:10D0D000B7E703235D4A40F2FF511846916303B05E
:10D0E000BDE8F0834FF6FF72944200F0A3805E002B
:10D0F0002DD4564B1B68980731D0564C94F8F40B3E
:10D10000042831D1FFF7EEFB03460028D6D14F4D5E
:10D1100040F24743D4F8BC2B40F2FF5601210720D0
:10D12000AE63AA60EB60FFF7C9F8AE63464A6B686E
:10D130001A4003466A600028C0D194F84E3D0BB1F6
:10D140004FF4006003B0BDE8F043FFF769BA414C0B
:10D1500002203E4B84F8F40B1B689D0704D1262364
:10D16000184603B0BDE8F083384940F2FF5200236F
:10D170008A6340F2C2428B604FF40033CA6000E021
:10D1800023B14A6B013B12F0450FF9D02F4A536B84
:10D190005B0751D4536BD90747D440F2FF530128A2
:10D1A00093635369C4F8D03B9369C4F8D43BD36903
:10D1B000C4F8D83B136AC4F8DC3B01D9062831D146
:10D1C000224D40F2434340F2FF5600220621032045
:10D1D000AE63AA60EB60FFF771F8AE630346002808
:10D1E0007FF46CAFD4F8BC2B40F2C943174D40F22A
:10D1F000FF5602210920AE63AA60EB60FFF75EF8DC
:10D20000AE63034600287FF459AF6B69C4F8C03B96
:10D21000AB69C4F8C43BEB69C4F8C83B2B6AC4F8DB
:10D22000CC3B6FE70228CBD0DCE740F2FF51012373
:10D23000916343E71B2341E740F2FF5103239163CE
:10D240003CE700BF003802400081FFFF002C014096
:10D25000000010807818012030B5394D87B015F8DE
:10D26000A30C0AF0E9FCC8B10446364A00681F2145
:10D27000354B0244E18003EB922393F874073BF0B3
:10D280008DFAA18800230122206804920593CDE93C
:10D2900000136946CDE902333EF002FD2B4C94F8B1
:10D2A000FA32D4F8FC2203F001031AB11168928813
:10D2B00003BB8A6194F94F2DD3B2012B17D8244BAD
:10D2C0004FF00C0C082003F521711CFB020C994255
:10D2D0000DD013F81C2F032AF9D15A78002AF6D161
:10D2E00053F80C000028F2D0FFF7B4FC20B901205D
:10D2F00007B030BD1204DCE7D4F84C3C43B11A68E7
:10D300009B881269134094F8492C62B9002BEED027
:10D3100015F89F3C53B10F4B93F874020028E6D1E7
:10D32000236D6365E4E7002BE1D1F1E7012305F804
:10D330009F3CFFF73FFE074B83F87402EEE700BF08
:10D34000702901200000FEBF100605087818012092
:10D35000A41805080000012070B52F4C636BD90597
:10D360001DD54FF4807240F2FF562C4BA263A6638A
:10D37000E26B2B4D1340E363D5F8F03B9A0721D4C1
:10D3800001220023C5F8E02BC5F8E43B224B40F214
:10D39000FF51224A9963D96B0A40DA6370BD636B0F
:10D3A000980704D51E4B0222C3F8E42BEEE7636B0B
:10D3B000190723D4636B9A0625D5194B0622C3F8A7
:10D3C000E42BE3E7D5F8482D136823F0010313603D
:10D3D0000022E36A23F00803E362C5F8EC2BD5F8DA
:10D3E000F03BDB07CCD540F24C43A6630121A260A1
:10D3F0000C20E360FEF762FFA663C1E7084B04223E
:10D40000C3F8E42BC2E7636BDB06BFD5044B0522F0
:10D41000C3F8E42BBAE700BF002C0140C53EFFFF74
:10D4200078180120C1F10301194A41EA800092F8FD
:10D430007532C0B283422AD01023164910B58AB083
:10D4400082F8750201EB430202F8203C013302F836
:10D450001F0C202BF6D100220F4C4FF0010C029331
:10D46000A4F19C0009928DF80CC08DF820C0CDE984
:10D4700000126946CDE90422CDE906220AF09AF8A5
:10D4800054F89C2C136A002BFCD10AB010BD7047D5
:10D4900000000120200000207029012038B5344D03
:10D4A00015F8043C012B43D0022B09D0002B46D0A9
:10D4B000304C94F876325B0606D54FF4F07305E0F5
:10D4C0002C4C082384F876324FF4C373FF220221D8
:10D4D0000020A4F8783284F87522FFF7A3FF94F8AF
:10D4E0007622002124480AF097F815F8032C02212F
:10D4F00021480AF091F815F8022C03211E480AF081
:10D500008BF815F8013C33B1012B2AD0032B14BF43
:10D51000C722F72200E04722012117480AF07CF8D1
:10D52000B4F8782200211248BDE8384042F0BCBE71
:10D530004823104C84F876324FF4F073C6E7A021EC
:10D54000A5F19C000AF0F2F900F00603094C022B49
:10D5500003D000F00500012805D0082384F87632B6
:10D56000B2E78722D8E7482384F87632A5E700BFE0
:10D570007029012000000120D4280120F0B5584F67
:10D580008DB0584D3E6D28B9D5F87C3203F57A73CD
:10D59000B34270D200230122FF21534C0B938DF82C
:10D5A0000610A4F19C0002A98DF814208DF8282003
:10D5B000C5F87C62CDE90332CDE90633CDE9083305
:10D5C0000DF10603029309F0F5FF54F89C2C136A41
:10D5D000002BFCD1802145480AF0A8F995F8763255
:10D5E00083424ED114F8040C10B100200DB0F0BDF0
:10D5F000D4F8E031F31AB3F57A7FF7D90123039019
:10D600000B9002A904938DF814308DF82830FF2375
:10D610008DF807300DF10703CDE90600CDE90800CC
:10D620003248029309F0C6FF54F89C2C136A002B71
:10D63000FCD1A0212D480AF079F994F8E431172B98
:10D640000FD195F8763203F04003002BA4F8E831AF
:10D6500000F00703A4F8EA3114BF10230D23A4F847
:10D66000EE31410712D50023C4F8F0310020C4F890
:10D67000E0610DB0F0BD1C4C14F8040C0028B4D1CE
:10D68000B6E7FFF70BFF01200DB0F0BD00F005007D
:10D6900001281BD00028E9D195F876325B06E5D544
:10D6A000D4F8F031BBB13A6DD31A642BDED9FFF751
:10D6B000F5FE94F8E431172BD8D1B4F8F4310133E6
:10D6C0009BB2A4F8F431A4F8EC31CFE795F87632A8
:10D6D0005A06E5D5CAE73B6DC4F8F031C6E700BF8E
:10D6E000781801200000012070290120D428012091
:10D6F0002DE9F04F7B4C85B094F8F6313BB1B4F88E
:10D70000BA05003818BF012005B0BDE8F08F54F805
:10D710009C3C1A7B002A40F094800A221B6A0C2150
:10D720000192002B40F09A809B460B1F6E4A012607
:10D7300003935D4694F8B835DFF8C091C3EB03134B
:10D74000B4F8BA75DFF8A48102EB431AB9F878325D
:10D7500007EB53070AF0CAFCB4F8BA3502904AE066
:10D76000FF2804D14FF0200220200AF803208BF07C
:10D77000010B46EA0B0B1BF0FF0B73D0E1189EF870
:10D7800001C049788C4500F08D8094F8BCC508EB49
:10D79000050102354CF0010C81F841C04FF0040C3A
:10D7A00081F840C008EB05014FF0050C043581F805
:10D7B00040C04FEA132C81F8433081F841C04FF04C
:10D7C000060C81F842C0691C08EB050C4FF0070EEF
:10D7D0000235414400268CF840E0E05481F84000D6
:10D7E0000133B9F878029BB29842A4F8BA353CD913
:10D7F000039A95423CDABB423ADA0AF077FC029B84
:10D80000C01A019B834233DDB4F8BA351AF803001D
:10D810000AEB030E14F803C08445A1D1002EDFD11A
:10D82000BBF1000F4CD008EB0500691C4FF0070C52
:10D83000023541445E4680F840C0FF2081F8400038
:10D84000CEE714F8142C1B6A002A15BF14220A22F2
:10D85000FA210C210192002B3FF466AF012005B0A4
:10D86000BDE8F08F4FF0010BADE70023A4F8BA3507
:10D87000BBF1000F26D04EB31C4B6A1C04211A4486
:10D880002B44023583F8401094F8BC3582F84030C0
:10D89000174B18491848C9F88852C9F8803209F05E
:10D8A00089FE2CE708EB05014FF0040C02354FF020
:10D8B000000B81F840C094F8BCC581F841C071E705
:10D8C00001268DE7002D3FF41AAFE1E7074B6A1CF4
:10D8D000072059191A44023581F84000FF2182F8C7
:10D8E0004010CAE770290120682B012000000020A9
:10D8F0004000002080020120D428012000000120E7
:10D900000A4B93F8A80218B9094B93F8BD05704764
:10D91000084AD1680329F7D105494FF0010C81F875
:10D92000BDC50021D16083F8A81270470000012016
:10D9300070290120502800400021032008B5FCF781
:10D9400077FF72B6FBF762FC2B4CD4F8C02594F835
:10D95000C60508B552B11168938809690B400028C3
:10D9600044D1003B18BF0123002BF3D114200DF04C
:10D970000DFD2249002000BFD4F8C03563B11D68F9
:10D9800094F8C6259B882D692B405ABB003B18BFD5
:10D9900001230BB1FFF7D0FF0A6D4B6DD31A322B69
:10D9A00011D8D4F8C8359342E5D2D1F8FC3233B15E
:10D9B0001D689B886E69334218BF1B04AB6132320D
:10D9C000C4F8C825D7E791F8FA32D1F8FC2203F061
:10D9D000010322B11568928803B11204AA61C4F848
:10D9E000C805C8E7B3FA83F35B09D2E7B3FA83F358
:10D9F0005B09002BAED1B9E770290120781801200E
:10DA000070B53EF001FA1B200AF016F908B129237F
:10DA1000C3801C200AF010F908B12923C380254CCB
:10DA2000D4F8583813B10023C4F858380023224ED4
:10DA3000012584F8CC35C4F8546884F840583BF08C
:10DA400081FC94F87D3806F11C02022BC4F858289A
:10DA500001D0284670BD14F8A03CAB4225D0022B63
:10DA6000F7D15436C4F87068D4F8744894F8BC33CD
:10DA7000012B14D023680122032084F8BC23D3F89F
:10DA8000042822F00202C3F8042832F0A5FA226822
:10DA90000021936843F00103936084F8BC130023D2
:10DAA000064A184682F8233070BD7436C4F8706890
:10DAB000DAE700BF70290120AC02012000ED00E090
:10DAC00000234FF6FF720121438101728381C381DC
:10DAD00002828274704700BFFF224FF0000C164B89
:10DAE000C270027102724272427382738274C27493
:10DAF0006246F0B54FF0FF3E03F10C076546644601
:10DB0000764602EB8202BB4200EB020184544D7068
:10DB100081F802C0CE7081F804E00BD093F90620A2
:10DB200006335C789D7893F803C093F9046093F909
:10DB300005E0E6E7F0BD00BF741B050800230222E4
:10DB4000037043708370C370027170470023012219
:10DB5000437002708370C370704700BF4FF4F0725F
:10DB600040F22E4C0921002302804FF4FA62A0F803
:10DB70001EC04FF47A7C028440F2262281700E216E
:10DB8000828302224371A0F822C040F2012C8360FC
:10DB9000C36080F8241040F20341427440F20562F1
:10DBA00043820723A0F814C0C182028383767047A2
:10DBB0008388C3F30B039342A8BF134670B51D4679
:10DBC0000C461A460646806842F0FAFA6219084B7B
:10DBD0009442B56908D0074814F8011B00FB03F311
:10DBE000A24283EA0103F7D101202B6070BD00BF80
:10DBF000C59D1C8193010001002303704370837055
:10DC0000C37070470023037043708370C370704704
:10DC1000002306214FF47A7201700373C0E90123D7
:10DC2000704700BF00234370C3700370037183709B
:10DC3000704700BF0023FF22411C10B500F81320DD
:10DC400001F813200133082BF8D10B4B4FF0FF31B3
:10DC5000002203F10F048C4605E093F904C093F908
:10DC6000051013F8032F00EB420E9C4200F812C07F
:10DC70008EF80110F1D110BD881B0508704700BF58
:10DC80000A4491421AD001F1FF3C41F2210100B552
:10DC900002F1FF3E1CF8012F082380EA022010F455
:10DCA000004F4FEA400281EA40000CBF90B280B2C0
:10DCB000013BF4D1E645EDD15DF804FB704700BFB0
:10DCC000704700BF2DE9F047089F002B0E46054620
:10DCD0003C4614BF4FF030094FF0200914F8011BE7
:10DCE00041B3002A2CDD234600E0B2B113F8010B4A
:10DCF0009046013A0028F8D1A8F102086AB1C2465C
:10DD000049462846B04753460AF1FF3A002BF7DC54
:10DD100028EAE8723978013249B1D71B2846B04762
:10DD2000E01914F8011B0029F8D1BDE8F08710466E
:10DD3000BDE8F087002A02F1FF38E0DC0846F4E78E
:10DD40000022EAE703685A1C02601970704700BF9E
:10DD5000024B186803681B68184700BF883201200F
:10DD60000378092B01D0202B05D110F8013F202B7F
:10DD7000FBD0092BF9D02D2B63D02B2BB7EE000A4B
:10DD800008BF01300278A2F13003D9B2092961D865
:10DD9000F2EE046ADFED4D7A07EE103A10F8012F2B
:10DDA000B8EEC77AA2F13003D9B2A7EEA67A092954
:10DDB000F0EE477AF0D92E2A50D0037803F0DF0333
:10DDC000452B3BD110B442782D2A73D02B2A62D038
:10DDD000A2F130030130092B63D80024002303EBA8
:10DDE000830302EB430310F8012FA2F13001303B13
:10DDF0000929F4D9B3F59A7F1A46B7EE007A28BFFD
:10DE00004FF49A72072B09D91346DFED316A083BAC
:10DE100027EE267A072BFAD802F007022AB1F2EE93
:10DE2000046A013A27EE267AFBD1002C3BD0C7EEDC
:10DE3000877A5DF8044B20EE270A704720EE270A08
:10DE4000704742780130BFEE000AA2F13003D9B228
:10DE500009299DD92E2ADFED1D7AAED143780130F4
:10DE6000A3F13002D1B20929A8D8B2EE047AF0EEBB
:10DE7000475A06EE902A10F8013FB8EEE66AA3F181
:10DE80003002D1B2C6EE076A092927EE257A77EE6D
:10DE9000A67AEED992E782780230A2F13003092BFC
:10DEA0009BD9B7EE007A67EE877A5DF8044B20EED7
:10DEB000270A704782780230A2F13003092B01D87B
:10DEC00001248BE7B7EE007AB1E700BF0000000045
:10DED00020BCBE4CF8B5164D6B78BE2B25D1AC1CC2
:10DEE000144F022229464FF6FF70FFF7C9FE228821
:10DEF0004AB1A618BE4218D2052A16D92146344680
:10DF0000FFF7BEFEF3E721460222FFF7B9FE022229
:10DF1000A1180634FFF7B4FE074B641B9C8041F642
:10DF20000F53C31A58425841F8BD0020FCE700BF08
:10DF3000004000080080000888320120F0B5067912
:10DF400006F0E003402B03D144794FF0FF3506E0A3
:10DF5000602B4FF00104F8D1457904FA05F5002350
:10DF6000012006F00706A34200D1F0BD042E0FD811
:10DF7000DFE806F00308101D240048B1C85CD75C38
:10DF800078400FE020B1C856D756C71B7842784179
:10DF90000133E8E70028FBD031F8130032F81370A2
:10DFA000784080B228420CBF01200020F0E7002812
:10DFB000EED031F9130032F91370E6E70028E7D00C
:10DFC00051F8230052F82370DAE7037903F01803BD
:10DFD000102B1DD004D82BB1082B06D00020704781
:10DFE000182BFBD1B0F80B007047104BB0F80B00AA
:10DFF00093F90030591C09D10D4B1B7A03EB8303B5
:10E00000C3EB031300EB430080B27047DBB2F5E7CC
:10E01000064BB0F80B0093F901305A1C04D1044BA5
:10E020005B7A00EB4310EFE7DBB2FAE788030120ED
:10E03000883201200022104B30B594464FF44874CA
:10E0400003F10C0596460260828002EB4202AB426D
:10E0500000EB420100F812E081F801C0DA788C8010
:10E060008A7008D093F90620063393F801E093F8FC
:10E0700002C09C88E9E730BD9C1B050801390022DD
:10E080004B00026001F0030103F00802C1EB011133
:10E090009300C1EB0111A3EB92038900C3EB0313BF
:10E0A00081809B004380704700B589B00022034601
:10E0B0004FF4807E0DF1100C0492ADF814205A80BC
:10E0C0009A601A82C3F81620A3F806E0A3F814E0B9
:10E0D0009CE803004FF40070ADF81C1018809CE819
:10E0E0000300BDF81CC040F20120ADF81C10BDF8C3
:10E0F0001C20A3F80CC0D8815A8309B05DF804FB3A
:10E10000144B1522144910B5044618681B79206277
:10E1100004F1250084F8243042F0F6F90F4B4FF05B
:10E12000010E1A7E84F83AE012B984F83B2010BD43
:10E1300003F11C0CBCE80F0020606160A260E3608A
:10E14000BCE80F0084F83BE020616161A261E361FB
:10E1500010BD00BF447B05084C7B050888320120B8
:10E160002DE9F84338220021064642F09DF80123AC
:10E17000164CDFF86C904525B373412186F82130A9
:10E1800041F61E63124A09F10808F384671E114B19
:10E19000B362114B336103F1C87303F2B633736199
:10E1A0000E4BC6E90623484642F085F9631E294610
:10E1B00028B1DA1B4045A0EB090338BFF25415B172
:10E1C00014F8015FEFE7BDE8F88300BF5D7B050849
:10E1D000001975031E7D01016400DC0543080E0073
:10E1E00038BB0508202108B542F065F9034618B18F
:10E1F0001A780130202AF9D0184608BDB5EEC00AB9
:10E20000DFED357A0023F1EE10FA70B5C8BF30EEBD
:10E21000270A86B0D8BF30EE670ADFED307A0546B0
:10E2200003A902936E4620EE270ACDE90033FDEEE6
:10E23000C07A17EE904A84EAE470A0EBE47039F0FB
:10E2400051F8002C03A8ACBF20232D238DF80030FB
:10E250003FF0A0FE012829D0022833D003281DD08A
:10E2600003A9304642F018F930463FF093FE0446C9
:10E2700031462846033CE4B2224641F0A1FF002388
:10E2800028462B553FF086FE2E22431C31192A5476
:10E29000E81842F01DF9284606B070BD302303A9E6
:10E2A00030468DF8013042F0F7F8DDE7302303A95E
:10E2B00030468DF801308DF802308DF8033042F091
:10E2C000EBF8D1E7302303A930468DF801308DF803
:10E2D000023042F0E1F8C7E76F12033A00007A44D7
:10E2E00008F084BF13B568B14C1E14F8011F21B9A2
:10E2F00002B0BDE8104008F08DBF019008F076FF35
:10E300000198F2E702B010BDF8B5E8B10138114A42
:10E31000CB43C60002EBC00003F0010390F840506D
:10E3200090F8417083EA0504A7420DD0C06B40B15C
:10E330000768AB420CBF10230023808800FA03F368
:10E34000BB61324482F84140CB0701D4FDF712FA99
:10E35000F8BD00BF883201202DE9F3410023124DA2
:10E36000044600EB8106114F05F85C3FB44203D12F
:10E370000F4802B0BDE8F081394628464FF000084A
:10E3800042F08AF82146684642F0A2F82021684609
:10E3900042F091F828B969462846043442F07CF8E6
:10E3A000E4E780F80080F1E78832012062BC0508CC
:10E3B000E4320120024BD3F880002AF0F5BE00BF02
:10E3C000883201202DE9FF471E46C368044689466E
:10E3D0009246BDF83070DDF834804BB3CBB20D2BD4
:10E3E00024D81A4AD556BAF1FF3F23D023683146C4
:10E3F000174A3846CDE9005AC04752465FFA89F1BC
:10E40000207909F0ABF8024600B10288D3B2314658
:10E4100038460393C2F30323120B02932368CDE91A
:10E4200000520C4AC04704B0BDE8F0870025DAE787
:10E430004D1CD8E77B06F6D423683146064A384699
:10E44000C4460C9504B0BDE8F0476047287B05083A
:10E450004DBB05085ABB05087EBB05082DE9F041F8
:10E46000154686B0884619466A1CBDF830600D9F77
:10E4700023D0030900F00F04174A30464033CDE99A
:10E4800000450593B847A8B12A4698F80510D8F872
:10E49000000009F0E5FA68B1028801783046059B72
:10E4A0000391C2F30321120B02910021CDE9004236
:10E4B0000A4AB84706B0BDE8F0817306FAD40309EA
:10E4C00000F00F00064ABC460C904033304606B0C0
:10E4D000BDE8F041604700BF8DBB05089FBB050844
:10E4E000C8BB05082DE9F0411E4688B003099046D7
:10E4F0000E9F00F00F04403349B307930DF0ACF8C2
:10E50000027A0546079B41463046CDE90042144A4F
:10E51000B847C8B12868FCF731FCE9796A7911F08D
:10E52000020FDFF84CC04FEA92020E492D7A08BF65
:10E5300061460132079B0094CDE90102CDE9031544
:10E54000094A00213046B84708B0BDE8F081074AC3
:10E5500041463046BC460E9408B0BDE8F0416047E5
:10E56000DCBB0508C2BD0508EEBB050810BC0508EC
:10E5700051D30508084B024608498B420AD2184677
:10E5800002E01C30884205D20388C3F30B039A4291
:10E59000F7D1704700207047E8010008E40900083F
:10E5A000F8B50A4E0546B0F80900FFF7E3FF96F804
:10E5B000847004462846FFF708FD2FB196F8853091
:10E5C00013B9E3681844F8BDA368FBE7883201205B
:10E5D00038B505460C46FFF7E3FF2B7903F0E00260
:10E5E00003F00703602A29D1022BDAB20ED0042AE5
:10E5F00018D03AB96A79012393400278DBB214B19A
:10E600001343037038BD22EA0303FAE76A79012352
:10E61000934002889BB214B113430380F2E722EACD
:10E620000303FAE701236A7903FA02F2036814B1DB
:10E6300013430360E6E723EA0203FAE7042BE1D879
:10E64000DFE803F00303050507000470DAE7048040
:10E65000D8E70460D6E700BF70B585880B4604464E
:10E660000021C5F30B0518462A4641F01DFE6169DD
:10E67000084A0346914202D3074A914205D319B191
:10E680001846BDE87040084770BD2A46BDE8704096
:10E6900041F096BDCC380608943A060838B5064CC9
:10E6A000064DAC4206D2A16820461C34FFF7D4FFC9
:10E6B000AC42F8D338BD00BFE8010008E409000807
:10E6C0000823484010F0800F4FEA400182EA4000E2
:10E6D0000CBFC8B2C0B2013BF4D1704730B5056879
:10E6E0008D421AD901F1FF3E6C1E00231EF801CFA6
:10E6F000082183EA0C0313F0800F4FEA430C82EAEF
:10E7000043030CBF5FFA8CF3DBB20139F3D17445DC
:10E71000ECD16A1C02602B7030BD00236A1C0260C1
:10E720002B7030BDB0EEC07AF0EEE06A86FE876AEC
:10E73000B5EE406AF1EE10FA3DD0C6FEC75AC5EEFE
:10E74000867ADFED1E2ADFED1E3ADFED1E4A9FEDD1
:10E750001E5A9FED1E3AB7EE006A9FED1D4ADFED8F
:10E760001D5AE7EEE23AA7EE834AE7EEA34AA7EE88
:10E77000846AA7EEA45AE7EE855AC5EE867AF4EECF
:10E78000C76AF1EE10FA03D59FED137A77EE677A38
:10E79000F5EEC00AF1EE10FA03D59FED107A77EE90
:10E7A000677AB5EEC00AF1EE10FA48BFF1EE677A6B
:10E7B000B0EE670A7047DFED077AE0E739094E3DB2
:10E7C000E3B59E3E88FA163E45FE7F3F99FB243F07
:10E7D00069A2163EA7DFA834DB0FC93FDB0F494013
:10E7E00091ED056AD0ED017AD1ED036A91ED047ADD
:10E7F00067EEA66AD0ED005A27EE877AD1ED014A7E
:10E8000067EE867A91ED025A91ED004AA4EEA57A60
:10E8100090ED026AE5EE257AD1ED064AE4EE256A2E
:10E8200091ED075AD1ED085AA5EE067AE5EE867A03
:10E83000E4EE866A80ED017AC0ED027AC0ED006AEE
:10E84000704700BFDFED277AB4EEE70AF1EE10FA69
:10E850000CDDDFED256A9FED257AF0EE407A30EE93
:10E86000660AF4EEC77AF1EE10FAF6DCDFED207AF4
:10E87000B4EEE70AF1EE10FA0CD5DFED1B6A9FED5E
:10E880001D7AF0EE407A30EE260AF4EEC77AF1EE09
:10E8900010FAF6D4DFED187AB4EEE70AF1EE10FACA
:10E8A00014DDDFED107A37EEC00A60EE006A9FEDEE
:10E8B000136A9FED137ADFED137AA6EE867A20EEC7
:10E8C000266AE6EE877AA6EE270A7047DFED0E7A13
:10E8D000B4EEE70AF1EE10FAE7D5DFED057A37EE90
:10E8E000C00AE2E7DB0F4940DB0FC940E4CB164129
:10E8F000DB0F49C0E4CB16C1DB0FC93F92E741B93A
:10E900009730083C15A82ABEDB0FC9BFFDEEC07AC0
:10E9100017EE903A2033402B00D893E79FED010A81
:10E92000704700BF00000000D0ED005A9FED2B4A59
:10E9300008B535EE840AFFF7E9FFB0EE405AB0EEB5
:10E94000650AFFF7E3FFD0ED014AF0EE405A34EEDE
:10E95000840AFFF7DBFFF0EE403AB0EE640AFFF7FF
:10E96000D5FF90ED023AF0EE404A33EE040AFFF78D
:10E97000CDFFB0EE404AB0EE430AFFF7C7FF25EEE9
:10E98000236A65EE046AC1ED024A25EE847A25EE1B
:10E99000005A81ED086A23EE844A23EEE53AB0EE90
:10E9A000666A65EE805A81ED004AB0EE454A81ED17
:10E9B000053A60EE637AA4EEE56AA4EE874AE4EED7
:10E9C000E65AC1ED017AA4EE857A81ED046A81ED03
:10E9D000034AC1ED065A81ED077A08BDDB0FC93F36
:10E9E000B7EE001A0022DFED050A10B541F0D4FDA4
:10E9F0000023836143610362C36110BDF304353FAB
:10EA00002DE9F04F1F461346894689B013F8011BC4
:10EA1000002900F02B8215468046002609E040467A
:10EA200001361D46C8472B4613F8011B002900F08C
:10EA30008C802529F3D16978302900F0DD800235FA
:10EA40000023A1F1300C5FFA8CF2092A4FF000028A
:10EA50005ED96C297DD07829E5D8572967D9A1F1ED
:10EA600058002028DFD801A454F820F0EDEC00086D
:10EA700027EA000827EA000827EA000827EA000832
:10EA800027EA000827EA000827EA000827EA000822
:10EA900027EA000827EA00082BEC000839EC0008F8
:10EAA00027EA000827EA000827EA000827EA000802
:10EAB00027EA000827EA000827EA000827EA0008F2
:10EAC00027EA000823EC000827EA000827EA0008E4
:10EAD00027EA000827EA00080FEC000827EA0008E8
:10EAE00093EC000827EA000827EA0008EDEC00088C
:10EAF000BEF1050F18D9BAF1050FAAD80A2CA8D172
:10EB000002EB820215F8011B04EB4202A1F1300C6A
:10EB10005FFA8CF0A1F1610EA1F1410AA1F1370475
:10EB20000928E5D86446EBE7A1F15704E6E761B1AF
:10EB300025297FF478AF25214046C8472B4601366A
:10EB400013F8011B00297FF474AF304609B0BDE80B
:10EB5000F08F15F801CBBCF1780F3FF664AFBCF134
:10EB6000570F4DD9ACF1580120293FF65CAF01A0F9
:10EB700050F821F04FED000827EA000827EA0008C6
:10EB800027EA000827EA000827EA000827EA000821
:10EB900027EA000827EA000827EA000827EA000811
:10EBA0002BEC000801EE000827EA000827EA00081D
:10EBB00027EA000827EA000827EA000827EA0008F1
:10EBC00027EA000827EA000827EA000823EC0008E3
:10EBD00027EA000827EA000827EA000827EA0008D1
:10EBE0000FEC000827EA0008AFED000827EA00084C
:10EBF00027EA00084FED0008A9780123033520E734
:10EC0000BCF1000FA1D0BCF1250F94D00BE757F851
:10EC1000040B0023494600904046FFF753F8064492
:10EC200001E757F8043B1E60FDE657F8041B404619
:10EC30000136C9B2C847F6E6D7F800C0BCF1000FEC
:10EC4000C0F2AC8005ACA246BCF1090FE6464FF01D
:10EC5000010108DD01EB81014900BCFBF1F009284D
:10EC6000F8D800293DD08948BEFBF1FBBBF10A0F63
:10EC7000A0FB01C001FB1BEE34BF4FF0300C4FF086
:10EC8000570CC0080929DC4401460AF801CBEAD830
:10EC900027E038680121092809D901EB81014900E1
:10ECA000B0FBF1F4092CF8D8002900F0E68005AC9F
:10ECB0000393A246754BB0FBF1FBBBF10A0FA3FB1C
:10ECC000013C01FB1B00B4BF4FF0300E4FF0570E5C
:10ECD0004FEADC0C0929DE4461460AF801EBE9D869
:10ECE000039B043700218AF8001029E057F804AB91
:10ECF0000120BAF10F0F40F2C6800001BAFBF0FC10
:10ED0000BCF10F0FF9D8002800F0BA8005ACA3467B
:10ED100001E0BAFBF0FCBCF1090F4FF0300E05DD4D
:10ED200058290CBF4FF0370E4FF0570EE64400FB4A
:10ED30001CAA00090BF801EBEBD100218BF80010A5
:10ED4000494640460094FEF7BDFF06446BE657F87F
:10ED500004BB0121BBF10F0F40F28D800901BBFB09
:10ED6000F1F00F28FAD8002900F0828005ACA24605
:10ED700001E0BBFBF1F009284FF0300E06DDBCF1DD
:10ED8000580F0CBF4FF0370E4FF0570E864401FB63
:10ED900010BB09090AF801EBEBD1A3E72D21CCF157
:10EDA000000C0DF1150A05AC8DF814104CE757F85E
:10EDB000040B0121092808D901EB81014900B0FBAE
:10EDC000F1F4092CF8D8002952D005AC0393A246DF
:10EDD0002E4BB0FBF1FBBBF10A0FA3FB013C01FB87
:10EDE0001B00B4BF4FF0300E4FF0570E4FEADC0C53
:10EDF0000929DE4461460AF801EBE9D8039B71E773
:10EE000057F8040B002829DB05ACA24609284FF06F
:10EE100001010AD901EB81014900B0FBF1FCBCF111
:10EE2000090FF7D800293FF45DAF0393174BB0FBF0
:10EE3000F1FBBBF10A0FA3FB013C01FB1B0034BF3C
:10EE40004FF0300E4FF0570E4FEADC0C0929DE442C
:10EE500061460AF801EBE9D8039B43E72D214042C4
:10EE60000DF1150A05AC8DF81410CFE70E466CE6CF
:10EE700005ACA24636E7584678E705ACA24630E72F
:10EE800005ACA34659E7D44640E700BFCDCCCCCC77
:10EE900073B5144C06460D460192D4F88800C0B1F3
:10EEA0001149FFF71FFA3146D4F88800FFF71AFA24
:10EEB0000E49D4F88800FFF715FA0D49019B2A4640
:10EEC000D4F88800FFF79CFD0A49D4F88800FFF7C2
:10EED00009FA94F88C3013B1012384F88D3002B014
:10EEE00070BD00BF8832012022BC050827C3050879
:10EEF000E1E200083CC505080EB400B584B008493D
:10EF000005AB019001A853F8042B0393FFF778FD9C
:10EF1000019B00221A7004B05DF804EB03B0704747
:10EF200045DD000800232DE9F0411C4682B007466C
:10EF3000038021460134384629F0D0FB082CF8D153
:10EF4000002307F1FC06DFF8608087F8EA301D46F1
:10EF5000C7F8EC30C7F8F030C7F8F430C7F8F8302D
:10EF60001F462A46414601A83446FFF7C5FF032243
:10EF700001A911F8013B5BB1013A04F8013BF8D15A
:10EF8000013504362770082DEBD102B0BDE8F081C1
:10EF9000013520462021144441F086F9082D06F160
:10EFA00004062770DDD1F0E7687B0508F7B5114E40
:10EFB000074600230C46304615460F498E3600F8AA
:10EFC0008E3F04EB45050D4B002F08BF19460C4F33
:10EFD00041F062FAAC4202D10A4803B0F0BD3946B2
:10EFE00034F8022B6846FFF787FF6946304641F048
:10EFF00053FAEFE7883201202FBC050838BC05081A
:10F0000041BC050816330120F7B500230B4E04461A
:10F0100000EB41050A4F06F8BF3FAC4202D1094858
:10F0200003B0F0BD394634F8022B6846FFF764FFA1
:10F030006946304641F030FAEFE700BF88320120E0
:10F040006CBD050847330120F8B54E1E054601F199
:10F050001F04054F16F8012F284639460235FFF7E1
:10F060004BFFA642F6D1F8BD46BC0508024608464D
:10F07000531C05D1034B1A681B790A600B7170474A
:10F08000014939E788BB05086DBD050810B5013198
:10F0900014460CF0E1FA28B9054B1A681B79226076
:10F0A000237110BD027A20460249BDE8104023E7D3
:10F0B00088BB0508E9BB050803685A1C0260197083
:10F0C000090A03685A1C02601970704702681146E9
:10F0D000531C0360D31C11F802CB0160517803600C
:10F0E00093781B0443EA0123111D43EA0C030160DA
:10F0F000D07843EA00607047A0F13003092B07D9AC
:10F1000020F02000413819288CBF002001207047D2
:10F1100001207047303809288CBF0020012070473B
:10F12000413819288CBF0020012070476138192808
:10F130008CBF00200120704720280BD0092809D05F
:10F140000A2807D00D2805D00B3801288CBF0020D5
:10F150000120704701207047A0F14103192B98BF8F
:10F1600020307047A0F16103192B98BF20387047F9
:10F1700010B56FF000440246044404E0B3EB0E0007
:10F1800015D1A24214D012F8013BA3F14100192875
:10F1900011F8010BA0F1410C98BF203300F1200EB3
:10F1A000BCF1190FEAD91B1A04D10028E9D110BD0E
:10F1B000002010BD184610BD02B3844610B5841857
:10F1C00004E0B3EB0E0014D1A44513D01CF8013BAE
:10F1D00011F8010BA3F1410200F1200E192AA0F150
:10F1E000410298BF2033192AEBD91B1A04D10028F9
:10F1F000EAD110BD002010BD184610BD1046704762
:10F2000070B5044608460D463EF0C4FE064602E0D0
:10F2100014F8013F43B1204632462946FFF7CCFFA0
:10F220000028F5D1204670BD1C46204670BD38B57B
:10F2300007490546FFF7E4FF041E0649284618BFA4
:10F240000124FFF7DDFF08B144F00204204638BD79
:10F250004BBC0508FBD005082DE9F0410646864663
:10F260009EF800C070460EF1010EBCF1200FF7D0E1
:10F27000BCF1090FF4D0BCF10A0FACF10B05EFD0D3
:10F28000ACF10D04B4FA84F46409002CE8D1012D2A
:10F29000E6D9BCF12B0F3DD0BCF12D0F39D0102A8F
:10F2A00086463DD04FF0FF359046B5FBF2F502FBA8
:10F2B00005F7FF43FFB20EF1010E002010E0ACF1A4
:10F2C000300C5FFA8CFC944512DA8542764602D304
:10F2D00034D1674532D21C404FF0FF301EF801CBCD
:10F2E000BCF1390FEBD94CF0200CBCF1600F0BD8FE
:10F2F00001B10E602CB3B0F1004F2BD9DB0729D53B
:10F300004FF00040BDE8F081ACF1570C5FFA8CFC87
:10F31000D9E70124102A00F1010E90F801C0C1D1F3
:10F32000BCF1300F19D04FF0FF354FF01008B5FB8E
:10F33000F2F502FB05F7FF43FFB2BCE708FB00C094
:10F34000CCE70028DEDA13F0010F18BF6FF00040A1
:10F35000BDE8F0814042BDE8F0819EF801C00EF1A9
:10F360000106ACF141056046192D01D80CF12000D1
:10F3700078280BD04FF0FF354FF01008B646B5FB9C
:10F38000F2F502FB05F7FF43FFB294E710229EF867
:10F3900002C06FF070450EF1020E0F2790468AE70B
:10F3A00001230A22002157E770B50D461446FEF7E7
:10F3B00019FF0646A0B1FFF7F3FF40F63403984269
:10F3C000A8BF1846B0F5617FB8BF4FF46170A0F5D3
:10F3D00061731920B3FBF0F32B7023780133237092
:10F3E0003046FEF7FFFE0646A0B1FFF7D9FF40F614
:10F3F00034039842A8BF1846B0F5617FB8BF4FF4F8
:10F400006170A0F561731920B3FBF0F36B70237882
:10F4100001332370304670BD028840F2B55CA2F51E
:10F42000FA6210B54FEA920E817802F00302C378B7
:10F430000139124C02EB4202013B01EB82020CFB50
:10F440000E33017904EB42028479928F134442799E
:10F45000008903EB430301EBC3030021C3EB031358
:10F4600002EB8303064AC3EB0313224402EB83023D
:10F470004FF47A73C2FB030110BD00BF741B050873
:10F4800080436D382DE9F04117461E4605464FF47E
:10F490007A72002338463146454C3FF0D9F9454948
:10F4A000454A0144454882FB01C34FEAE17C0B44D5
:10F4B000CCEB631382FB03C24FEAE37C1A44CCEB30
:10F4C000621284FB02C44FEAE27CCCEBA40C80FB0A
:10F4D0000C404FEAEC74C4EBE010C3EB0314A1EB57
:10F4E0008401A971C2EB0211A3EB81036B710CEBD8
:10F4F0004C03A2EBC30240F2B55303FB10CC8000D7
:10F500002A71BCF5896F44DA40F2DA239C4547DC66
:10F51000BCF5B77F2A4BB4BF0022012202EB4201A7
:10F520004FEA420803EBC10391B2B3F8523008EB43
:10F53000020E244C04EBCE044FF00B0E163401E007
:10F5400034F8023D63451FDDBEF1010EF8D11C4BBE
:10F5500042444FF0010E03EBC202938F00F5FA60B4
:10F560000CF1010C4FF47A7285F802E00844ACEB20
:10F57000030C314600232880384685F803C03FF04D
:10F5800067F92A81BDE8F0810EF1010E5FFA8EFE67
:10F59000E4E7032140F296534FF006080A46C6E717
:10F5A000022140F229434FF004080A46BFE700BF9A
:10F5B000ABAAAA2A80BC92C78988888873B06D16C6
:10F5C000741B0508B01B050808B50D4BD3E93A2399
:10F5D00052EA030C0AD10146002340F201121846F8
:10F5E0000B804A808B808B710B8108BD05490968AF
:10F5F0008A1843F10003FFF745FF012008BD00BF53
:10F6000088320120C818012090420B462DE9F041B4
:10F61000B0FBF2F60446154608D2124A05FB164422
:10F620001846135D00F8013BBDE8F0819642B6FB39
:10F63000F2F706D20B4A05FB1767D15D03F8011BF1
:10F64000ECE7BA42B7FBF2F807D905FB1878054A90
:10F6500012F8081003F8011BEDE74046FFF7D4FF4E
:10F660000346F2E7707B0508674B9A88B2F57A7F0C
:10F6700010B582B002D94FF47A729A80DA88B2F566
:10F680007A7F02D94FF47A72DA801889B0F57A7FDE
:10F6900003D94FF47A7210461A81B3F80AC0BCF548
:10F6A0007A7F02D9002294465A819989B1F57A7FEE
:10F6B00003D94FF47A7211469A81DA89B2F57A7FCA
:10F6C00001D90022DA81844501D3002018818A42C1
:10F6D00001D300229A81598B9A8B914201D9002241
:10F6E0005A834A4B1A88002A5FD0494CA378062BCC
:10F6F00074D8484901EB830191ED270A217900294B
:10F7000050D1454B07EE902AA27993F8C803F8EE42
:10F71000E77A07EE100AF8EEC76A86EEA77A0AB112
:10F7200030EE000AB4EEC70AF1EE10FA3EDD67EEE5
:10F73000807ABCEEE77A8DED017A9DF8041007EE31
:10F74000101AB8EEC77AF4EEC77AF1EE10FA01DDBE
:10F750000131C9B2002954D01029A8BF1021C9B263
:10F7600081420A462D4938BF024683F8C8234A79A8
:10F77000012A1FD100224A715A7A032A2AD828491D
:10F7800001EB42111A7AC3F8D013032A1BD802EBFB
:10F7900082022449C2EB021201EB4202C3F8D423D5
:10F7A00002B010BD042B1CD8F3B91B4B1B494A797E
:10F7B000012ADFD0022ADFD11B4A1279002ADBD1CD
:10F7C00000224A71D8E70021164A1972C3F8D423DF
:10F7D00002B010BD002212495A72D3E79FED130AFE
:10F7E0008CE7053B032BE0D9F7EE007A87EE800A21
:10F7F00040F06EF82288084B904228BF10462080C7
:10F80000D4E70121ABE700BF78190120881E002052
:10F81000C41B0120741B050888320120E831012037
:10F8200078330120F8330120CC2801206F120338EF
:10F830002DE9F04F9D4E85B096F8D83300AFA3F177
:10F840001702022A00F29582994BBB60DFF86882AA
:10F850004FF0000A96F8E81308F16C094446DFF807
:10F8600078B2944D2FE00AF1010A5FFA8AFA430850
:10F87000820803F0773302F033321344C208C31A0C
:10F8800002F011329B1A03EB131303F00F33ABFB9F
:10F8900003E2D209C2EB02229A1A830301D5012A9C
:10F8A00019D0012A0BD9082A15D8BCF1000F01D0B4
:10F8B000284204D1F9603DF0E7FCF96858B10C34F6
:10F8C0004C4500F04F82206810F0010CCBD194F928
:10F8D0000430142BCBD178480CF0A0FF0024022078
:10F8E00086F888440FF056FB96F88C34022B00F013
:10F8F000DB82002800F02F83704B4FF47A7E96F85D
:10F9000015A54FF0000C03F5167B5A88B2F57A7FE7
:10F91000B3F8462088BFA3F802E0B2F57A7F9A8850
:10F9200088BFA3F846E0B2F57A7FDA8888BFA3F8EB
:10F9300004E0B2F57A7F02D90022A3F806C09988C4
:10F940009142B3F85A10B3F85C2098BFA3F804C0F2
:10F95000914293F86B2002F1FF3288BFA3F85AC09E
:10F96000632A03D94FF0640283F86B2093F86C206C
:10F9700003F1660019460132D2B2092A4FF00002A3
:10F9800088BF83F86CC08D7A013210F8014B0631C4
:10F99000A54238BF00F801CC032AF4D1BAF1010F17
:10F9A00003F1960318BF03F812CC5B45ADD1444B6D
:10F9B0009B78042B00F0AC822BB9414A1388B3F535
:10F9C000F07F00F2E881FFF74FFE96F82F15092926
:10F9D00003D011B13B48FEF751FB96F83D150929BC
:10F9E00003D011B13848FEF749FBB6F84A25B6F8FE
:10F9F00048351343B6F84C2513431BB213B101230A
:10FA0000A6F84E35D6F80435304A1A40002A00F0E0
:10FA1000B182DA0700F12E825D0440F1C0812C49E9
:10FA2000D6F808250B400A40C6F80435C6F8082564
:10FA300013F4004200F00182002286F8EF2386F8DA
:10FA4000FF23D90440F1038296F85B35022B02D1E3
:10FA5000012386F85B35DFF87CB05B460BF1780458
:10FA600002E006339C420CD01A78072AF9D1997823
:10FA7000DA78914202D35A79002AF2D0072019F09D
:10FA8000AFFF00234FF4806086F888340FF082FACD
:10FA9000002800F053820F4DAA469AF8051041B392
:10FAA0009AF8000018B35B461BE000BF88320120C3
:10FAB000741B0508BC020200A0360120F8330120A7
:10FAC000C41B0120B8370120C6370120096000029D
:10FAD000F6DFFFFDE83701208180808006339C42FD
:10FAE00007D01A788A42F9D15A79002AF6D019F04B
:10FAF00077FF0AF1060A5445CFD1BB4B93F802B009
:10FB0000BBF1080F00F0C481B849D6F80435D6F827
:10FB100008250B401140C2F3C032C6F8043596F8F0
:10FB20001535C6F80815A3F1010386F8DA25B3FAEE
:10FB300083F35B0986F8D83596F81635A3F10103EF
:10FB4000B3FA83F35B0986F8DC35B6F8F035002BA1
:10FB500040F0C881D6F8F43513F07F4F02D000236F
:10FB6000C6F8F435D6F8FC35A14A1A4012B1002384
:10FB7000C6F8FC3596F8F835013B042B02D9012371
:10FB800086F8F835ABF1050B9A4BBBF1030F93F8F0
:10FB900090B540F24881BBF1000F20D00023FB60FC
:10FBA000914B6FF007017C60C91A03F1080A0C46FB
:10FBB00004E004EB0A035B4580F0F5801AF8010BC2
:10FBC0000028F6D00BF06EFD0028F2D0C3799B0719
:10FBD000EFD5FB6801227C68002B40F0EA80824B65
:10FBE0009B7913B10023804A9371B6F8063613F05F
:10FBF0000C0F03D1C3F30313022B03D94FF420637B
:10FC0000A6F80636B6F8083613F00C0F03D1C3F386
:10FC10000313022B03D940F60123A6F8083696F801
:10FC2000752696F881369A4200F2F28096F874367C
:10FC300096F880269A4204D2002386F87436A6F8F5
:10FC4000783696F8762696F86A379A4202D90023D3
:10FC500086F876366848FC6000F1800BBC6810F8C6
:10FC6000043C03EB4303234493F890A193F891E100
:10FC700093F892C1C31E1A785245A8BF524603F8A2
:10FC8000012B59799A787145A8BF71466245A8BF82
:10FC90006246834259719A70EDD103F12000834589
:10FCA000DDD1D6F81014FC68002900F025814FF052
:10FCB000000C012002E00635AC4211D02B78282B35
:10FCC000F9D16B781A1D00FA03F30B4200FA02F225
:10FCD000F1D0063521EA02014FF0010CAC42EDD122
:10FCE000BCF1000F01D0C6F81014444C04F1080513
:10FCF000234613F8012B072A68D89D42F9D1EA461A
:10FD000088B02022FF21EB46584640F0CDFA3B4A0E
:10FD100012F8013B5BF8231001315ED195424BF89C
:10FD20002330F5D1B6F80E25D546B6F80C359A42F3
:10FD300002D3334BC6F80C35FF23324986F89C3783
:10FD400098F90430142B05D0D8F8002031EA0202CB
:10FD500000F0D88008F10C08C845F1D11437BD4631
:10FD6000BDE8F08F0AF1FF3ABAF1020F7FF6B6ADA7
:10FD7000B1E5254A02EBC303BA6093F8B820002A24
:10FD80003FF464ADD3F8BC30002B7FF45FAD172394
:10FD900086F8D8335AE54FF4F073138013E61C0746
:10FDA00071D51A493CE6FB6800227C68002B3FF4C1
:10FDB00016AF0D494B7C002B7FF417AF4B79012B0D
:10FDC0003FF40DAF002A7FF40AAF0EE7EA4688B091
:10FDD0002022FF21684640F067FA002304F8013B27
:10FDE0000133082BFAD19DE7C41B0120DEDDCDFDD8
:10FDF000FDFDFFFF881E00207E330120D71B012060
:10FE0000AE014A0101000200741B0508FE9FFFFDC0
:10FE1000002296F8743686F87526002B3FF411AF51
:10FE2000A6F8782604E70023584A1371BBF1000FA7
:10FE300000F09E800123FB60B2E696F8EF130029E4
:10FE40003FF4FFADD90486F8FF233FF5FDAD1A0658
:10FE50007FF5FAAD96F8D833182B06D801229A40D0
:10FE60004B4B1340002B7FF4EFADDFF834B10BF1B7
:10FE7000780406E64749D6F808250B400A40C6F83C
:10FE80000435C6F8082598047FF5D2AD4249C7E588
:10FE90001A469B79002B3FF437AE537C012B7FF43D
:10FEA00033AE022353742FE600283FF425AD3B4BBD
:10FEB0004FF0FF0C90F9045096F8951403F16C0084
:10FEC00093F90820AA4204D10139012483F808C01B
:10FED000C9B20C338342F3D1002C3FF40DAD86F848
:10FEE000951409E596F8EC050BF0DCFB00287FF48F
:10FEF00031AEA6F8F0052DE6282019F071FDD6F8F0
:10FF00001014D4E6143786F89C37BD46BDE8F08F50
:10FF1000D6F804351D4A23F48053C6F80435D6F8C4
:10FF2000083523F48053C6F80835538CB3F57A7F2F
:10FF3000BFF449AD4FF47A73538444E5D6F80435E1
:10FF400023F00063C6F80435D6F8083523F00063C3
:10FF5000C6F808359FE5D6F80425D6F8083522F00E
:10FF6000800223F08003C6F80425C6F80835C3E4F0
:10FF70005A461EE7D6F8082543F0080342F0080267
:10FF8000C6F80435C6F8082543E500BFC41B0120A8
:10FF900000410001F79FFFFDF6BFFFFD2037012064
:10FFA000E83701202DE9F04F964E83B0964B4FF085
:10FFB000010AD6F8AC27DFF8888202F2DC5243450A
:10FFC000C6F8AC274DD29B46904B914D9F1C8F4B52
:10FFD0005988002900F0F6807A18AA4234BF002020
:10FFE0000120052998BF40F00100002840F0EA8078
:10FFF000BBF800C03C46CCF30B0C0CE01188144657
:020000040801F1
:100000005018002900F0DE800529024640F2DA800F
:10001000A84280F0D78061886145EFD161798B0774
:10002000ECD123885846DBF8081094F8049001932B
:10003000FEF712FBBBF80010B9EB113F00F0CA80CD
:100040004FF0000ABBF804100BF11C0B5BF8140C0A
:10005000C1F30B0137F022FD5BF8042CC34510609F
:10006000B5D3D6F804356B4DC6F80835FFF7E0FB7D
:10007000337AA5F18002717A03EB8303664C02EBBD
:100080004112C3EB0313C6F8D02305EB4303C6F8B4
:10009000D43317F0F1FF4FF0FF33D6F8D403636089
:1000A0001FF0B4FB19F0EEFC05F57C7305F58D61CE
:1000B00003E00633994200F097801A78002AF8D1BD
:1000C0009D78D878854202D358790028F1D096F8E7
:1000D00058352272642203EB830303EB83039B00F6
:1000E000C72BD8BFC823C6F8A437B6F85C3502FBC7
:1000F00003F3C72B7DDD1A46C6F8A8370023474C0B
:100100004749C6F8AC37C1F80447C6F8B037C6F857
:10011000B437C6F8B837C6F8BC37C6F8C027A6F853
:10012000C43786F8C63720F095FA96F8D8379FED91
:100130003D6A07EE103AB6F8D6379FED3B0AB8EEA7
:10014000C77A07EE903ADFED396AF8EEE77AB6F84B
:10015000D417A7EE060AB6F8C83767EEA67AC4ED3C
:10016000A17AFDEEC07A17EE902A07EE901A96F863
:10017000CA17F8EEE77A2032402A67EEA67AC4ED75
:10018000A27A3BD8FEF75EFB07EE903ADFED286AD5
:10019000284BF8EEE77AC6F8E417A3EC010A86EEDE
:1001A000A77A83ED007A29F093F814F063FF224BCD
:1001B000012250461B6886F8C527C6F8AC3703B045
:1001C000BDE8F08FDBF8081058464FF0000AFEF744
:1001D00043FA37E7019BA11D58469A1FFDF7E8FC3B
:1001E00000287FF42FAF2BE7F27D003A18BF0122E1
:1001F0006DE7C8231A46C6F8A8377FE79FED0F0AB8
:10020000C2E700BF88320120E80100080040000872
:1002100000800008F833012088030120D037012036
:10022000881E002035FA8E3CDB0FC93F17B7D13846
:10023000C0C9FB48643A0120C81801200000000032
:10024000E409000838B501221C4B032805461C4C64
:1002500083F80C2720D96A1C00231A490220D2B245
:100260004FF0140E5200402A28BF4022C8540233D7
:1002700001EB030C9A420CF801ECF7D8FF2D4FF07C
:10028000FF034FF00E0008BF0222224482F8E83735
:10029000BDE8384013F012BE00EB800004F5B873DF
:1002A0002572C0EB001003EB4000C4F8D4031FF02C
:1002B000ADFA1EF00BFC1EF0DDFCCCE7881E002022
:1002C00088320120703A0120054B0121D3F82C28F7
:1002D00083F8291842F40012C3F82C28704700BF95
:1002E000883201200368C3F30D032DE9F041054670
:1002F00086B00C46002B41D1394A0120394E0221EB
:10030000B242CDE90233CDE9040120D3364B9A4203
:100310001CD303F580439A4224D3344B9A4223D909
:1003200003F580339A4221D903F500339A421FD94D
:1003300003F500339A421DD903F500339A421BD9C5
:100340000A2105200BF080F83DF0EEFB034601A9E1
:1003500002A8039337F024FB80B14FF0FF3006B0C2
:10036000BDE8F0810B46F2E70323F0E70423EEE754
:100370000523ECE70623EAE70723E8E71C4E96F897
:100380004438012B02D16FF00100E8E701232F6808
:10039000D4F8008086F8443837F0A2FAB0B9154C8A
:1003A000236923F440732361236943F400732361B9
:1003B000236943F001032361C7F80080BFF34F8F27
:1003C00037F08EFA236923F001032361002386F8B6
:1003D00044380028D7D12B6804332B60BFE700BF17
:1003E000004000080040000800800008FFFF0008EF
:1003F00088320120003C02402DE9F041594F8AB07B
:100400003B78AF2B6ED1FDF765FD80F00104E4B2BF
:10041000554B04F00104554DB3F89F31544EADF8DF
:100420000030B54260D3002C00F09A8010220021E9
:1004300006A83FF039FF4F4B0497DB1B05934E4B4B
:100440001A69002A05DA4D4A5A6002F188325A6068
:100450001B69012300250222694604A88DF8243077
:1004600008953DF0BBF9022269464FF6FF703F4FF9
:10047000FDF706FC0446B74245D30025022201A938
:1004800004A8ADF804503DF0A9F9022201A92046C4
:10049000FDF7F6FB40BA022202A9C043ADF80800FE
:1004A00004A83DF09BF9079868B106ABC0F10402BF
:1004B000294618443FF0F8FE089818B906A904A880
:1004C000FFF710FF08909DF82430089823B12A4ABE
:1004D000136943F000431361B0FA80F040090AB099
:1004E000BDE8F081012493E7A9881C3555F8140C68
:1004F000C1F30B0137F0D2FA55F8043C1B68834274
:1005000018BF01248DE7B7F8048002A904A88DF86C
:100510000D50C8F30B081C3708F10603ADF808307E
:1005200037F81C3CC3F30B021B0BADF80A20062264
:100530008DF80C303DF052F9062202A92046FDF755
:100540009FFB044657F8141C424604A83DF046F9A8
:10055000204657F8141C4246FDF792FB04468AE7F2
:100560000120BCE700400008741B0508E8010008F2
:10057000E409000800800008003C024023016745B0
:1005800010B51B4CFFF754F90122D4F8AC3784F8AE
:100590004C2803F2DC53C4F8AC37FFF72DFF10B939
:1005A000FFF72AFF60B1134B1B78AF2B02D1FDF789
:1005B00091FC78B90A2105200AF046FF3DF0B4FA13
:1005C000FFF71AFF0028EED10A2105200AF03CFFB0
:1005D0003DF0AAFA084A00230121126884F84C3839
:1005E00084F8C51784F84D38C4F8AC2710BD00BF97
:1005F0008832012000400008C818012010B50B4ABD
:1006000002230B4C0121A37582F80C17FFF7B8FFEA
:10061000FFF7C8FC41F20242FF230E20A4F8E827AE
:1006200084F8EA37BDE8104013F048BC881E00206B
:100630008832012090F88630F7EE002ADFED695A03
:10064000002103EE903A90F88A3006EE103A90F8C6
:100650008830F8EEE33A04EE103A90F88930B8EEBC
:10066000C66A04EE903A90F88C3063EEA57A03EEF9
:10067000903A26EE256AB8EEC44AF8EEE44AF8EE5F
:10068000E33A26EE276A24EE254A64EEA54A63EE95
:10069000A53A24EE064A64EEA74A63EEA73AF0B5FF
:1006A000514D062600F1660EA5F10C0CB7EE005A6E
:1006B00006FB01F290F88570AC180244F0EE456A32
:1006C00015E0012904F1060402F10602EED190F8CA
:1006D000873007EE903A90F88F3006EE903AF8EEB9
:1006E000E77AF8EEE66A27EEA55A66EEA56A237861
:1006F00066EE867A07EE103AB8EEC77A27EE277ACA
:10070000FDEEC77A17EE903A66EE847AFA2BA8BF10
:10071000FA2323EAE3731372637807EE103AB8EE14
:10072000C77A27EE277AFDEEC77A17EE903AFA2BB2
:10073000A8BFFA2323EAE37353725CF8213007EE73
:10074000903A002BF8EEE77A49DDA37807EE103AED
:1007500090F88B30B8EE477A03EE103AB8EEC33A11
:1007600037EE677A23EE253A87EE272AB0EE627AD3
:10077000A2EE037A64EEA77A66EEA36A67EE857A44
:1007800027EE877AFDEEE77ABDEEC77A17EE103ACC
:10079000FA2BA8BFFA2323EAE373937217EE903A79
:1007A000FA2BA8BFFA2323EAE3730EF801300131D4
:1007B000A38807EE903AF8EEE77A67EEA67AFDEEA8
:1007C000E77A17EE903AB3F57A7FA8BF4FF47A73C1
:1007D0008F4223EAE3739381BFF673AFF0BDB7EEA8
:1007E000007AC7E70AD7233CD01F050890F88D3060
:1007F0006BB3B0F85A308BB190F88E20642102EBC5
:100800008203C3EB0313B3FBF1F3A0F85A30962332
:1008100012FB03F3B3FBF1F3A0F85C3043884BB158
:1008200090F88E30642203EB8303C3EB0313B3FB16
:10083000F2F34380B0F846304BB1962290F88E30F8
:1008400013FB02F36422B3FBF2F3A0F846307047C7
:1008500090F821304BB3438B83B190F82230FA22C9
:10086000642113FB02F203EB8303B2FBF1F2B3F555
:100870007A7F4283A8BF4FF47A738383838843B11E
:10088000FA2290F8223013FB02F36422B3FBF2F356
:100890008380C3884BB190F8223003EB8303B3F518
:1008A0007A7FA8BF4FF47A73C3807047034BD3F8A5
:1008B000580D08B106F0AEBC704700BF8832012069
:1008C00008B50B4605490246D1F8580D28B1044930
:1008D000FEF796F8BDE80840E8E708BD8832012039
:1008E000E1E20008024B0146D3F8580DFDF7FABCCF
:1008F0008832012008B504460848FFF7F3FFFFF7E8
:10090000D5FF074BD3F8800013F04AFA0AF04CFAEF
:10091000012C01D13DF008F9FAF72CFF53BC050872
:10092000883201200048DDE753C605080CB4C30631
:1009300007B500D561B905A904980191FFF7C0FF7B
:10094000FFF7F0FF012003B05DF804EB02B0704741
:100950000020F8E708B5FFF7C5FFBDE80840E1E76C
:1009600010B504460348FFF7BDFF2046BDE8104020
:10097000F0E700BF5FBC05080948002408B5FFF791
:10098000EFFFFFF793FF074B83F85C4DC3F85C4E16
:1009900083F8604E1EF00EFA2046FFF7ABFF00BF53
:1009A00064BC050888320120034B0146D3F8580D7A
:1009B00008B106F01BBC7047883201200CB407B5A3
:1009C00010F020000BD079B92320FFF7EDFF05A927
:1009D00004980191FFF774FFFFF7A4FF012003B013
:1009E0005DF804EB02B070470020F8E70FB407B5DC
:1009F00004A951F8040B0191FFF762FF03B05DF801
:100A000004EB04B0704730B52B4885B0FFF76AFFA0
:100A10002A4B1B7923B92A4805B0BDE8304099E735
:100A200033F02CFF08B92748F6E733F03DFF08B94B
:100A30002548F1E7254B1B68DB6998470028F7D06C
:100A400033F03AFF02680446037D81795208407C06
:100A5000E51D0C34029020790190E08800901C483C
:100A6000FFF7C4FF15F8010BFFF79EFFA542F9D170
:100A7000184C1948FFF736FF6378022B06D007D9C8
:100A8000032B10D11548FFF72DFF0CE01448FAE7AF
:100A900004F580541348FFF725FF94F8E437022B40
:100AA00005D0032B05D005B0BDE830403AE70E482D
:100AB000E9E70E48E7E700BF8BBC0508CC2801201A
:100AC00095BC0508A4BC0508B2BC0508C4180120E3
:100AD000C1BC050818570120EFBC0508FFBC05087C
:100AE00005BD050812BD050818BD050831BD05087E
:100AF0000FB407B504A951F8040B0191FFF7E0FE0C
:100B0000FFF710FF03B05DF804EB04B070472DE968
:100B1000F041037903F0E002402A4AD004D85AB1E8
:100B2000202A23D0BDE8F081602A45D0802AF9D15F
:100B30008279417922480BE003F00703022B02D0AF
:100B4000042B08D06BB9B0F80720B0F805101D4889
:100B5000BDE8F041CCE7D0F805101B48BDE8F041F6
:100B6000C6E7B0F90720B0F90510F0E74679002490
:100B7000164D174805EBC605FFF7B4FE012395F89F
:100B80007474A74202D8BDE8F041CBE6D5F8706492
:100B90004FEA840856F824204AB113B90D48FFF7EC
:100BA000A1FE56F808100C48FFF720FF002301347F
:100BB000E7E741790948D1E70948BDE8F04197E7FF
:100BC00095BD050859BD050843BD0508741B0508FA
:100BD00070BD050881BD050884D1050884BD0508E0
:100BE000ACBD05080249034801F521610EC97FE744
:100BF0000070F01FC4BD050810B5752104461FF034
:100C0000D7FF01460948FFF773FF1A2120461FF05E
:100C1000CFFF01460648FFF76BFF1B2120461FF060
:100C2000C7FF01460348BDE8104061E7D8BD05088D
:100C3000EBBD0508FEBD050838B50B4DE87810F092
:100C4000FD0405D10948FFF753FF2046FFF7D4FF05
:100C5000EB78013B012B06D80548FFF749FF01203F
:100C6000BDE83840C8E738BD7819012011BE050835
:100C70001CBE0508B44BB5491A68B54B2DE9F04FB9
:100C8000B44C93B00746B448B44EDFF86883DFF83D
:100C90006893DFF8F0A2B2FBF3F2FFF7A7FEB4F817
:100CA000622E4FF47A730A20B2FBF3F103FB112298
:100CB000B4F9643E92B2B2FBF0F2A948FFF718FF14
:100CC000A84AA949A948FFF791FEFFF72BFEA17D8D
:100CD000A74A06EB8101A74BA748D31AD1F82016E3
:100CE000A288FFF705FFA548FFF7FCFD94F8661EF4
:100CF000A348FFF77BFEA348FFF7F4FD94F8671EB7
:100D0000A148FFF773FEFFF70DFEA048FFF7EAFDCD
:100D100000210A4698F81F304D1C0B4113F0010FBB
:100D200008D012B15046FFF7DDFD29464846FFF7CF
:100D30005DFE0122072D2946ECD1954D95F86A15E7
:100D400005F5EC7305F13C02012918BF134693F831
:100D5000DC30032B02D08F48FFF748FE8E4B95F80E
:100D60006A15A3F5CE72012918BF134693F8DC303B
:100D7000012B02D18948FFF739FE874B95F86A1598
:100D8000A3F5CE72012918BF13461B695B7B012BAB
:100D900002D98348FFF72AFEDFF86082FFF7C2FD21
:100DA0000025D4F8683E08F12009DFF854B2039317
:100DB00058F8041B31B3012303FA05FA039B1AEA1E
:100DC000030F1DD01AF01F0F1AD0764B59F82520AB
:100DD000585D52F8202035B17348CDE90412FFF771
:100DE00081FDDDE904125846FFF700FEBAF1020F5B
:100DF00006D16E4B93F8A11011B16D48FFF7F6FDC7
:100E00000135D5E7FFF78EFD94F8B61CD4F8B82C61
:100E100006EB81016748137AD1F86016527AFFF722
:100E200067FE65496548FFF7E1FD65496548FFF7DD
:100E3000DDFDFFF777FD644B644819684FF47A7362
:100E4000B1FBF3F1FFF7D2FD07A8FEF7BDFB38B108
:100E500007A90AA83CF0C0FD0AA95D48FFF7C6FD36
:100E6000FFF760FDD4F8F42E002A5AD007EE902A3E
:100E7000DFED586AB8EEE77AC6EE877AFDEEE77ADC
:100E800017EE903ADFF87C81B8F8740458B107EE99
:100E9000900ADFED506AF8EEE77A86EEA77AFDEE6B
:100EA000C77A17EE900AD4F8745E5DB107EE905AD7
:100EB000DFED486AF8EEE77A86EEA77AFDEEC77AAC
:100EC00017EE905A3949B1F8DC106429CDE90005D4
:100ED000A8BF64214048FFF70BFE98F8763498F8D5
:100EE0007724012506EB8303B8F878143B48D3F840
:100EF0007436FFF7FDFD3A4B3A48198889B2FFF77F
:100F0000F7FD38463849FFF77EFD3848FFF7EAFC21
:100F1000374FD4F82C4834B9FFF704FD13B0BDE8BF
:100F2000F08F1346AEE794FAA4F33846B3FA83F38E
:100F300005FA03F206EB8303D3F8881624EA0204C9
:100F4000FFF754FDE7E700BFE419012027BE0508BD
:100F500040420F00883201202CBE0508741B050892
:100F60003FBE0508000001200008000060BE050823
:100F7000008000080040000884BE0508B3BE0508D4
:100F8000C5BE0508CDBE0508CFBE0508D7BE0508FD
:100F9000881E0020F0BE050860200020F8BE05086D
:100FA000FDBE0508CC03012081BD0508802F00206F
:100FB0000BBF05080FBF050821BF050842BF050884
:100FC00050BF050856BF0508C81801205CBF0508BA
:100FD00076BF05080024744989BF0508CFBF0508FE
:100FE000701B0120F6BF050851D3050805C0050890
:100FF00079C3050878190120E7BE0508A021050876
:1010000005BF0508804301202DE9F04FDFF874810A
:1010100099B098F80B30002B00F0978050480025CD
:10102000504EDFF864B1FFF795FC2F46DFF85C9176
:10103000DFF85CA10BA9E8B215F08EFF9DF8343003
:10104000002B53D0139C54B107EE904A9FED460AF3
:10105000F8EE677A80EE270A3EF03AFC04460B9AD7
:1010600029465846FFF7C2FC109A002A6FD002FBAF
:1010700004F04FF47A73B0FBF3F30993DDF848C042
:10108000BCF1000F65D00CFB04F142F21073B1FB10
:10109000F3F1082D98F80B3018BF7F18002B5AD0A9
:1010A00017984FF47A7E0A230790159806901698A1
:1010B00005901198B0FBFEFECDF810E00998B1FB49
:1010C000F3FE03FB1E11CDE902E10999B1FBF3F137
:1010D00003FB1100BCFBF3F3CDE9001021465046A1
:1010E000FFF706FD0023B362C6E90D330135403634
:1010F0001C2D9FD198F80B3023B31C4C4FF47A73FE
:101100001B48D4F88014D4F88424B1FBF3F3D2083C
:10111000D4F88814FFF7ECFC0A221648B7FBF2F16A
:1011200002FB1172FFF7E4FC134B1B78432B06D133
:10113000D4F88C24D4F890141048FFF7D9FC00237D
:10114000C4F8883419B0BDE8F08F0D4867E70992FC
:1011500094E761469DE721464846FFF7C9FCC1E791
:101160001BC00508F44001208096184B80430120E5
:10117000C2C00508E2C00508542B012006C10508BD
:1011800079C005088832012083C00508E2D205082D
:1011900092C0050838B52748FFF7A4FB264B93F803
:1011A0000134002B43D02548FFF7D4FB244C16F024
:1011B00011FD40B1B4F850512248FFF793FB2DBB0D
:1011C0002148FFF7C7FBB4F846112048FFF70EFC93
:1011D00094F844312BB31E48FFF7BCFBB4F84C1114
:1011E0001C48FFF703FC94F84A31E3B11848FFF7B5
:1011F000B1FBB4F848111848FFF7F8FB94F84531F3
:101200009BB11348BDE83840FFF7A4BB4FF47A7296
:101210001248B5FBF2F102FB115292B2FFF768FCE3
:10122000D1E70F48D8E70E48E1E70D48EAE70D4857
:10123000E8E700BF30C105088832012046C1050833
:10124000802F00204DC1050868C105087CC1050834
:101250009CC10508ACC10508C6C1050872C10508D6
:10126000A5C10508E7FD05080EB403B503AA52F8A9
:10127000041B0192FDF70CFE064BD3F8582D22B942
:101280000549D3F88800FDF72DF802B05DF804EBAE
:1012900003B070478832012053C605082DE9F04796
:1012A00015460A7981460F4602F0E0049846402C24
:1012B0002DD10024DFF874815B4EDFF8949115E0A6
:1012C0003B7903F00703013B032B03D8DFE803F06E
:1012D0001315181B295D3046FFF788FB7B79013B0E
:1012E000A34202DD4846FFF7FDFA01347B79A342B1
:1012F000E6DCBDE8F0872957EDE735F81410EAE79A
:1013000035F91410E7E755F824104046E4E702F0F9
:101310000702042A3ED8DFE802F0030C1416190075
:101320002E78602C44D02BD8002C4CD0202C61D0AF
:10133000DFE795F90060602C3AD021D8002CF5D178
:101340002EE02E88EDE7B5F90060F4E7D5F800A0AF
:10135000202C56464ED011D8002CCAD151463348C5
:10136000FFF744FBD7F805108A4553D8B8F1000FB2
:10137000BFD02F48BDE8F047FFF738BB602C17D02F
:10138000802CB6D129782B4B2B48002914BF294635
:101390001946EFE7202C2CD007D8002CA9D12646DF
:1013A000B7F90540B7F9075011E0602CE8D10026E5
:1013B0007B7946FA03F3DB07BDE8F0474CBF1F48D3
:1013C0001F48FFF713BBB7F80540B7F80750314681
:1013D0001548FFF70BFBB4421CDCB5421ADBB8F131
:1013E000000F86D02A4621461648BDE8F047FFF791
:1013F000FDBA00267A79144B03EBC20393F87424E8
:10140000B24207DDD3F8703453F82600BDE8F04748
:10141000FFF768BAFFF786FA33463A6848460B4941
:10142000BDE8F04720E700BF6DBD050856BD0508C3
:10143000E6C1050823E7050884D10508C1BD0508F4
:10144000E7FD050853BB0508741B0508ECC105083A
:10145000CDBE050813B50446084601920091FDF77C
:101460009FF802462046DDE9001302B0BDE81040B7
:1014700014E70EB403B503AA52F8041B0192FDF75A
:1014800007FD054B0549D3F88800FCF72BFF02B098
:101490005DF804EB03B070478832012053C605089D
:1014A00002460149E5E700BF06C20508154BD3F81F
:1014B000A0392DE9F041044688B0F3B11A6804A9B7
:1014C0001846D56A6A46A847064688B104AC6D46F8
:1014D0000027DFF83C80013735F8022B34F8021B77
:1014E0004046FFF705FBBE42F5DC08B0BDE8F081E1
:1014F00005492046FFF7BDFFF7E7044908B0BDE8FE
:10150000F041B6E78832012037C205084FC205080E
:101510001DC2050813B50446084601913CF03AFD8A
:10152000024670B10D2804D1019909483EF0D8FF58
:1015300038B1074B2046074A074902B0BDE81040C2
:1015400097E70349054802B0BDE81040FFF7D0BA5D
:101550004C7B050856C2050861C205088BC2050808
:1015600013B50446084601913CF014FD019902466A
:1015700068B1042803D109483EF0B2FF38B1074BE7
:101580002046074A074902B0BDE8104071E7034909
:10159000054802B0BDE81040FFF7AABA447B050831
:1015A00099C2050861C20508A9C205082DE9F043E2
:1015B00000279BB0064608460C463CF0EBFC05466F
:1015C0001C22394602A801973EF06EFE25B3402D3D
:1015D00007D040232A46384930461BB0BDE8F043C7
:1015E00047E70DF1040804F140090222214668464C
:1015F0003EF08AFF0023102209A968468DF8027088
:10160000FDF72AFE099B0DF10202934222D102341A
:1016100008F8010BA145E8D100213D220AA8099153
:101620003EF042FE002D3AD0244C257ED5B120223A
:1016300004F11C0101A83EF00DFE98B104F11C015B
:1016400009A8FDF701FD09AB1D4A30461D49FFF70A
:1016500010FF04E01A7830461B49FFF70AFF1BB061
:10166000BDE8F08394F88430CBB9C5B901AD174C0F
:101670000FCD0FC495E80F0084E80F00144B012232
:1016800009A8A4F1100183F89424FDF7DDFC1148AA
:10169000FFF766F909A91048FFF72AFADFE70C4BB4
:1016A00093F894341BB9054B1B7E002BF2D00749ED
:1016B00009A8FDF7C9FCEDE7BCC205088832012086
:1016C000FAC2050861C20508DEC20508A43201207D
:1016D0008043012004C3050813C305082DE9F74F13
:1016E0003D4F834608460D463CF054FCD7F8049520
:1016F0000446B8B9394D0126394F3A48FFF7F2F898
:1017000055F8041B49B106FA04F313EA090F02D095
:101710003846FFF76BF90134F2E703B0BDE8F04F4C
:10172000FFF700B9024630492846FDF745FD78B974
:101730002A4C2E4D2E48FFF7D5F854F8041B0029EB
:10174000EBD00B78002BF8D02846FFF74FF9F4E7E1
:101750002B782D2B11D10135013C4FF0010A1F4B85
:10176000002653F8048BB8F1000F09D12A4621490D
:10177000584603B0BDE8F04F7BE64FF0000AEEE7B5
:101780002246414628460193FDF716FD019B00BB0A
:101790000123B3409A0505D5174803B0BDE8F04FC3
:1017A000FFF7D8B8BAF1000F0DD029EA03031348A8
:1017B000C7F80435FFF796F841460C4803B0BDE87A
:1017C000F04FFFF795B949EA03030D48C7F8043510
:1017D000F0E70136C5E700BF883201206422050822
:1017E0002AC3050820C305087EC0050879C305087B
:1017F0002EC3050839C305084AC3050856C30508A2
:101800005FC305082DE9F74F814608460E46174687
:1018100098463CF0BFFB0446E8B9404D4048FFF70E
:10182000E5F820460DF0C8F93B68184206D020467E
:101830000DF0D4F901462846FFF7D8F80134182CEA
:10184000EFD13B6813B93748FFF74CF803B0BDE858
:10185000F04FFFF767B8024633493046FDF7ACFC5E
:101860000546A8B92C46314D3148FFF73BF82046D4
:101870000DF0A2F910EA080F06D020460DF0AEF9DF
:1018800001462846FFF7B2F80134192CEFD1DDE705
:1018900033782D2B2AD10136013C012548F0807385
:1018A0004FF0000A019350460DF098F92246834606
:1018B00001463046FDF780FC18BB50460DF07CF920
:1018C000019B03421DD09DB1BAF1180F02D03B68B5
:1018D00040EA03081748C7F80080FFF703F85946A5
:1018E000124803B0BDE8F04FFFF702B90025D5E775
:1018F000BAF1180F02D03D6825EA00050E483D6098
:10190000EBE70AF1010ABAF1190FCCD132460B49C3
:10191000484603B0BDE8F04FABE500BF78C305080B
:1019200067C3050871C305087EC0050879C30508AB
:101930002EC3050856C305085FC3050839C305084B
:1019400040F20223004A5DE7843801206FF07F43B4
:10195000004A57E77C3801202DE9F04F074691B047
:1019600082480E46824DFFF7C3F800238149402488
:10197000062285F89C343046012391F89015C5F86D
:1019800098D485F89D4409F08DFA0A2009F0FEFCF0
:1019900095F89C340C2BDAB240F2E4809DF80C50A0
:1019A000FE2D30D0FF2D0BBF15240F24012600265D
:1019B000944240F0D780611E6846C9B22CF03AFCD0
:1019C00004F140030DEB030414F8413C834240F062
:1019D000C48006F1FF389DF80D305FFA88F8B8F141
:1019E000010F12D903F01F075C0961376248FEF747
:1019F00079FF022E6AD0013C042C65D8DFE804F0A0
:101A00000B5E606462000226D2E79DF80E701D46F0
:101A10009DF80F40EAE759486C464FF0000ADFF89E
:101A2000B891FEF797FFDFF8B4B15548FEF75AFFBB
:101A30000AF1010A14F8011B4846FEF7D7FFBAF174
:101A40000C0F49D1FEF76EFF022E4FD064223B46A9
:101A50004C48B5FBF2F102FB1152C9B2D2B2FFF70A
:101A600047F8B8F1010F71D8474A484B9DF810105C
:101A70004748002914BF11461946464DFFF738F86C
:101A80009DF81110444B4548002914BF19462946BA
:101A9000FFF72EF8022E59D19DF812404048FEF76C
:101AA00021FF4CB3FF2C37D00A223E48B4FBF2F1A1
:101AB00002FB1142D2B2FFF71BF820E03A48ABE735
:101AC0003A48A9E73A48A7E73A48A5E700230DF1C5
:101AD0001F008DF83F309FE7374B03FB0AF2B2F14E
:101AE000553FA5D85846FEF7FDFEA1E73A462946E0
:101AF0003248FEF7FDFFB7E72846FEF72BFF9DF8BB
:101B000013402F48FEF7EEFE44B1FF2C21D02146B2
:101B10002C48FEF7EDFF04E02B48EEE71D48FEF7EA
:101B200019FF0DF1130500241A4E274FDFF86880C6
:101B300015F8013F7BB1FF2B0CBF3A4642462146C8
:101B400001342248FEF7D4FF042CF1D111B0BDE8D6
:101B5000F08F1D48E3E73246F1E71D493846FFF7AD
:101B600088FCF3E71B48FEF7F5FEEFE79DC3050889
:101B700080430120881E0020AEC30508B9C30508B4
:101B8000E7C30508F9C305087DC3050886C3050832
:101B900030C405088DC30508CED0050847C4050824
:101BA0004EC4050862C40508C0C30508C8C30508BB
:101BB000D0C30508DFC30508ABAAAAAA15C4050847
:101BC0006AC405086DBD050891C305087AC40508F7
:101BD00085C4050895C4050846BC050823E7050823
:101BE0002DE9F84F07460C46DFF8A480DFF8849013
:101BF000DFF8A0A020463CF0CDF9064660B91D4BA9
:101C00001D4893F8D8231D4B03EB8203D3F86817C4
:101C1000BDE8F84FFEF76CBF024641462046FDF78F
:101C2000CBFA58B1DFF85CB000255BF8041BA9B90A
:101C3000224638461249BDE8F84F1AE4114C124DBD
:101C40001248FEF74FFE54F8041B19B12846FEF760
:101C5000CDFEF8E7BDE8F84FFEF764BE32462046F9
:101C60000135FDF7A9FA0028DFD1544689F8D85389
:101C7000C0E700BF883201209EC40508741B050818
:101C800039C30508E022050879C305082EC30508F5
:101C90007EC0050851D3050838B50D460446052217
:101CA00019492846FDF788FA68B9184B93F88C2033
:101CB00022B9012183F88D2083F88C101448BDE8E7
:101CC0003840FEF747BE032212492846FDF774FA52
:101CD000A0B90E4D95F88C3063B195F88D304BB1AD
:101CE0000D492046FFF7C5FB002385F88C3085F8A9
:101CF0008D3038BD0948FEF72DFEF5E7204608492E
:101D0000BDE83840FFF7B5BB19D00508883201207F
:101D1000A8C4050877D10508BEC40508F5C40508A0
:101D200009C5050808B5034610462AB1DB0600D5EB
:101D300011B1FEF715FE002008BDF8B50D4E0546A1
:101D400096F8843093B9F8BD25B12388C3F30B030B
:101D50009D4204D0A288D4E902013EF031FA1C343D
:101D6000BC42F1D3002386F88430ECE7024C034FE9
:101D7000F6E700BF88320120E8010008E409000806
:101D80000A4B93F8843010B504460BB904F0C8FF31
:101D9000FCF784FC44B1012004F05EFF20B9044844
:101DA000BDE81040FEF7D6BD10BD00BF883201204F
:101DB00018C505082DE9F04F164685B01A4682462B
:101DC000019130460021334CFFF7ACFF4FF0000982
:101DD00006F0100305460293FEF768FD2379019A89
:101DE00003F01803934203D0002A48D1182B46D1A0
:101DF0004FF00D0B274B0BFB0933B3F80900FCF731
:101E0000B9FB80462046FCF7E0F80746D8E90221F6
:101E1000024401442046FCF791F880F001012A4673
:101E20000390C9B23046FFF77DFF0546DDE9022386
:101E300002B123BB174A0BFB09FB52F80BB0B206E9
:101E40000FD573B9594614480393FEF7CFFDD8F860
:101E500008202146039B50463A44FFF71FFAFEF73D
:101E600061FD59460D48FEF7C1FDD8F80C2000234E
:101E700021463A445046FFF711FAFEF753FD09F1A7
:101E8000010940F23A230D349945A5D105B0BDE8CA
:101E9000F08F00BF0032050840C5050841C50508A0
:101EA0000149FFF7E6BA00BF4BC505082DE9F0432D
:101EB000064687B008460C463CF06CF8082844D12A
:101EC000671E03AD073429463A46A84612F8010FAB
:101ED000FDF748F901F8010BA242F7D10023DFF822
:101EE00080908DF8143017F8010FFDF73BF905F8D5
:101EF000010BC1B2484601913EF0DDFA20B10199D3
:101F000028463EF0D8FA28B13046FFF7C9FF07B09F
:101F1000BDE8F083A742E6D1104940461EF016FB0B
:101F20000E4808230E4910F8012B013B11F8014B14
:101F300002F118026A4402F80C4CF4D103A90948D2
:101F40008DF81430FEF7D4FDE1E70028E8D03046E4
:101F500007B0BDE8F043FFF7A3BA00BF6836012021
:101F600038BB05085AC5050807B5009313460A464D
:101F70000249FFF77EFA03B05DF804FB61C505086E
:101F800020B10078B0FA80F0400970470120704716
:101F90002DE9F34106460846FFF7F2FF0D460746D6
:101FA00070B1002401A92046013435F09BF90146A7
:101FB0003046FFF7EDFF122CF4D102B0BDE8F081FE
:101FC0000846FDF7EDF9C4B2112C72D8681C3D4DDE
:101FD000FCF708F98046E8B93B4B03EB440393F860
:101FE000A0148A1E51425141374B03EB440393F82E
:101FF000A024AA5C002955D093F8A134192040F2FE
:10200000EE2100FB03132146304802B0BDE8F04149
:10201000FEF76EBD017828463EF04DFA78B1032CEC
:102020002B49A0EB050394BF0022012202EB4202E0
:102030000A4452FA83F393F8D877032F04D1304639
:1020400002B0BDE8F0412BE74046FCF7CBF808B3FF
:10205000022FF4D1FDF7A4F940F6CA0280B21A4B60
:10206000904203EB4403A8BF104640F2EE22904298
:10207000B8BF10461922A0F2EE20B0FBF2F083F8B0
:10208000A104BB1E594259410F4B03EB440383F893
:10209000A074A9E7022FF4D1304602B0BDE8F041A8
:1020A000FFF7FEB921460B4802B0BDE8F041FEF74C
:1020B0001FBD11233A460849304602B0BDE8F04141
:1020C00052E700BFA08E0508804301207AC50508AD
:1020D000741B05088AC5050897C505082DE9F04F4A
:1020E000024691B008460B46FFF74AFF044628B166
:1020F000104611B0BDE8F04FFFF7D2B94FF0FF32F4
:1021000027462646DFF8E482DFF8E492DFF8E4A20F
:10211000CDE90820A34AD2F8802092F83810CDE902
:102120000E02CDE90C10CDE90A0007AA9E49184617
:102130003EF07CF8054604944DB9089A0C9FBA42CB
:1021400062D19A48FEF7D4FC11B0BDE8F08F062F9B
:1021500012D8DFE807F0041E2328454C51005146F1
:102160002846FDF74DF878B14FF4806001240CF05B
:1021700031FF90F90430089307AA8B4900200137FA
:102180003EF054F80546D7E72846FDF709F90890D0
:10219000F2E72846FDF704F90990EDE72846FDF738
:1021A00046F80A90E8E728463BF0F4FE414602462E
:1021B00005902846FDF700F818B3059A49462846C9
:1021C000FCF7FAFF06460028D6D02846FDF7E8F8C7
:1021D00004280646D0D901467548FEF789FCB3E7C6
:1021E0002846FDF7DDF800230C900F93C4E728463E
:1021F000FDF7D6F80D90BFE72846FDF718F80E90CA
:10220000BAE701230493B7E7DFF8EC8151B2434604
:1022100013F9010B884208D00135092DF8D10021AE
:1022200001316448FEF764FC8EE701216248FEF745
:102230005FFC00237AB218F9011B8A4200F00D817D
:102240000133092BF7D13A460121E9E7A7F114023E
:1022500053425341059308AD002303F10108EB6895
:10226000A3BB95F900B058460CF080FED5F804A049
:1022700020B1D0F80090B9F1000F5ED1BAF1000F93
:1022800019D14FF461434FF0010A6B60AB680BB991
:102290000323AB600023D5F80490584602931946F7
:1022A0002A7ACDE900921A4611F0B2FCE86028B90A
:1022B0004146424891E74FF0000AE7E74A46414667
:1022C000BAF1000F37D03E48FEF790FBB8F1020F8D
:1022D00005F110054FF00103BFD1059BDDF83C80EF
:1022E0000B9D53B13748FEF735FBD8F800301B6A19
:1022F0001BB12A46344940469847049B002B4ED0D8
:102300003249334B142F18BF19463248FEF7F0FB01
:10231000142F09D1049B03B936B12B68DB691BB1BB
:1023200032462D4928469847002C67D10022414665
:10233000284634F08BFF2948C6E7C5F80C90BAF15F
:10234000000F25D0414626485246FEF74FFB514626
:10235000484603F0B3F9D5F808A0BAF1000F0FD042
:1023600099F8042092450BD0534641461D48FEF78C
:102370003DFBD9F800305FFA8AF148469B699847DF
:10238000D9F82C30002BA1D00023C9F82C309DE7C0
:10239000D9F8082041461448FEF728FBDBE70C4932
:1023A000B3E700BF8832012062BC0508D5C5050827
:1023B000BDC5050819C70508EEC50508FAC5050815
:1023C00016C60508CDC60508BD5601089FC50508F7
:1023D00051D30508F6C6050809E300083AC6050802
:1023E00056C60508A8C6050883C60508B7C505086A
:1023F00073C30508ACC50508801E05081C4F0026E0
:10240000DFF874904FF0030A05F006FD052008F090
:10241000BDFF99F89035B34288D917F801BBBBF1DD
:10242000000F15D0584609F03DF9044680B15846D2
:1024300005F002FC08B1A0F806A00121049005F007
:1024400067FCE379049813F0010F03D004F0EEFE6B
:102450000136DEE704F0F0FEFAE73A4602210548CD
:10246000FEF746FB099B002B3FF4F0AE0023F1E69C
:10247000CC1B0120EEC50508881E002010B50446BF
:1024800008460B46FFF77CFD28B903220849184689
:10249000FCF792FE28B90748FEF762FA0120FEF722
:1024A00029FA20460449BDE81040FEF7E2BF00BF0C
:1024B0002BC705082FC7050809C505082DE9F74FE3
:1024C00005460846FFF75CFD0B46044618B9334A3B
:1024D00092F8C47427B9284603B0BDE8F04FDFE492
:1024E0002646DFF8C880DFF8C89001AADFF8C4A04C
:1024F00018462B493DF09AFE10B905F09BFC07E009
:102500004EB90146284634F001FE421C04461BD158
:1025100003B0BDE8F08FFCF743FF2F28834636D881
:102520000FB105F079FCBBF1060F14D01D49012352
:102530005FFA8BF291F89015E0B208F0B3FC002737
:1025400059464846FEF7D4FA01AA1549002001363B
:102550003DF06CFED0E7DAF808351B0113D5FF2CEF
:102560000FD0E1B22846FFF7F7F9E8E70137284630
:10257000FFF7F2F90B4BF9B293F890258A42F5D8A0
:10258000DDE70027F6E70848FEF7E4F9D7E72F2252
:1025900041462846FEF76DFFD6E700BF8043012085
:1025A00062BC0508881E002051C7050871C70508D0
:1025B00060C70508883201202DE9F74380460846A8
:1025C000FFF7DEFC0B46054628B14046FEF768FFE4
:1025D00003B0BDE8F08301AA2D4918462F463DF00F
:1025E00025FE2E460446DFF8A8907CB9022DECD1DA
:1025F000A7F57A73B3F57A7F20D94FF4FA634FF4D5
:102600007A7224494046FFF7AFFCE1E74DB1012D56
:102610000FD001AA4946002001353DF007FE0446CF
:10262000E3E72146404634F071FD431C0646F0D1F5
:10263000CEE72046FCF7B4FE0746EAE7164BB8B2F1
:10264000D3F880305B689847FF2EBCEEC00A134B6E
:102650000CD1134AF8EE407A92F89025A24212DC8F
:1026600010EE101A0F48FEF743FAB1E7F8EE407A81
:1026700003EB860310EE102A31460B48C3ED007AB7
:10268000FEF736FAA4E70134E3EC017AE6E700BF8F
:1026900062BC050881C80508802F00204848012039
:1026A000881E00209EC7050891C70508F8B5074693
:1026B0000846FFF765FCC8B11F4BDE6C013630469B
:1026C00034460CF08BFA0546F0B90134192CA8BF3A
:1026D000002420460CF082FA0546A8B9B442F4D191
:1026E00038461649BDE8F840FEF7C3BE0846FCF779
:1026F00057FE04460CF072FA054628B921461048E8
:10270000BDE8F840FEF7F4B90B4BDC6411F0A0FB18
:102710002A4621460B48FEF7EBF9182C09D80A483F
:102720000C2101FB040090F8E007BDE8F84011F02F
:10273000C5BB0020F9E700BF88030120ADC705082D
:10274000C1C70508D7C70508741B050838B5044676
:10275000114D0846FFF714FC68B1104B93F90010B7
:102760004B1C06D10E4B197A0E48BDE83840FEF7D7
:10277000BFB9C9B2F8E70846FCF712FE032804D82F
:10278000C0B2FDF75FFD2946E3E720460322064974
:10279000BDE83840FEF76DBE51D30508880301201F
:1027A00088320120F0C7050800C8050838B504467E
:1027B000114D0846FFF7E4FB68B1104B93F9011087
:1027C0004B1C06D10E4B597A0E48BDE83840FEF737
:1027D0008FB9C9B2F8E70846FCF7E2FD032804D830
:1027E000C0B215F01FFD2946E3E720460322064943
:1027F000BDE83840FEF73DBE51D3050888030120EF
:1028000088320120ECC70508FBC705082DE9F74F02
:10281000414B0026DFF818A105461A7AB1465B7ACB
:1028200001203E4C88468AF800208AF80130FFF7E4
:10283000A7FA0D23394A4146734352F803B058466C
:10284000FCF7DEFC002841D0B9F1000F01D0FEF703
:1028500069F859463248FEF7C9F800222146284651
:10286000FEF7F8FDFEF75EF8237903F01803082B56
:1028700045D0102B48D02046FEF749F9274A0D23B2
:1028800003FB0623B3F80900FBF774FE0746D8B133
:102890002046FBF79AFB0090D7E90221024401444D
:1028A0002046FBF74BFB78B9594601901D48FEF7CF
:1028B0009DF8019AB96828461346009A0A442146B1
:1028C000FEF7ECFCFEF72EF809F10109013640F2A3
:1028D0003A230D349E42ACD10020FFF72EFAFF239D
:1028E0008AF800308AF80130B9F1000F11D1424660
:1028F0000D49284603B0BDE8F04FFEF7BABD0B49BD
:102900002846FFF723FFB6E708492846FFF74EFFA2
:10291000B1E703B0BDE8F08F88320120003205082E
:1029200045C505081BC8050839C3050851D3050866
:10293000880301202DE9F74F804608460F463BF0FB
:1029400029FB044620B1012825D13B782A2B22D12E
:10295000A84E00254FF00D0BDFF8B892B24640F2BA
:102960003A27A548FDF7F6FF0BFB05F3484601356E
:102970005AF80310FEF73AF8221E3146404618BFB7
:1029800001220D36FEF766FDFDF7CCFFBD42EBD10F
:1029900003B0BDE8F08F3D2138463DF08CFD0028A6
:1029A00000F0218103469A4613F8012D202AFAD01F
:1029B000AAEB070A0130054610F8013B202BFAD09C
:1029C0004FF00009DFF82CB20D235FFA8AFA03FBFF
:1029D00009F25BF802100BEB0204084601913BF090
:1029E000D9FA0199024600903846FCF7E5FB0D2321
:1029F0000646002853D1009A524550D1277907F056
:102A0000E003402B00F0B8800ED8002B55D0202BCF
:102A100000F08A8040467949FEF72BFD204603B03E
:102A2000BDE8F04FFEF773B8602B7ED0802BF1D15C
:102A300028463BF0AFFAE3790646A779DB070CD5C9
:102A40002046FBF7ADFD0378014633B132462846F8
:102A50003DF046FD002840F0C080002E00F0BD8013
:102A6000B742C0F0BA800D23204603FB09B393F8A8
:102A700005A0FBF795FD3A4600213DF015FCB24557
:102A80002CD832465E4928463DF02AFD30B3204618
:102A9000FBF786FD324629463DF036FD1EE009F182
:102AA000010940F23A22914591D13A4655494046B2
:102AB00003B0BDE8F04FFEF7DCBC07F00702042AC4
:102AC0001CD119460A222846FCF7C6FBD4F805306B
:102AD000014683429ED32046FBF77AFD0D234A48E8
:102AE00003FB09F95BF80910FDF780FF002221467E
:102AF000404603B0BDE8F04FFEF7ACBC2846FCF7FB
:102B00004FFCB4F80550B4F8071017F0050FAAB23F
:102B10008BB201D02AB20BB29042FFF67BAF984243
:102B20003FF778AF0146D6E76679384A002702EBCF
:102B3000C606BA463B4696F874240092009ABA42FA
:102B400002D9BAF1000F03D0002B3FF463AFC5E701
:102B5000D6F8701451F8270060B129460193FCF7AC
:102B600007FB019B30B94FF0010A39462046FBF7BD
:102B70002FFD53460137E1E707F007076379013F6F
:102B80000093009BB342A9DDAA4615F8013B202B18
:102B9000FAD02046FBF704FD0546032F03D8DFE8F3
:102BA00007F0020D0D135046FCF7FAFBA8552C2137
:102BB00050463DF080FC0136451CE2E75046FCF7EC
:102BC000EFFB25F81600F2E700230A2250461946CB
:102BD000FCF742FB45F82600E9E73A460C49404637
:102BE000FEF747FC16E73946404603B0BDE8F04F14
:102BF0000CE600BF003205082BC8050879C8050897
:102C000023E7050839C305086EC80508741B0508C5
:102C10003EC8050845C505082DE9F04F914689B025
:102C20000C461A46002180464D46FFF77BF80027E8
:102C30000646DFF8E0B0B9F1000F69D02946062258
:102C400020463DF007FB00283246404613BF0121D5
:102C500000214FF0010A4FF0000AFFF763F8064623
:102C6000287812F0DBF9079010B3687912F0D6F9E2
:102C7000079B4FF461714FF0190C5B79EA78079369
:102C8000AB781CFB021295F801E01CFB03132979B9
:102C900000B14079CDF804E0CDE90232079B5A46F5
:102CA000CDE90410009351463B464046FDF786FEB1
:102CB000207812F0B3F9079010B3607912F0AEF9F2
:102CC000079B4FF461714FF0190C5B79E278079321
:102CD000A3781CFB021294F801E01CFB031321797A
:102CE00000B14079CDF804E0CDE90232079B5A46A5
:102CF000CDE90410009351463B464046FDF716FED1
:102D0000013706340635142F95D109B0BDE8F08F90
:102D1000CA46CDE787C805082DE9F041064686B0CA
:102D200008460F46FFF72CF9054638B100235C49E9
:102D300001201A4606B0BDE8F0416DE70846FCF7F1
:102D40002FFB1328044600F3A28006268DF81750A7
:102D5000544D4643781CFBF745FA074670B1FCF723
:102D60001FFBC0B212F070F940B1AB19027983F8C1
:102D700060259DF8173001338DF817303846FBF782
:102D800031FA074668B1FCF70BFB0D2809D806237A
:102D900003FB045383F861059DF8173001338DF868
:102DA0001730DFF8FC80B11C0DF1170238464144A2
:102DB000FCF7FAFAFBF716FA074668B1FCF7F0FAE7
:102DC000012809D8062303FB045383F864059DF802
:102DD000173001338DF817303846FBF703FA80B10E
:102DE000FCF7DEFAC0B212F02FF950B106230279D7
:102DF00003FB045383F865259DF8173001338DF8E4
:102E000017309DF817200623042A2FD103FB045303
:102E10000022A3F8642516F035FE06234FF46176F0
:102E200003FB045595F8600512F0F8F895F8632552
:102E300095F862751923804695F8650513FB0767B9
:102E400013FB026612F0EAF84379214698F8052050
:102E5000039395F8643514480097CDE9016395F81C
:102E60006135FDF745FE06B0BDE8F081052A05D1C4
:102E700003FB0453002283F86525CCE7062ACAD059
:102E8000002308EB060248F806309380C3E71323BB
:102E90002A460649304606B0BDE8F041FFF764B85F
:102EA000E83701208832012087C80508A0C8050836
:102EB0002DE9F04F174689B01A460C46002181468D
:102EC0003D46FEF72FFF3A4E07F16C038046DFF8D0
:102ED000E8B0079394F904100023364A92F90800E9
:102EE000884260D001330C32092BF7D10C35079B97
:102EF0000C349D42EED109B0BDE8F08F29460C227A
:102F000020463DF0A7F900284246484613BF01215C
:102F100000214FF0010A4FF0000AFEF703FFEA79A3
:102F200095F90430804606EB820251464846D2F8B5
:102F30000C2904922A7A06EB8202D2F80C29039219
:102F4000AA7906EB8202D2F80C2902926A7906EB82
:102F50008202D2F80C2901922A6800925A46FDF7A3
:102F60002DFDE279514694F90430484606EB820281
:102F7000D2F80C290492227A06EB8202D2F80C29AC
:102F80000392A27906EB8202D2F80C2902926279AE
:102F900006EB8202D2F80C290192226800925A466E
:102FA000FDF7C4FCA2E7002FA8D1BA46D9E700BFBD
:102FB000741B050820370120A6C805082DE9F04735
:102FC00007468AB00846FEF7DBFF044638B1002307
:102FD000544901201A460AB0BDE8F04768E70DF1F0
:102FE0001C0807904E1CC8E901000846FCF7D8F9F8
:102FF0004C4B40B21A4693F90410814200F08A808B
:1030000001340C33092CF6D1002425463046FBF759
:10301000E9F8064638B1013500230A22EDB2194617
:10302000FCF71AF907904FF00009DFF800A13046CD
:10303000FBF7D8F8064640B3FCF7B2F93A4900224C
:1030400051F804CBD3B2604503D00132102AF7D136
:1030500000230AEB8302D2F80C29904215D1B9F172
:10306000020F1FD0B9F1030F21D05A1EB9F1010F81
:10307000D2B212D00B2A03D88DF821300135EDB22F
:1030800009F10109B9F1040FD1D1052D15D8384640
:103090000AB0BDE8F047FEF703BA042AF0D88DF86D
:1030A0002230EBE7052BEBD88DF82430E6E79A1EAB
:1030B0000D2AE5D88DF82330E0E798E807001B4B90
:1030C00084E807009DF82320002103EB82020846D4
:1030D000D2F80C2904929DF8242003EB8202D2F846
:1030E0000C2903929DF8222003EB8202D2F80C29CE
:1030F00002929DF8212003EB82030D4AD3F80C398C
:103100000193079B00939DF92030FDF70FFC0AB057
:10311000BDE8F0870C2301258DF8200003FB042473
:1031200074E700BFA036012080240508741B050841
:10313000A6C805082DE9F04F8BB00C4600210746C4
:1031400008921A46FEF7EEFD0026089D4FF0190979
:103150004FF46178DFF8A4B00990089B002B49D0A8
:1031600029460A2220463DF075F80028099A38467B
:1031700013BF012100214FF0010A4FF0000AFEF7B2
:10318000D1FD2A890990334606925146EA8838468D
:1031900005922A790492EA780392AA7819FB0282AE
:1031A00002926A7819FB028201922A7800925A46AA
:1031B000FDF704FC22893346013651460692384613
:1031C000E2880A35059222790492E2780392A27885
:1031D00019FB02820292627819FB0282019214F8B2
:1031E0000A2B00925A46FDF7A1FB1E2EB5D10BB05B
:1031F000BDE8F08FDDF820A0DCE700BFC3C80508FC
:103200002DE9F04380468BB008460F46FEF7B8FE26
:10321000044638B10023654901201A460BB0BDE8C9
:10322000F04387E70846FCF7BBF81D28054600F386
:10323000B3800A268DF827404643781CFAF7D2FF60
:10324000044630B1FCF7ACF89DF8273001338DF817
:1032500027302046564CFAF7C5FF074668B1FCF701
:103260009FF80D2809D80A2303FB054383F8E804D7
:103270009DF8273001338DF82730DFF83091711C2D
:103280000DF1270238464944FCF78EF8FAF7AAFFF9
:10329000074668B1FCF784F8222809D80A2303FB03
:1032A000054383F8EB049DF8273001338DF8273070
:1032B0003846FAF797FF074668B1FCF771F80D2812
:1032C00009D80A2303FB054383F8EC049DF8273053
:1032D00001338DF827309DF82730062B0CD00023C2
:1032E00009EB0602404649F8063053601381FEF7A9
:1032F000D7F80BB0BDE8F0830A260023384606FB5A
:103300000546A6F8EE34A6F8F034FAF76BFF074648
:1033100040B1FCF745F89DF82730A6F8EE040133DC
:103320008DF827303846FAF75DFF58B1FCF738F8CA
:103330000A2303FB0543A3F8F0049DF8273001336B
:103340008DF827301B4B4FF0FF324FF461705A60FD
:103350000A2202FB0542B2F8F0340693B2F8EE34CA
:10336000059392F8EC34049392F8EB340393192309
:1033700092F8EA1413FB0101029192F8E91413FB8D
:10338000010300210193084692F8E8340A4A0093A9
:103390002B46FDF7CBFAACE71D23224607494046F2
:1033A0000BB0BDE8F043FEF7DFBD00BF6848012069
:1033B0008043012088030120C3C80508A0C8050870
:1033C0002DE9F04F804691461F460C4616464FF0B9
:1033D000000BDFF820A12DED088B95B094ED008A4D
:1033E000B5EE408AF1EE10FA7DD0D4ED019A94ED5D
:1033F000029AD4ED038AB9F1000F49D0D6ED00BA94
:1034000096ED01BAB4EE6B8AD6ED02AA96ED03AA48
:10341000F1EE10FA6CD1F4EE4B9AF1EE10FA67D19E
:10342000B4EE6A9AF1EE10FA62D1F4EE4A8AF1EE45
:1034300010FA0CBF012100213A460D46404681F0AA
:103440000101FEF76FFCB0EE6B0A074611A8FAF710
:10345000D5FEB0EE4B0A07900EA8FAF7CFFEB0EEFD
:103460006A0A06900BA8FAF7C9FEB0EE4A0A059060
:1034700008A8FAF7C3FE0599069A079B03904046F1
:10348000029129460192524600935B46FDF796FA57
:10349000B0EE480A11A8FAF7B1FEB0EE690A054687
:1034A0000EA8FAF7ABFEB0EE490A06900BA8FAF7A1
:1034B000A5FEB0EE680A059008A8FAF79FFE069BE5
:1034C000059A00210390404602925246103410366D
:1034D000CDE900535B460BF1010BFDF727FABBF179
:1034E000080F7FF47BAF15B0BDEC088BBDE8F08F03
:1034F0000021A1E7E6C805082DE9F74F07460D466C
:10350000DFF894A1DFF894B12846FEF739FD0646AE
:1035100038B10023594901201A4603B0BDE8F04FE5
:103520004EE7052251462846FBF746FE60B9534B4D
:1035300000221A601A611A621A631A641A651A66FE
:103540001A6703B0BDE8F08F04224D492846FBF707
:1035500033FE04462846002C44D1FAF743FE804649
:103560000028EED03AF016FD464BC2B253F8049B49
:10357000B9F1000F07D12A464349384603B0BDE8E8
:10358000F04FFDF776BF494640460134CDE90023B0
:10359000FBF712FE0646DDE900230028E6D1374A94
:1035A000034600211546013342F8101B082BFAD1BF
:1035B0000BEBC404D4F8BCC0BCF1000F03D094F8EA
:1035C000B8E0764505DB49463048314DFDF790FAC5
:1035D0009AE70CEB061305EB061401360FCB84E8D3
:1035E0000F00EEE7FBF7DCFE072804463DD828462F
:1035F000FAF7F8FD064658B3FAF7B2FB1F4B012560
:1036000003EB041383ED000A3046FAF7EBFD0646A0
:1036100038B1FAF7A5FB194B013503EB041383ED21
:10362000010A3046FAF7DEFD064638B1FAF798FB94
:10363000124B013503EB041383ED020A3046FAF70F
:10364000D1FD38B9384603B0BDE8F04FFDF728BFCB
:103650000546D9E7FAF784FB0848032D00EB04146C
:1036600084ED030A3FF455AFECE7072332460949DE
:10367000384603B0BDE8F04FFEF776BC1C3B012096
:10368000FAC80508E022050839C30508FFC805087F
:1036900051D30508A0C80508B7C50508741B05085F
:1036A0002DE9F74F92460C461A46002181465646B0
:1036B000FEF738FB00258046DFF864B0BAF1000F52
:1036C0002CD03146042220463CF0C4FD002842465E
:1036D000484613BF0121002101270027FEF722FBE6
:1036E000738880465A46019339463AF82530484651
:1036F00000932B46FDF762F963885A4639464846DF
:103700000193043634F8043B00932B460135FDF752
:103710000DF9042DD2D103B0BDE8F08F5746EBE789
:1037200009C905082DE9F34105460846FEF728FCBE
:103730000C46074638B10023334901201A4602B02F
:10374000BDE8F041ACE731492046FBF711FD0346E7
:1037500068B92D4A4FF47A704FF4FA610133108042
:1037600051800432042BF9D102B0BDE8F08120462B
:10377000FBF716FE0328064641D82046FAF732FD2D
:10378000074670B1FBF70CFE4FF0010804463846BF
:10379000FAF728FD48B9284602B0BDE8F041FDF728
:1037A0007FBE40F2EE248046F1E7FBF7F9FDB8F169
:1037B000000FF0D0A4F2EE2240F2DC539A4203D87C
:1037C000A0F2EE229A420AD940F6CA0340F2EE2253
:1037D0000F49284602B0BDE8F041FEF7C5BB0D4BCE
:1037E00000210D4A03EB8603A3F81446A3F816063E
:1037F0003346CDE900400846FDF798F8B4E70323C7
:103800003A460649E5E700BF94490120B7C50508D7
:103810001AC905088043012009C9050897C505088C
:103820002DE9F04F8FB08946174600211A4606460B
:103830000024FEF777FA0DF1240B0546DFF86CA0A3
:1038400059F82430594602A8029333F0AFFC57B31D
:1038500057F824303046029A039393422A4613BF06
:10386000012100214FF001084FF00008FEF75AFA3D
:1038700004A9054603A833F099FC04A9234652463F
:10388000009130464146FDF799F8234601345246EF
:1038900041463046CDF800B0FDF748F8202CCFD196
:1038A0000FB0BDE8F08FB846EFE700BF28C90508A4
:1038B000F0B5074689B008460E46FEF761FB05469F
:1038C00038B10023194901201A4609B0BDE8F0407B
:1038D000A6E70846FBF764FD1F2804461DD83046BE
:1038E000FAF780FC014620462AF052F978B103AE7F
:1038F0000E48314600EB840033F058FC23460C4A56
:10390000294628460096FDF711F809B0F0BD384663
:1039100009B0BDE8F040FEF7C3BA1F232A460549A7
:10392000384609B0BDE8F040FEF71EBBA4490120AF
:1039300028C90508A0C805082DE9F04F924685B0B2
:103940000C461A46002181465546FEF7EBF9002643
:103950008046DFF86CB0BAF1000F2FD02946042260
:1039600020463CF077FC00284246484613BF012120
:10397000002101270027FEF7D5F9EB7880465A464B
:1039800002933946AB78484601932B88009333461F
:10399000FDF714F8E3785A46394648460293043551
:1039A000A378019334F8043B009333460136FCF7C7
:1039B000BDFF102ECFD105B0BDE8F08F5746E9E727
:1039C00032C90508F0B5074685B008460E46FEF731
:1039D000D7FA054638B100231C4901201A4605B024
:1039E000BDE8F040A8E70846FBF7DAFC0F280446DC
:1039F00023DC3046FAF7F6FB0146204629F060FD4D
:103A0000A8B104F12002124B2946284603EB820399
:103A100093F82726029293F826260192B3F82436CB
:103A20000C4A00932346FCF781FF05B0F0BD3846F1
:103A300005B0BDE8F040FEF733BA0F232A46064929
:103A4000384605B0BDE8F040FEF78EBA244A0120A2
:103A50008043012032C90508A0C805082DE9F04FB0
:103A600087B014461A46054603910021FEF75AF91D
:103A70004FF000080646DFF820B106234FF000099A
:103A800003FB08F7C037039BDB5D0493002C7FD05A
:103A9000E35D2846049A05939A42324613BF0121FA
:103AA00000214FF0010A4FF0000AFEF73BF9059B99
:103AB00006465A4651462846CDE900934346FCF750
:103AC0007DFF049B5A46514628460137CDE90093B5
:103AD00009F101094346FCF729FFB9F1060FD2D1DC
:103AE00008F10108B8F1060FC7D1E427DFF8A8B044
:103AF000039BA7F1E40913F807A0002C4AD0E35D6B
:103B0000324628469A45049313BF012100214FF005
:103B100001084FF00008FEF705F9049B06465A46D7
:103B200041462846CDE900930623FCF747FF0137BD
:103B30000623194A41462846CDE9009AFCF7F6FECD
:103B4000EF2FD5D1039B93F8EF70ACB194F8EF80D1
:103B500032462846474513BF012100210124002495
:103B6000FEF7E0F800230C4A21460093284607237D
:103B7000CDF80480FCF722FF0023074A214628469F
:103B8000009307230197FCF7D1FE07B0BDE8F08F43
:103B9000A24696E7A046CAE744C90508F0B505461F
:103BA00087B008460B46FEF7EBF9044638B1002310
:103BB0001C4901201A4607B0BDE8F0404EE703AEAD
:103BC000194F02AA184918463CF030FBB8B1032C33
:103BD00004D12846FDF764FC07B0F0BDFBF7E0FB1D
:103BE00002AA46F8040B3946002001343CF01EFBC3
:103BF000ECE7324621460D48FCF77AFFECE7032C50
:103C0000E7D1059BDDE903461A4601933146E0B250
:103C100029F0A0FC019B0028EBD12846FEF740F9D3
:103C2000DAE700BFA449012062BC050844C90508C1
:103C30002DE9F04F89B000260C46002107921A4664
:103C40000746B246FEF76EF84FF01909079D4FF48C
:103C50006178DFF894B00690079B3BB329460622B3
:103C600020463CF0F7FA0028069A384613BF012197
:103C700000214FF0010A4FF0000AFEF753F86A796D
:103C80000690334619FB02825146384605922A793E
:103C900019FB02820492EA780392AA7802926A7867
:103CA00001922A7800925A46FCF788FE62793346E0
:103CB0000136514619FB02823846063505922279B3
:103CC00019FB02820492E2780392A278029262784F
:103CD000019214F8062B00925A46FCF727FE0A2E92
:103CE000BAD109B0BDE8F08F58C905082DE9F04FE9
:103CF00080468BB008468946FEF742F9074638B140
:103D00000023554901201A460BB0BDE8F04F8FE75C
:103D1000524C084694F86A3794F880B694F881A615
:103D20000793FBF73DFB0928054600F38B80062629
:103D30008DF82770464309F10100FAF753FA074658
:103D400058B1FBF72DFB0D2807D8A31983F8A40958
:103D50009DF8273001338DF827303846FAF742FABC
:103D6000074668B1FBF71CFB834509D3062303FB19
:103D7000054383F8A5099DF8273001338DF82730D6
:103D80003846FAF72FFA074668B1FBF709FB5045AA
:103D900009D8062303FB054383F8A6099DF82730BD
:103DA00001338DF827303846FAF71CFA074670B110
:103DB000FBF7F6FA079B834209D3062303FB05436F
:103DC00083F8A7099DF8273001338DF82730DFF8F5
:103DD0008890311D0DF1270238464944FBF7E4FA7B
:103DE0009DF82730062B0BD0002309EB0602404636
:103DF00049F806309380FDF753FB0BB0BDE8F08F18
:103E000003FB05444FF46171192394F8A92913FBAE
:103E10000212059294F8A82913FB02130021104AFC
:103E20000493084694F8A739039394F8A6390293AB
:103E300094F8A539019394F8A43900932B46FCF724
:103E400075FDDAE709233A46064940460BB0BDE85E
:103E5000F04FFEF789B800BF2C3C012088320120CA
:103E600058C90508A0C805082DE9F04F144689B0C7
:103E70000F461A4600210646FDF754FF0546002C62
:103E800000F0D58022783B789A42024630460DBF3A
:103E90004FF001084FF0000801210021FDF742FF1B
:103EA00023780546994A41463046FCF787FD3B7822
:103EB0004146964A3046FCF739FD002C00F0B980A7
:103EC000627830467B789A422A460DBF4FF001084F
:103ED0004FF0000801210021FDF724FF637805461B
:103EE0008B4A41463046FCF769FD7B784146884A5B
:103EF0003046FCF71BFD07F1CA0304F1CA0B4FF073
:103F0000020904934FF0000A822305933B7853453E
:103F100000F39180002C00F0F28097F8EA303046F0
:103F200094F8EA209A422A460DBF4FF001084FF05C
:103F3000000801210021FDF7F5FE94F8EA3005465E
:103F4000744A41463046FCF739FD97F8EA3041465D
:103F5000704A304607F1EC09FCF7E8FC002C00F051
:103F6000D08004F1EC034A4604F1FC014FF0010853
:103F70009A4633F802CB32F8020B844518BF4FF053
:103F800000088B42F5D188F001012A463046C9B2BB
:103F9000FDF7C8FE082105465046FBF735F85E4A96
:103FA000034641463046FCF709FD97F8EA104846BB
:103FB000FBF72AF8584A034641463046FCF7B6FC60
:103FC000002C00F0A0804FF0FC094FF0010807EB37
:103FD000090104EB0900FBF7CBF809F104090028FB
:103FE00018BF4FF00008B9F58E7FF0D188F00101BD
:103FF0002A463046C9B2FDF795FE082104F1FC00BF
:10400000FAF7AAF9454A034641463046FCF7D6FC82
:1040100097F8EA1007F1FC00FAF79EF93F4A0346C9
:104020004146304609B0BDE8F04FFCF77FBCA046E2
:104030003DE7A04659E7059B3B440693002C5CD026
:10404000059B0698234419460793FBF791F8049BB8
:104050001A789BF800309A424CD1B0FA80F84FEAB7
:1040600058184B4609F11002F85AE15A02338842B7
:1040700018BF4FF000089342F6D188F001012A469C
:104080003046C9B2FDF74EFE627804EB09010546E1
:104090009BF81800FAF78AFF02909BF8003041461F
:1040A0001F4A30460193079B00930AF10103FCF776
:1040B00085FC049B07EB09017A780AF1010A187E56
:1040C0000BF1010B0793FAF771FF079B4146049A26
:1040D00009F11009029030461B7801320193069BCA
:1040E0000492009353460E4AFCF720FC059B0933CB
:1040F00005930BE74FF00008B3E7A046D9E7A046C9
:1041000023E7A04651E7A04682E700BF71C9050832
:1041100083C90508B1C90508C9C90508E0C905086A
:1041200098C905082DE9F04F8FB004460846B049FC
:1041300002AA3CF07BF8064640B903460246AD4968
:104140004120FFF791FE0FB0BDE8F08FAA49FBF7C1
:104150000FF8074620BB02AAA5493CF067F8FBF719
:104160001FF90828054606D908233A46A3492046E0
:10417000FDF7FAFEE7E7A24C94F88036834202DCB2
:1041800084F88056DFE7064604F5D06731463846A6
:1041900024F0A4FA013694F88036B342F6DCEFE757
:1041A00098493046FAF7E4FF0546E0B902AA90497B
:1041B0003CF03CF8FBF7F4F80828064603D908233E
:1041C0002A469149D3E78E4C94F88136834202DC2B
:1041D00084F88166B7E728460135314632F0BEFFE4
:1041E000082DF8D1F4E789493046FAF7C1FF0746B0
:1041F00000BB02AA7E493CF019F80028A3D0FBF7C7
:10420000CFF80828054603D908233A468049AEE787
:104210007B4C94F86A37834209DD014604F5D0608F
:1042200024F0A6FA294604F5D06024F0AFFA84F809
:104230006A5788E777493046FAF79AFF054618BB70
:1042400006AE6F4BDFF8A8910146B046102230460B
:1042500093F86A773CF028F8BD4202AA80F20E81FA
:10426000494600203BF0E2FF10B93A466A490EE1A8
:10427000FBF796F8013528F8020BEDE7674C96E856
:104280000F0084E80F005EE765493046FAF770FFDB
:10429000054600283BD15A4B0DF11808074693F804
:1042A0006A9746464F4502AA51494FF0000080F2F6
:1042B000F2803BF0BBFF014610B94A465949E6E09F
:1042C000B2464FF0000B032230463CF01DF9304659
:1042D00039F060FE584502D801370436E2E79AF813
:1042E00000000BF1010BFAF73DFF0AF8010BEEE7B6
:1042F0004A464D49CBE0414620460135043408F199
:104300000408032224F0D4F9AF42F4D11BE7474953
:104310003046FAF72DFF0546002840F0AC80384FB4
:1043200002AA334997F880863BF080FF00283FF4CB
:104330000AAFFBF735F8461E01D4B04503DC43460F
:1043400001223B4913E72A4902AA00203BF06EFFF5
:10435000014600283FF4F7AE4FF000080DF10C09BC
:10436000082203A88DF81480CDE903883CF0CCF82E
:1043700003A839F00FFE40451CD802AA1C490020B2
:104380003BF054FF00283FF4DEAE90F800A04FF061
:10439000000897F88196DFF8A8B04D4502AA1449A5
:1043A0004FF000007EDA3BF041FF024658B94A4622
:1043B00020496CE099F8000008F10108FAF7D2FEF4
:1043C00009F8010BD4E7002D40D11378303B092BBD
:1043D0003CD919490192FAF7CBFE019A90B31046E5
:1043E0005946FAF7C5FE019A002838D013494EE025
:1043F00062BC050808390120F7C90508FDC9050890
:104400008832012008CA050811CA05081FCA050814
:104410002BCA05083DCA05082CCB0508F439012034
:1044200067CA05084CCB050873CA050891CA050878
:1044300096CA05086CCB050830BC0508A9CA050852
:10444000A2CA05084FF001084FF0FF35104601924F
:10445000FAF7A6FF0028019A03DA214917E0A846D7
:10446000F2E70EAB03EB4503013523F8200C94E78C
:104470004A461C490BE032461B4908E01B49002014
:104480003BF0D4FE00283FF4F9AE3A4618492046E6
:10449000FCF7EFFF57E63BF0C9FE00287FF428AF9A
:1044A000144C31E73BF0C2FE0028E1D106EBC60018
:1044B000114C082203A982303744204424F0F8F834
:1044C0005046FAF74FFE87F84A0704EB061006A994
:1044D0006A0002303BF074FE87F8628733E600BF63
:1044E000DECA0508F3CA050816CB050862BC050834
:1044F00049CA0508043A01200839012070B50A4C60
:1045000000250A4E94F8853013B12046FCF792F846
:1045100020460135FCF76AF93046FCF799F9042D7D
:1045200004F19604EED170BDF83301207819012012
:1045300038B50C46054616492046FAF719FE30B93B
:10454000FFF7DCFF1348BDE83840FCF703BA124917
:104550002046FAF70DFEA8B9104A82F8F50182F854
:10456000FD0182F88B0282F8930282F8210382F81F
:10457000290382F8B70382F8BF03094A82F82100B1
:104580000848E0E72846BDE83840FDF789BC00BF91
:1045900091CB050897CB0508B2CB050888320120DE
:1045A00078190120BACB05082DE9F04F0F46914646
:1045B00089B0002187EA09099846139A0646002522
:1045C000FDF7B0FB6FEA09030446DFF8809006931D
:1045D00028460AF0F1FA129B184230D0069BDFF809
:1045E00070B0034014BF4FF0010A4FF0000A04936B
:1045F00010EA0703284614BF4A465A460593079215
:104600000AF0ECFA4346079A514603900090304670
:10461000FCF7D4F9049B22463046B3FA83F14909EA
:10462000FDF780FB039B059A0446009351464346E1
:10463000002A14BF5A464A463046FCF777F901353E
:10464000182DC5D109B0BDE8F08F00BFF4C805082A
:10465000D6CB050837B504460846019139F09AFCD7
:104660000199054602462046FAF7A6FD70B9625D3B
:104670001046FAF761FD00B932B901352C442046E5
:1046800001340378202BFAD003B030BD0020FBE7C3
:104690000329F0B5054685B00C46164614D80B4FD5
:1046A0003970FCF73FF90A492846FEF74FF82246D1
:1046B000084901A8FAF720FC01AB32460821284638
:1046C000FDF778FBFF233B7005B0F0BD88030120A8
:1046D00051D30508F0C705080329F0B5054685B094
:1046E0000C46164614D80B4F7970FCF71BF90A4993
:1046F0002846FEF75BF8224608496846FAF7FCFBB5
:104700006B46324610212846FDF754FBFF237B7091
:1047100005B0F0BD8803012051D30508ECC705089A
:10472000F8B5114B93F88500D0B993F88C2012B1ED
:1047300093F88D20A2B90D4E96F894748FB1187E1F
:1047400070B90B4D06F214740FCD0FC495E80F002D
:1047500084E80F00012386F84F3707F035F9384613
:10476000F8BD0120FCE700BF883201208043012012
:10477000A432012038B50546FFF7D2FF044660B9E0
:1047800007492846FCF775FE06492846FCF771FEE6
:10479000054B83F88C4083F88D40204638BD00BF20
:1047A000BEC40508DDCB05088832012008B5FFF737
:1047B000E1FF50B1054B02229A75FBF7E1FE044878
:1047C000FCF7CEF80020FCF795F808BD88320120F0
:1047D000FBCB050810B5094C94F850375BB9084B72
:1047E0000C22084918683BF07BFE012308B984F8C5
:1047F000513784F8503794F8510710BD8043012099
:104800000028000802CC05082DE9F74F4FF00009F9
:104810000126054601AA084648493BF007FD4F46D8
:1048200082464C46B046DFF840B1BAF1000F28D1BD
:10483000B9F1000F2ED1424F002C7BD021464148C8
:10484000FCF756F997F884300BB902F069FAF9F7DA
:1048500025FF002087F88D000EB102F0FDF9FFF76B
:104860004DFE14B12046FDF768FAB8F1000F14D0E0
:104870002846FFF77FFF80B1FBF782FE0020FCF7A0
:1048800039F8B9F1000F0BD05046FAF789FD84B220
:10489000002C3ED12846FDF703FB03B0BDE8F08FA6
:1048A00029495046FAF7ACFC00283CD1274950462C
:1048B000FAF7A6FC002839D159465046FAF7A0FC71
:1048C000002835D122495046FAF79AFC0028E1D059
:1048D000002FDFD1FFF77EFFB0B11E4B1E4D1C68CD
:1048E0001E4E013C14F8011F4B1EDBB2FD2BD4D829
:1048F0002B689C42D1D20A2903D03046FCF776F8C7
:10490000F0E7FCF70FF8EDE715492846FCF7ACFC9B
:10491000C3E74FF0000901AA0849002001373BF026
:1049200085FC824681E74FF00109F4E7C846F2E7CB
:104930004E46F0E70B48FCF713F888E762BC050821
:10494000883201203BCC05080FCC050850D0050863
:104950001DCC05080028000804280008F7C2050837
:1049600022CC05085ECC050818CC050830B5154BDF
:1049700087B0154A054604930C46144B144903931B
:10498000144B15480293154B0193154B0093154B8F
:10499000FCF72CF8FBF7C6FFFFF71CFF58B11248D5
:1049A000FBF7DEFF64B1114A1149124807B0BDE8B8
:1049B0003040FCF79DB810492846FCF755FCF1E75C
:1049C00007B030BDA9CC050874CC0508AECC0508ED
:1049D00004CC0508B8CC05087ECC0508C1CC050878
:1049E00050BF050897320120CDCC05084C7B050847
:1049F000447B0508E9CC0508D9CC05080121B5E7B9
:104A00002DE9F04F3E4C87B00A4600210646FDF7DF
:104A100089F905903B4A2378608802EB8303D3F839
:104A20002CAAF9F7A7FD8368C1680493364B93F865
:104A30008420002A4BD0DDF81080049100272179D2
:104A40006279049B07FB012213F80290B8F1000F72
:104A50003FD018F802504D45059A304607F101073E
:104A600013BF012100214FF0010B4FF0000BFDF7A8
:104A700059F905907DB305F00F022D0953465946AB
:104A8000403502923046214ACDE90075FBF796FF8A
:104A9000B9F1000F2AD009F00F024FEA1919534655
:104AA0005946029209F140023046CDE90072174A98
:104AB000FBF73CFFA279012A38BF0122BA42BEDCD3
:104AC0000834134BA342A5D107B0BDE8F08F904640
:104AD000B4E74546BFE7B8F1000FD9D053460D4AB9
:104AE000594630460097FBF769FFD1E77306E1D4DA
:104AF0005346084A594630460097FBF717FFD9E757
:104B0000C0240508741B05088832012016CD05084D
:104B1000A02505082CCD050838B50C4B0C4603EB39
:104B2000C0050B4895F84C2903EB8203D3F82C1AE7
:104B3000FBF75CFF95F8523933B1611C0548C9B2E7
:104B4000BDE83840FBF752BF38BD00BF741B0508F5
:104B500084D105086CBD050873B50E46114905469C
:104B6000FAF706FB18B93070012002B070BD2C783E
:104B7000602C8CBF613C413C072C10D801350123CF
:104B80000A2201A92846FAF767FB019B9D4206D03D
:104B90000F2804D8013440EA04143470E4E70020FC
:104BA000E3E700BF88BB05082DE9F04F714D0A46C9
:104BB0000021824605F1800B2DED028B8BB0FDF7B5
:104BC000B1F8814600266C4B93F88440AB7AB3422F
:104BD00000F393801035AB45F4D140F21620F9F77D
:104BE000C9FCD0E902530CB12C461D460DF1100B47
:104BF00000271522002158463BF056FB2E78002E48
:104C000043D069783046039106F026FD95F90230CD
:104C100008EE100A5A1C029353425341002C00F034
:104C2000A6800022039914F802C0A018B44540F0F1
:104C30009A8090F90280029A424540F09280427830
:104C40008A4208BF0123012203F001030BF8072069
:104C50004A4683F0010150460393FDF763F8039B36
:104C600081464CB1454A18EE101A3046CDE900A2F3
:104C70004246F9F7F3FB039B414A18EE101A3046FF
:104C8000CDE900A2029AF9F7E9FB01370335152FA8
:104C9000B4D16CB304F13F06384FDFF8E4801BF861
:104CA000013B02930BBB2078F8B194F9022001324A
:104CB0001BD0617806F0D0FC05464A4601215046DB
:104CC000FDF730F894F90220029B294681462078AE
:104CD000CDE900A7F9F7C2FB2078029B4FF0FF3225
:104CE0002946CDE900A8F9F7B9FB0334B442D6D17F
:104CF0000BB0BDEC028BBDE8F08FE888F9F73AFC09
:104D0000D0E902230CB114461A46297A6B7A06FBC5
:104D1000013312F903800CB3E756B8454A465046B2
:104D20000DBF01230023012100210293FCF7FAFFAC
:104D3000029B814644B1114A31462846CDE900A282
:104D40003A46F9F73FFB029B0D4A314628460136A9
:104D5000CDE900A24246F9F735FB34E74FF0FF37C3
:104D6000DBE700236FE703323F2A7FF45CAF4FF0AD
:104D7000FF386DE7D803012088320120BD09010802
:104D80002D0901082DE9F04F80468BB008460D46ED
:104D900039F000F9024670B3A7492846FAF70CFA31
:104DA000044640BBFBF7BEFDA44DA548A54FFBF74D
:104DB000D1FDA54E1420DFF8DC8232F0E3F9E110DA
:104DC00004F0070238460131FBF710FE2B7F6A7FA3
:104DD00006EB8303D3F82C1A4AB19C48FBF788FEF4
:104DE00001342435102CEAD10BB0BDE8F08F4046D9
:104DF000FBF77EFEF4E7284605AA95493BF016FA34
:104E0000054620B901464120FFF7CEFEECE7914967
:104E1000FAF7AEF920B990494046FCF72AFBE3E7E0
:104E20008E4E0827002431682846FAF7A1F9002899
:104E300008BF3446013F06F11006F4D154B9884941
:104E40002846FAF795F928B12A4686494046FCF7E4
:104E500010FBC9E7002005AA7D498DF813003BF03F
:104E6000E5F90646002C40D080B1FAF799FA451EC4
:104E700009D4A37A9D4206DAE2684AB1012303FA13
:104E800000F0104204D132467749DFE7774EFAE767
:104E9000E088F9F76FFB764A92F884301BB192F8FC
:104EA000853083F001030027D0E902120397002B1D
:104EB00008BF0A46217A637A05FB013302EB030B34
:104EC00012F903A005AA624900203BF0AFF9814620
:104ED000A0BB0123674944B39BF900202046CDE9DC
:104EE00000312946F9F76EFA7EE768B10DF113013A
:104EF000FFF732FE28B19DF81350284602F09CFEC1
:104F000020B932465C49A1E7584EFAE72846A34645
:104F100002F090FD8246284606F08AFB0390284660
:104F2000254606F0BFFB0746CCE7CDE900315246E7
:104F300039469DF81300F9F791FA55E74549FAF714
:104F400017F9064658BBACB1EDB24C4F72B22946C8
:104F5000207902F003FB00283FF446AF0288314677
:104F60000378384601360093C2F30323120BFBF794
:104F7000BFFDEBE7414C72B27979386802F070FD01
:104F800000283FF431AF02883146037820460136CD
:104F90000093C2F30323120BFBF7AAFDEBE738499A
:104FA0004846FAF7E5F810B34846FAF7F9F9064625
:104FB00042B26CB1E9B2207902F0D0FAC8B9CDF8AA
:104FC00000906B1C22682F494046FCF752FA0BE711
:104FD0007979386802F044FD58B99DF813302A49B0
:104FE0001A09CDF8009003F00F034032ECE74FF0C0
:104FF000FF3606AF30463946FAF738F808A950466A
:10500000FAF734F8564547D076B24CB18BF80060C9
:1050100008AB00976A1C21681C48FBF769FDE3E6B2
:105020009DF81320039B110919489E7002F00F028E
:1050300008AB40310097F0E71DCC050800000120C7
:1050400040CD050856CD0508741B0508C9CE0508D6
:1050500062BC05087EC0050867CD0508D80301209D
:105060007BCD05087FCD05088ECD050851D30508F9
:10507000883201202D0901089ECD0508B0CD050814
:1050800073C30508D1CD0508F4CD05081CCE05086D
:105090003FCE050879C3050834B108AB6A1C216806
:1050A0000648FBF725FD9FE69DF8132008AB044852
:1050B000110902F00F024031F3E700BF67CE050887
:1050C00082CE05082DE9F04F07468BB040F216203E
:1050D0000391F9F74FFA039A044600213846FCF78A
:1050E00021FE404A0646D4E9025392F884400CB1AE
:1050F0002C461D461522002104A83BF0D5F805F1E9
:105100003F03039395F80090B9F1000F30D095F864
:1051100001A0002C63D0224600231178494557D1C5
:10512000283392F8018001226B4403F8182CD045F3
:105130003246384613BF012100214FF0010B4FF0DA
:10514000000BFCF7EFFD064654B1B8F1000F07D095
:10515000254B5A464146484600933B46F9F7C2F96B
:10516000224B5A465146484600933B46F9F7BAF956
:105170000335039B9D42C5D13CB3651C0DF110085E
:105180004034DFF86490DFF864A018F8013BCBB935
:1051900015F8013CB3B116B13046FBF7E1FB2978B5
:1051A0003B4615F8010C0022CDF800900026F9F7D7
:1051B00099F9002215F8010C3B461146CDF800A0E4
:1051C000F9F790F90335A542DFD10BB0BDE8F08FB8
:1051D00001330332152BA0D14FF00008A7E7A046FA
:1051E000A5E700BF88320120BD0901082D0901088B
:1051F0002DE9F04F80468DB008460D4638F0CAFEC6
:10520000024628B9014601200DB0BDE8F04F59E72C
:1052100003902846B149F9F7CFFF039A30B9B04956
:1052200040460DB0BDE8F04FFCF723B9AD49284624
:10523000F9F7C2FF044600285BD1FBF773FBAA4FC6
:10524000AA48DFF8F0B2FBF785FBDFF8EC82172005
:1052500031F098FF17F9015B002D3CD029465846E4
:10526000FBF7C4FB0023DFF8A4921A46DFF88CA2F8
:1052700091002846059389B2049206F049FA0390FA
:1052800006F0CEFA049A0178561C059BC9B11BB9E9
:105290000490FBF747FB0498039B4178DA79037885
:1052A00002F0020208EB8303C1B10091002A14BF8F
:1052B0004A465246D3F82C3A31468D48FBF718FC43
:1052C0000123042E3246D3D113B98A48FBF742FB9F
:1052D00001340E2CBED10DB0BDE8F08FD3F82C3ABE
:1052E000002A14BF4A46524631468348FBF700FC69
:1052F000E6E7002407AA814928468DF81B403AF0CA
:1053000095FF18B94046FCF7CBFDE4E70DF11B0112
:10531000FFF722FC05460028F4D09DF81B603046BC
:1053200002F08AFC20B976494046FCF7A2F8D2E7A1
:10533000234674494FF0FF3403EB4302525C96421C
:105340000BD0601C02D1002A08BF1C460133152B6C
:10535000F2D1631C15D16C49E6E71C4607AA6749E0
:1053600000203AF063FF0646002800F0A1805B4968
:10537000F9F7FEFE30BB0446644E654FDFF8BC8192
:1053800016E00025EAE7297A28680391F5F7F6FC8C
:105390000246E8796B7910F0020F03994FEA930304
:1053A00014BF30463846013300904046FBF7A0FB5F
:1053B00001349DF81B00214606F04EF905460028F1
:1053C000E1D188E7022253493046F9F7F5FE074656
:1053D000002849D1B01CF9F7E3FF9DF81B908246E5
:1053E000BB4601374846394606F036F938B94FEA28
:1053F000191209F00F0348494032009641E0037A40
:105400005345EDD1002D42D14FF0FF37BBF1FF3FA7
:105410009DF81B5008BF0025404B04EB440459463F
:105420009DF81B001C440BF1010384F85537FF2342
:1054300084F8545784F856370AAC2246F9F726FE0A
:1054400008AA39469DF81B00F9F720FE9DF81B209D
:10545000BB454FEA121122D108AB02F00F024031D6
:105460002F48FBF745FB36E72E493046F9F780FE1B
:1054700068B39DF81B302C491A0903F00F030096FE
:1054800040324046FBF7F5FF25E74FF0FF3B04EBCA
:105490004402224B134493F85577013FB6E708AB1B
:1054A00002F00F02403121480094FBF721FB12E784
:1054B0001A4B04EB440402469DF81B001C441C4B91
:1054C0000093012394F85517F9F70CF803E7002D22
:1054D000DBD14FF0FF37BB469EE700BF7EC005081B
:1054E00067CD05081DCC0508287B05089ECE05085C
:1054F000BECE0508DFCE0508D0CE050862BC050883
:10550000E5CE0508D44A0120FCCE0508C2BD050839
:1055100051D3050825CF050892CF05088043012007
:105520004ECF050873C3050828CF05086CCF0508C2
:105530002D090108B7CE0508741B050810CF050812
:10554000224BB0F5FA6F1A680346A8BF4FF4FA630E
:10555000B3F57A7FB8BF4FF47A73D20416D540F210
:10556000DC52904215D040F2DB5207EE903A904266
:10557000F8EE677A1FD8DFED166A9FED167A77EEA0
:10558000E67A9FED150AA7EE870A7047B0F57A7F95
:1055900002D89FED120A704707EE903ADFED106ACD
:1055A0009FED107AF8EE677A9FED0F0A77EEE67AB4
:1055B000A7EE870A7047DFED0D6A9FED0D7A77EE53
:1055C000E67A9FED0C0AA7EE870A70479037012014
:1055D00000007A44D62000C000E0824400000000B1
:1055E00000407A44661000400000404200A0BB44E6
:1055F000D62000400000834410B584464FEA810E57
:10560000102312F4004F4FEA420214BF0E24072465
:10561000013B92B2CCF80040F444F2D100EB81128D
:105620008C010351122042F8213010BD10B5844680
:105630004FEA810E0424130B013C4FEA021203EBE4
:10564000430392B203F11803CCF80030F444F2D1D2
:1056500000EB01130A018450062043F8214010BDDD
:10566000704700BF704700BF034B00EB400003EBE7
:10567000C000407C704700BFE0150020002303708D
:1056800043708370C3707047704700BF002070473D
:10569000704700BF0020704701207047704700BF6F
:1056A000704700BF704700BF704700BF9FED010A01
:1056B000704700BF000000000020704703681B69AE
:1056C00018470B4B002130B593F9002001315D786C
:1056D0000433092AC8BF143A082900EB02042573D1
:1056E00013F8025C855413F8012C2276ECD130BDFE
:1056F000F44E0508D0F8FC304BB1D0F88C31D0F81E
:1057000014211B685B689A4205D3D01A7047D0E910
:1057100007239A42F9D2C0681044C01A704700BFEC
:10572000D0E9091291420ED38A1AD0F80011036908
:1057300081B1D0F88811013B096849680A44934255
:105740000BD9981A7047036919448A1AD0F80011C6
:105750000029EED1013B981A70470020704700BF26
:10576000D0F8003113B190F8A4017047D0E90903D3
:10577000181AB0FA80F04009704700BFD0F8FC203A
:10578000034610B472B1D0F81421C1685C69881A5C
:10579000013A205C08BF0A465DF8044BC0B2C3F86A
:1057A00014217047006A5C69411C205CDC68C0B24F
:1057B000A14238BF0A465DF8044B1A62704700BF29
:1057C00070B5094C236873B10546002606E0996858
:1057D0001A681E7321609047236823B15A681846DF
:1057E000AA1A002AF3DA70BD806F01200B4AF8B5BF
:1057F000136855692B4003EA000555616DB1084FE8
:105800000126B5FA85F4C4F11F0457F8240006FAFE
:1058100004F403689847A543F3D1F8BD003C014068
:105820009C19012008B5294B1B68DB041ED5B5EE79
:10583000400AF1EE10FA26D0DFED257AB4EEE70A41
:10584000F1EE10FA1FD49FED237AB4EEC70AF1EE01
:1058500010FA2AD870EE677A9FED1F7A9FED1F0A23
:10586000A7EE870A3AF034F880B208BDDFED187A67
:10587000B4EEE70AF1EE10FA0BDA9FED190A3AF0EE
:1058800027F880B208BD9FED170A3AF021F880B2E0
:1058900008BD70EE677A9FED147A9FED140AA7EEAB
:1058A000870A3AF015F880B208BDDFED117ADFED16
:1058B000116A70EE677A9FED107AA7EEA67AB0EEC5
:1058C000470A3AF005F880B208BD00BF90370120C2
:1058D0000000404200E0824466BEFFBE0060BB4460
:1058E00000007A440080BB4438DFFF3E00407A4429
:1058F0000000834466BEFF3E00A0BB442DE9F04F8C
:105900000C4695B00546354920461746FEF7A2FEDF
:105910000646002850D132492046FEF79BFE064637
:1059200000284BD12F492046FEF794FE064600285A
:1059300046D12D492046FEF78DFE0646002841D16E
:1059400020462A49FEF786FE0028064612BF082494
:10595000264601240FB144F0100425493046FEF7D5
:1059600079FE88B344F0200414F480730CBF012046
:1059700000200793FCF704FA14F0090F00F01983D4
:105980001C48FAF7EDFF00212846FEF7EFFF079BC2
:10599000002B3BD11848FAF7E3FF1848FAF7DAFF73
:1059A00004F01803182B05D11548FAF7D9FF15484C
:1059B000FAF7D0FF01232AE00124CBE70224C9E74C
:1059C0000424C7E78124C5E70F493046FEF742FEAD
:1059D0000028C9D044F48074C6E700BFD1CF0508C1
:1059E000D8CF0508E0CF0508E6CF0508EFCF0508BA
:1059F00055CC0508F3CF0508FBCF050813D00508E3
:105A00001FD0050847D0050818CC050800230693C9
:105A1000FAF788FF04F01003B749B8480593FBF77D
:105A200067F8B749B748FBF763F804F48473082BA9
:105A300007D1B5492846FBF7D5F8B3492846FBF707
:105A4000B5FD14F0800309930CD1B04B204613F838
:105A5000042F002AAE4A06BF012113460021AD4A99
:105A6000FAF764FFAC492046FEF7CAFFAB4920466F
:105A7000FFF728FBAA492046FFF796F8A94BD3F871
:105A800000B0A94B1B680493059B002B40F0D2810A
:105A9000A648FAF765FF059EA54B4FF00008DFF812
:105AA0003CA399460893049B6BEA03030A9359F8B5
:105AB000047B002F40F0C081049BDFF8249363EA4D
:105AC0000B0A089B53F8042B03920893002A40F01A
:105AD000DD81984B2046984A9849FDF7E9F9099BE2
:105AE000002B40F07882DFF8FC922046DFF8F8A225
:105AF00099F800209AF80030DFF8F0829A42904A34
:105B000013BF0121002101270027FCF70BF99AF8A8
:105B1000003006463946013B8A4A204658F8233071
:105B2000FAF74CFF99F800303946874F013B854A18
:105B3000204658F82330FAF7F9FED7ED007A834A69
:105B40002046F5EE407AF1EE10FA0CBF012100215B
:105B5000FAF7ECFE33463A467D4920467D4FFDF785
:105B60002FFC7D4B6FF07F427C4E019320460092CC
:105B70003A683168FEF718FD794B40F20222204660
:105B800001930092BA68B168FEF70EFD059B002BE9
:105B900040F0AB817348FAF7E3FE059A7248082695
:105BA00072490127DFF848C210F8013B11F8018B58
:105BB00003F1500EEE440EF8208C1CF801EB0EF1B0
:105BC0005009E94409F8108C2FB1A3EB0E0EDEF159
:105BD000000747EB0E07013EE6D187F001012046A2
:105BE0008DF83860FCF79EF810AB614A39462046C4
:105BF0008DF84860FAF7E2FE0CAB5D4A3946204664
:105C0000FAF794FE5B4B5C4A20465C49FDF708FEC0
:105C10005B4B5C4A20465C49FDF78EFE5B4B564A67
:105C200020465649FDF71AFF594B5A4A20465A4911
:105C3000FCF7F2FF594B5A4A20465A49FDF77AFAC7
:105C4000594B5A4A20465A49FDF72AFD594B5A4AA0
:105C500020465A49FEF708F9594B5A4A20465A49F4
:105C6000FDF7E6FF059B002B40F041815748FAF70E
:105C700077FE574F4FF0000BDFF878814146022244
:105C800038463AF0E7FA002897F800A0204614BFFB
:105C900001210021039A0CBF4FF001094FF00009C8
:105CA000FCF740F8BAF1020F039040F0238198F816
:105CB00001204FF0190A40F2EE23494620461AFB14
:105CC0000232444B019298F800209A5C5B460092A5
:105CD000414AFAF773FE7A7840F2EE213D4B2046B6
:105CE0001AFB0212494601923A789A5C5B4600928E
:105CF000394AFAF71BFE7FE057D005088BC205082A
:105D000065D00508A9C2050851D30508806F012098
:105D100023E705086AD0050877D0050881D0050873
:105D2000F9BE0508A05501208C370120BECF05081B
:105D3000642205089ED00508A03601204C510120A0
:105D4000A5D00508ABD005081C3B0120B4D0050840
:105D5000DC5301207C380120C3D0050828560120DF
:105D6000CAD00508C6CF05082453012038BB050852
:105D70005AC5050863C30508A4490120184B012032
:105D8000D6D00508244A0120984B0120D1D005081F
:105D9000DCD00508E8370120204E0120E0D00508BE
:105DA00068480120204C0120E9D0050894490120D1
:105DB0000C4C0120F1D0050808390120C051012008
:105DC000FAD005082C3C0120A4540120CACF0508B4
:105DD000504D0120A08E05087AC5050887D005081A
:105DE00093D00508BC56012060360120E02205084A
:105DF00068360120204801200BF1010B023708F121
:105E00000208BBF1120F7FF439AF764B2246002116
:105E10002846FBF7CFFF230700F18280724E22460F
:105E200028463178FEF734FC224671782846FEF782
:105E300053FCB4E06D4E2FE63B7823B301230A9A5E
:105E4000204603FA08F31A400B930CBF01210021EE
:105E500003923246FBF766FF049B0646204663EA40
:105E60000B020B9B1A423B46524614BF01210021F4
:105E7000FAF7A4FD03993B4652460039204618BF65
:105E80000121FAF753FD08F1010810E6039B1B7886
:105E90004BB34FF00108049B08FA07F813EA080F08
:105EA0000BD06BEA03034A46204613EA080F039B14
:105EB00014BF01210021FAF781FD1BEA080F12D05F
:105EC0001AEA0808324620460CBF01210021FBF7E0
:105ED00029FFB8F100010646039B4A4618BF01217D
:105EE0002046FAF723FD0137EBE5414A56E6414BE0
:105EF0000393BEE698F8002049463F4B20469A5C43
:105F00005B4600923D4AFAF759FD3A783A4B4946CA
:105F100020469A5C5B460092384AFAF707FD6BE729
:105F20000027F9B2013722462846FEF7B1FB042FBD
:105F3000F7D12D4FDFF8E8803B7888F80030079BD9
:105F400033B92F48FAF70CFD2E492846FCF7FEFB23
:105F5000FF2388F80030F1B2013622462846FEF7CA
:105F6000BBFB042EF7D17B78274C2370079BA3B98A
:105F70002648FAF7F5FC23492846FCF717FC244885
:105F8000FAF7EEFC2348FAF7ADFCFF23237000205C
:105F900015B0BDE8F04FFBF7D0BEFF232370069B82
:105FA000002BF4D01C48FAF7DBFC1C48FAF7D2FCB3
:105FB000EDE7A10706D50C4B224628461978FEF7D7
:105FC00067FBE4E76207E2D5074B2246284659788B
:105FD000FEF782FBDBE7034B224618212846FBF73E
:105FE000E9FEDCE7D1CF050804570120BECF050844
:105FF000C6CF0508CACF0508A08E05088AC50508C2
:10600000FED0050851D305088903012021D10508D8
:1060100048D1050852D005085BD1050871D10508A3
:1060200088030120002269E4012267E42DE9F84F8A
:1060300006460C461E4D32274FF00008DFF87890D8
:10604000DFF878A02046FBF79BFFD5F800B048B9F1
:1060500021465846F9F7D4F820B921466868F9F77F
:10606000CFF880B15846FAF73DFC696811B1504647
:10607000FAF7BCFCA96811B14846FAF7B7FC4FF033
:106080000108FAF74FFC013F05F11005DAD120466F
:10609000FBF776FF48B9B8F1000F06D1224630462B
:1060A0000449BDE8F84FFBF7E4B9BDE8F88F00BF3D
:1060B000144F050887D1050881D105087BD1050853
:1060C0002DE9F0412F4C2368002B4AD00A2801D03B
:1060D0000D2844D12C4DFAF725FC232128463AF00F
:1060E000EAF908B1401B2060236800229BB902B185
:1060F00023604FF48072002123483AF0D5F8234BF7
:106100001B78002B3CD02248BDE8F041FAF7EABBEF
:1061100001220B46EAE7591E685C2028F8D002B13C
:10612000236000223226DFF86080EA54194D2F6880
:1061300040463946FEF78EFA014640B9013E05F168
:106140001005F4D114491548FBF78EF805E0144BFF
:106150009D42F7D2EB68384698470023C8E7FF2BEB
:106160000ED8A0F120025E2A0AD80BB9202807D049
:106170005A1C2260044AD054BDE8F041FAF714BC1E
:10618000BDE8F081E4400120E43F0120E840012027
:106190005FBC0508144F05089BD10508B7D1050859
:1061A0003452050870B5056804462B6A1B6943B173
:1061B0002B6AD0F894001B699847012824D0022844
:1061C0001FD02B6ADA6952B95869002839D0996909
:1061D0002962BDE87040C3E905223AF0F5B9296AA1
:1061E000143395F824200E7B2B62F6B2C2B906BB9D
:1061F0002046F4F795FA20460121BDE87040F4F7F7
:106200000FBA00232B6270BD2B6A01462046143B57
:106210002B62F4F705FA2B6ADA69002ADFD1D3E79B
:1062200000212046F4F7FCF9002385F82430002EE5
:10623000DED0A368002BDBD09A88196812048A612B
:10624000D6E7286270BD00BF38B58569002D3DD006
:106250002C68236A1B7B5BBB204637F007FC236A54
:106260005B680BB3236A5A68236A22F01F025B68DB
:10627000216A886803F01F0100F11F03194421F00F
:106280001F01BFF34F8F00290ADD02F120031144E3
:106290000F488B42C0F85C221A4603F12003F8D164
:1062A000BFF34F8FBFF36F8F2846BDE8384079E7C3
:1062B000AB68002BD0D01A6820469B88936137F0DA
:1062C000D5FB236A5B68002BCCD1EDE738BD00BF5E
:1062D00000ED00E038B5846904B938BD256828466A
:1062E00037F0C4FB2B6A1B7B1BB92046BDE8384046
:1062F00058E7A368002BF8D01A6820469B88936162
:10630000BDE838404EE700BF8160F5F7B9BA00BF7D
:106310000171F5F7B5BA00BF426A10B48469A1549F
:10632000426A04690132D0F80011A24228BF00225B
:10633000426219B15DF8044BF5F750BCD0F820214A
:106340005DF8044B136843F080031360704700BF8F
:10635000AF4B1B6893B35B692DE9F04786B0984754
:1063600048B3AC4DD5F8CC36002B01DD2FF030FC16
:10637000A94C6378022B22D0032B1CD195F8E83767
:1063800013B1A6482FF09AFC95F8D43613B1A4485F
:106390002FF094FC95F8183713B1A2482FF08EFC1B
:1063A00095F85C373BB1A04806B0BDE8F0472FF048
:1063B00085BC0323637006B0BDE8F0877047A378FF
:1063C00004F1040804F1080704F5BD56072BF2D8C0
:1063D00001A252F823F000BF716401089D65010815
:1063E0009B64010865640108F96301081B650108E5
:1063F0002F650108B363010823784FF0010A207D5F
:10640000032B0CBF4FF080094FF48079002800F077
:10641000B0800128FAD1D5F8403800215A024FF057
:10642000FF33B3FBF2F362689A18D5F8383803F1FA
:10643000020341EB01009342814139464FF00200D3
:1064400038BF1A462EF0BAFB032800F25B8101A385
:1064500053F820F0B763010847650108B7630108E6
:106460004765010895F8A037002BA4D06F489BE73B
:10647000002305A90922184603912EF047FA0128A6
:1064800099D1059B93F8FE21552A00F0D580022270
:10649000012385F8E42763708DE7654803213023E5
:1064A00005220090A1706148624933F09DFB82E7AC
:1064B0000623A3702369652B39D92278653B032A0B
:1064C0000CBF6FF07F026FF0FF0203EA02030CBF04
:1064D00080224FF4807201339A42236127D2E2680E
:1064E000D5F8381898180231884207D395F8E41780
:1064F00011B9012185F8E41701216170C5F8C4279D
:10650000C4E90120D5F8402802FB03F35B02C5F87B
:10651000A837C5F8AC370523A370A268414601200F
:106520002EF0E2FB012840F0A5800623A370002195
:1065300030462EF08FFC012840F09C80A378013378
:10654000DBB2A37042E7D4E901C32269A3EB0C01DB
:10655000914288BFC4E903C10328A9D00133B3FB2A
:10656000F9F209FB12320AB14B449B1A0020636016
:106570002075D5F83828414602322EF01FFB03283B
:1065800000F2C08001A353F820F000BFB7630108F8
:1065900005660108B7630108B164010805A9002375
:1065A0000922D5F82C082EF0B1F901287FF403AFA9
:1065B0000022059B2270B3F80B20B2F5007F1BD19F
:1065C0001A7C022A18D193F8FE21552A14D193F887
:1065D000FF21AA2A10D1B3F80EC0D5F82C68664462
:1065E000C5F830685F7B7A1EC5F840787F2A03D8EB
:1065F0007A4237EA020245D00322012385F8E427D4
:106600006370D8E6636884F814A00133A360FDE6E4
:10661000C41801201867012018570120006F0120BD
:10662000EC6D0120306E0120746E0120B86E0120E7
:10663000F50B04087CD4050893F8FF21AA2A7FF4FF
:1066400026AF03F5DF72039903F5FF73906840B13D
:106650001679A6F10B0706F0F706012F05D9062ECD
:1066600003D010329342F1D111E70123C5F82C0871
:10667000A37094E702287FF49EAE012385F8E437E7
:10668000637098E67A02013AC5F84828D88A00B9BA
:10669000586AC5F83408B3F81120520102F2FF120B
:1066A0005212C5F85028B3F8131001B9196A94446E
:1066B0000CEB400C4000A1EB0C01B1FBF7F140F6F4
:1066C000F477C5F83818B94219D94FF6F477B942BA
:1066D00011D903212170DB6A3244C5F84C3895F892
:1066E00010381044C5F83C080BB92FF0DDFBA37837
:1066F0000133A3705FE6022323700023ECE701233C
:10670000237079E7207D81E62DE9F84F9E4C804685
:1067100094F82630DA072DED028B71D59B4B94F857
:1067200027509B4E1F88012D5AD0022D37D0002DA7
:1067300041D094ED0F8AF37B33B1B38923B1954BEC
:106740001B78002B40F0CC8094F82820337A632B00
:1067500007D8022D00F0DF8094F83410002940F0B3
:10676000F18095428C4BB0EE487ADFED8C6A38BFF1
:106770001546B27B1D70D4E9133123655B1A07FB04
:1067800003F307EE903AF8EEE77AA7EEA67A84EDE7
:106790000F7A002A5FD1BDEC028BBDE8F88FA38D84
:1067A000BB42C6D27E4B012594ED0F8A1B6884F84C
:1067B00027502364BFE7E38DBB421BD3784B216C8A
:1067C0001A68F37D521A03EB830303EB8303B2EBE6
:1067D000830FAEDB012594ED0F8A84F82750AAE7DA
:1067E000238EBB4280F08480638DBB4202D20025A1
:1067F00084F827506A4B94ED0F8A1B6823649AE74C
:1068000094F82750EB1E012B604B1F882ED95B8814
:106810005F4EFB1A1433282B85D8F3889F4203D38D
:106820003288BA42BFF47FAFB7EB430F3FF77BAF7D
:106830000323DFED5C7A574A84F82730B0EE678A8D
:1068400084F828300023C4ED0F7A13706385A38584
:10685000E38523868AE0012D7DD0022D9BD1072080
:10686000BDEC028BBDE8F84F0DF028BB484EF28816
:10687000974202D33188B94202D2B7EB420F71DDA1
:106880005A88BA1A1432282A7AD80022357D84F818
:10689000272084F82820002D00F08A803D4B2946CF
:1068A0001D70154689B2B288738812FB01F213FB82
:1068B00001F3717C92B29BB28A426285A38540F259
:1068C000C180521A92B28B42E28540F2B9805B1AC3
:1068D0009BB22386642384F835300023A36322E728
:1068E00010F076FD002843D1022284F828202DE7FD
:1068F0002B4B216C1A68337E521A03EB830303EB94
:106900008303B2EB830FFFF614AF022594ED0F8AD9
:1069100084F827500FE794F8340098B90121C4F89F
:106920003880804684F83410C3F164031E4908FBA4
:1069300003F381FB0301DB17A3EBA153643384F85A
:1069400035300EE7A06B1949A8EB00088845EBDB52
:1069500084F8353005E7BDEC028B0820BDE8F84F20
:106960000DF0ACBA032D75D194ED0F8A0325E2E644
:10697000337C83422CBF0122002284F82820E5E6E4
:10698000032DF1D0D5E600BF806F0120F84701202C
:1069900094370120F7470120F6470120ACC527377F
:1069A000C8180120000000006BCA5F6B8096980039
:1069B000B6F800C02B4ADFF8BC901268B7FBFCFCAD
:1069C0000CF1010C92F96C20BCF1080F28BF4FF0BC
:1069D000080C5FFA8CF189F80010002A3FF462AFCE
:1069E00062453FF45FAF204A92F800A00AF101022D
:1069F00002F0030252453FF455AF4FF0FF300B4613
:106A000009E019B930EA200028BF1046013202F02F
:106A10000302524518D015494FF0960E93460EFBCF
:106A2000021E9EF96C108C45EBD15FFA8BF0F9F7E2
:106A300009FC0F4B99F800101F8894F8275031E794
:106A4000002346E700223EE71946431C3FF42AAFE5
:106A50008346EAE75B88FB1A1433282B7FF6DDAE0A
:106A600067E600BF5C36012090320120F833012038
:106A7000F8470120F74701202DE9F0476C4CA36847
:106A800020469847002869D0B4F90E3004F1480533
:106A9000A17D06EE903AB4F91030092907EE103ABC
:106AA000B4F91230F8EEE66A07EE903AB8EEC77A1B
:106AB0004FF00103F8EEE77AC4ED126A84F854301F
:106AC00084ED137AC4ED147A4AD05A4F284619F04F
:106AD00033FEBB8D002B4CD1574B1B685B0770D42A
:106AE000BB6AD4ED127AB3F90220D4ED135A06EE44
:106AF000102AB3F90420B3F9003007EE102AB8EEDB
:106B0000C66A00EE103AD4ED146AB8EEC77A4B4D5F
:106B1000B8EEC00A4A4E35EEC66A05F1080836EEF0
:106B2000C77A37EEC00A84ED136A84ED147A84EDD7
:106B3000120ABDEEC00A3B8810EE102A12B200EE17
:106B4000102A002B40D1B8EEC00AA84506F10C0669
:106B500005ED010A02D0B5EC010AEAE7BDE8F087CD
:106B6000344F04F12001284619F0AAFDBB8D002BFB
:106B7000B2D0D7F828C02846DFED326A0025324966
:106B8000ACF102020CF10406B3F5C87F22D0D1EDBE
:106B9000007AB8EEE77AD0ED007AE0EC016A77EEA1
:106BA000877AFDEEE77AE1EC017A22F8025F9642FD
:106BB000EAD1012B12D0013BBB851F4B1B685B0741
:106BC0008ED530F0E3F98BE73046B8EEC00A39F0E5
:106BD000F7FCBAE7B0EE667A0D60DCE71B48DFF839
:106BE00074E0C16DB4F80C80C831194E8EFB01A958
:106BF000C917D0E91520C1EBE911C832C830A1EBA3
:106C00000801ACF804108EFB0281D217C2EBE1122E
:106C1000ACF800208EFB002EC017C0EBEE10ACF8D5
:106C20000200B581F5817381F9F7E8FCBB8DC2E7FD
:106C300004300020642500209037012050300020CF
:106C40006825002000000000D46F0120806F012023
:106C5000CC3701201F85EB512DE9F84FDFF8B490B8
:106C6000064699F800501DB100242046BDE8F88F73
:106C7000FDF7B0FD04460028F6D0DFF89C80D8F878
:106C80000070C8F800500EB11C4B1D604FF48072AC
:106C90001B491C4839F094FA1B4E0023DFF87CB0E6
:106CA000D6F800A03360012389F80030174B1D6827
:106CB000013D15F8010F431EDBB2FD2B03D8DBF8B5
:106CC0000030AB4216D80D20FFF7FAF9002389F8FF
:106CD00000301FB1094BC8F800701F604FF480727C
:106CE0000849074839F06CFA094B0122C6F800A0A0
:106CF0009A73BAE7FFF7E4F9DBE700BF103301202E
:106D0000E43F0120E06F0120E4400120002800085A
:106D1000903201200D330120E03F012004280008BB
:106D200038B5074C074DAC4203D3074B01221A700C
:106D300038BDA288D4E9021039F042FA1C34F2E7D7
:106D4000E8010008E40900080C3301202DE9F04FA8
:106D5000814C83B094F80661012E07D000EB8000CF
:106D600004EB8004E08903B0BDE8F08F7B4B1B6827
:106D700093F82C70002F57D0794B4FF0000E794DBF
:106D800040F6FF7A1B78F046F1464FF6FF7B009302
:106D90002346019619E001F47062B2F5006F7BD0D2
:106DA00055D8B2F5806F70D0B2F5C06F40D1C9B27E
:106DB0004CF0080C998283F81EC00EF1010E1433BA
:106DC00002355FFA8EF2974227D993F81EC099894F
:106DD000BCF1010FDFD1514500F09580C1F30802ED
:106DE000490A02FA01F18AB2002A00F081805E4E5F
:106DF00089B2BEF1030F06EB5202B2FBF1F103D8E8
:106E0000009A2D2A00F088805945D6D0894483F80D
:106E10001EC0D98108F10108CFE7B8F1000F03D0F7
:106E2000B9FBF8F8A4F80481022384F8063195E749
:106E3000B2F5007F37D14CF0020CCAB283F81EC005
:106E400093F81FC01A829445B7D2D977B5E7B2F547
:106E5000406F13D0B2F5606F06D1C9B26CF07F0CF1
:106E6000998383F81EC0A8E7B2F5206F1BD1C9B281
:106E70004CF0200C198383F81EC09EE7C9B24CF079
:106E8000400C598383F81EC097E7C9B24CF0040C3C
:106E9000598283F81EC090E7C9B24CF0100CD98219
:106EA00083F81EC089E7514548D0C1F30802490A5A
:106EB00002FA01F18AB2DAB12B4E89B2BEF1030FA8
:106EC00006EB5202B2FBF1F10ED8009A2D2A0BD13B
:106ED000594529803FF471AF894489B24CF0010CC7
:106EE000D98183F81EC095E759453FF466AFF3E7B3
:106EF000BEF1030F3FF661AF009A2D2A7FF45DAF1C
:106F0000A5F800B059E7BEF1030F0FD94FF000020A
:106F1000DA81019A9A777DE7594529803FF44DAF90
:106F2000894489B2019AD9819A7773E7009A2D2A08
:106F3000ECD14FF0000200212A80F3E7BEF1030FED
:106F400002D8009A2D2A01D00021C7E74FF0000295
:106F500000212A80C2E700BFB811002000300020C5
:106F6000542B0120582B0120C02709006E4B1B78A1
:106F70002DE9F04F87B0002B00F0D0806B4E4FF022
:106F800000096B48B168F9F7B3FD71686948F9F712
:106F9000AFFD694B6948DFF8DCA1D3E90031C91ABC
:106FA000674B1A68B1FBF2F2F9F7A2FDF9F7BAFCE8
:106FB0006448F9F7CFFC6448F9F7CCFC634B5FFAFF
:106FC00089F41B78A34221D8614C0025614FF9F761
:106FD000A9FC2646013556F8041B3846F9F706FD8C
:106FE000162DF7D101255B4EF9F79CFC234661680D
:106FF000013530461B680434C91AF9F7F7FC162D21
:10700000F4D107B0BDE8F04FF9F78CBC2046C82595
:10701000FFF79CFE4FF014084F4B454308FB0468F4
:107020004FF03C0B93F82430671C98F81EE0B5FB3A
:10703000F3F51EF0010FA9B2ADB214BF52222D22FA
:107040001EF0020F049514BF54232D231EF0040FCD
:1070500007EE903A14BF56232D231EF0080F00931D
:1070600017EE903A14BF4FF0430C4FF02D0C1EF06A
:10707000800FCDF804C014BF4FF0530E4FF02D0E0B
:10708000B1FBFBF10591642148433946CDE902E0AB
:107090005046F9F7ABFC98F81E30DB073AD55C2375
:1070A0002E4A6343D118D05891ED010A70B1B8EE61
:1070B000400ADFED2B7A20EE270A07EE900AF8EE61
:1070C000677A80EE270A38F003FC00B2642290FB56
:1070D000F2F102FB11022348F9F788FC142122483F
:1070E00009F1010901FB076701FB0464F988628A61
:1070F0000491218B02F0030392080391E18A02912B
:10710000A18B0191A18A009119214B43218AF9F7A2
:10711000EFFC53E71548F9F7E5FBDFE7144807B044
:10712000BDE8F04FF9F716BC80010020B81100202F
:10713000BDD10508CDD10508A0150020E4D1050872
:107140002024012011D205086DD205081824002042
:10715000641200201DD30508C41B0120C0120020AA
:1071600000401C46E6D20508FBD20508F2D205080D
:1071700021D30508C9D2050870B41A4C1A4BA4FBD8
:1071800002425209A3FB0243DB0803EB8303A2EB99
:10719000430390F858205FFA83FC62451ED09A00A2
:1071A000046800EB830346689D68641B04601D6BE4
:1071B000751B456000259D601D6380F858C08318CD
:1071C000013404609A6801329A6029B94268013238
:1071D00042601A6B01321A6370BC704704689A00EF
:1071E000EDE700BF1F85EB51CDCCCCCC10B5437B78
:1071F00004468268581C6073D154627B237B93429F
:1072000000D802B910BD2368D4E9010198470023D2
:10721000637310BD427B42B1036810B50446D0E9E8
:10722000010198470023637310BD704718B183882C
:1072300002681B049361704710B1036882889A61E9
:10724000704700BF0139032931D81E4B01EB810C77
:10725000024610B403F5B07403EBCC0304EBCC048A
:107260004FF0010C046003F5B07480F888C093F807
:10727000600102281DD0C9B21348C1EB011150F8BA
:107280003110C3F8641171B10221604683F86011B6
:107290004FF48071A18102F110014C325DF8044B72
:1072A000C3E95E12704700205DF8044B7047002070
:1072B000704793F86D2160465DF8044B624483F893
:1072C0006D217047806F0120EC1B0120954B2DE94B
:1072D000F04FDFF864B285B04FF001094FF0000ABB
:1072E0001D469BF80030022B0CD00AF1010A09F16F
:1072F00001090BF1280B0535BAF1040FF1D105B0E6
:10730000BDE8F08F95F90320511C00F0E680D2B261
:1073100001924FF00C0C4FF008085FFA8AF1AE466C
:10732000012A50B225D800247F4D1CFB008723463C
:1073300034B10133182B1CD015F81C4F002CF8D198
:107340006E788E42F5D1EE59002EF2D0774D6F68EF
:1073500001342435BE4214D0102CF8D1734B13F8ED
:10736000083C33B9714B4FF0140003F8079C03F845
:10737000080C0132019BD2B29A42D1D97546002441
:1073800029E0E4B2694D671E07EBC70605EB8606E8
:10739000357F039506F11C050295039D002DE8D16C
:1073A000C3EBC303029A00EB400075469B00964670
:1073B0005D4A07F0070703EB800386F81D9020461F
:1073C00037721344CBF81060DB68F36014238EF837
:1073D0000030F2F7E9FA95F904104B1C00F09680A2
:1073E000C9B201914FF008085FFA8AF302940129AB
:1073F0004FFA81FC1FD80C224B4812FB0C8600224E
:107400000132182A17D010F81C4F012CF8D14478FB
:107410009C42F5D18459002CF2D0444F0026786864
:1074200001362437844227D0102EF8D13F4A12F873
:10743000082C002A6ED00131019AC9B29142D6D9E6
:10744000029C002C45D02423384A601E002603FBF2
:107450000020CBF81460CBF81000F3F7BBF85846C7
:10746000F3F78CF83346324620463149F2F7AEFA4C
:1074700001238BF80C3038E7F6B22C4C06F1FF3EB6
:107480000EEBCE0004EB800000F11C04077F039498
:10749000002FD0D1034660460EF0070E029C9C469A
:1074A000C2EBC20300EB40001F4A9B008CF808E0CF
:1074B0008CF81D9003EB80033046CBF814C01344C6
:1074C000039ADB68CCF80C3013231370F2F76CFAD4
:1074D0003CB90023CBE9043307E7012300220193E1
:1074E00017E7DBF81400F3F775F8DBF81000F3F793
:1074F00071F85846F3F742F83B463A4630460D4994
:10750000F2F764FA01238BF80C30EEE60123002138
:10751000019367E7054A4FF0130002F8079C02F851
:10752000080C88E7B43B0120A418050800000120DE
:10753000D562010849620108E0700120064A002373
:10754000516801332432814203D0102BF8D100203E
:107550007047D8B2704700BF00000120D3B2012BA2
:1075600023D802EB42024FF0000C70B54FEA820EB6
:107570000F4C634622460EF1080504E00133182B38
:1075800011D012F81CCF6045F8D192F801C08C459B
:10759000F4D15659002EF1D0C3EBC3030EEB830395
:1075A0000433E01870BD002070BD0020704700BF9C
:1075B000A418050830B40568EFF3118C102383F389
:1075C000128803681B6AEBB18B6804460A461BB13C
:1075D000D3691432002BFBD12B6ADBB1986838B920
:1075E000934209D0186828B15B6898680028F7D0E2
:1075F0001433F3E7C3E900415FFA8CFC8CF3118884
:1076000030BC70475FFA8CFC29628CF3118830BC67
:1076100038F0DABF1C60FFDE30B593B000230446BB
:107620008DF807100DF106018DF806200DF1070504
:1076300001228DF8183003958DF82C208DF840200C
:107640001193CDE9073103A9CDE90432CDE909321F
:10765000CDE90C33CDE90E33FFF7ACFF2268136A96
:10766000002BFCD113B030BD10B592B08C4604464F
:1076700009920DF107020A9300230392012203A944
:107680008DF807C005928DF82C208DF840200493CA
:107690008DF818301193CDE90733CDE90C33CDE9DE
:1076A0000E33FFF787FF2268136A002BFCD112B05C
:1076B00010BD00BF2DE9F04F046885B02678012E7B
:1076C0000AD0022E03D1246A002C00F0B4800024DA
:1076D000204605B0BDE8F08F94F90480B8F1030F9F
:1076E000D4BF00240124B8F1FF3F08BF44F00104D7
:1076F000002CECD19A46DFF8309208EB480396460E
:107700004FEA480C09EB43135A69002AE0D00546BA
:1077100093F85500202840F0A38093F854000128E6
:1077200000F09E80287983F85460784E356804E034
:1077300033685B1B192B00F2B380936913F4004389
:10774000F6D11F46C44443000A4622204021039339
:107750001FFA8AF34FEA4C1A00950AF1140BCA4437
:10776000CB448AF85500CAF838E08AF856105846D3
:10777000CAF858700399AAF83E300A23CAF848702C
:1077800030F062FF4FEA480C002840F0BB80BAF8A6
:107790003E309BB2FF2B40F2A280DAF81410FF2398
:1077A0005B48AAF83C304B685A4A034003980343AD
:1077B0001A434A600CEB080A574A4FF0FF0E07EED7
:1077C00090BA09EB4A17786903E03168491B0A2926
:1077D00037D8836913F00403F7D0406ABB6B187085
:1077E000FB8F013B9BB2FB87BB8F013B98B2BB6B0E
:1077F0000133B887BB63FB8F9BB208B9002B35D12F
:10780000FB8F9BB2002BDED1294617EE900A30F099
:1078100059FF28BB7B692021404C09EB4A19D961EB
:107820005A68224001245A6087F8551089F854009C
:1078300087F856004CE741F080010124FFF714FF60
:1078400046E7C444202109EB4C19D9F8582089F89F
:1078500054300A43C9F8582089F8551089F8563031
:107860002F4A138801339BB2138031E7786903E014
:107870003168491B0A29E4D8836913F08003F7D0E3
:10788000FB8F9BB2FF2B1CD9436803991340A7F8C9
:107890003CE00B4343F0FF7343F480334360AFE7B6
:1078A000C4442021002209EB4C19D9F8583089F83A
:1078B00054200B43C9F8583089F8551089F85620E0
:1078C000CEE7FB8F03999BB2BB87DBB241EA034350
:1078D000416811400B4343F00073436090E7BAF8EE
:1078E0003E30039A9BB2DAF814100948AAF83C30EB
:1078F000DBB242EA03434A6802401343094A1A438F
:107900004A6057E78AF85470AAE700BF6C1B012051
:10791000009800FC0024FF81009C00FC00E800FEB1
:10792000701B012000240082EC19012030B50023D7
:1079300093B0012204468DF818300DF1070511931C
:107940008DF8071003A90A928DF82C208DF840209D
:107950000395CDE90432CDE90733CDE90C33CDE908
:107960000E330DF10B030993FFF724FE2268136A0F
:10797000002BFCD19DF80B0013B030BD036810B58F
:107980009B68044698470122FF236273A37310BDCE
:10799000036810B504461B689847012123682046F8
:1079A0009B689847E37B0133E37310BDF0B583B068
:1079B00004460D461646089F0193384636F0EAFA0B
:1079C000216828443246E672A07220468E69294614
:1079D000019BB44603B0BDE8F040604703689B6A72
:1079E000184700BF03685B6D03B11847704700BFBD
:1079F0000368DB6C03B11847704700BF002310B564
:107A0000C373044642748A6C016003730AB1194659
:107A100090472368012120469B689847FF212368EF
:107A20000122A173DB6C62731BB12046BDE81040DC
:107A3000184710BD0023094901E0152B0AD003EBBC
:107A40004302013311F802C00A448445F5D192F98A
:107A5000020070474FF0FF30704700BFD44A01204A
:107A6000D3B2022B21D802EB4202002330B54FEAF9
:107A7000820C0F4D0F4C2A460CF10C0E04E0013322
:107A8000172B10D052F82C4FA042F8D114798C4209
:107A9000F5D152F80E40002CF1D02C2202FB03C38A
:107AA0000833E81830BD002030BD0020704700BF0B
:107AB0007008050800000140002836D000231B494B
:107AC00030B5047901E0152B2DD003EB43020133CF
:107AD00011F802C00A44A445F5D192F902300468B5
:107AE000DAB290F805E0022A1DD803EB43031048F0
:107AF00010494FEA830C024600230CF10C0504E008
:107B00000133172B0FD052F82C1F8C42F8D111796A
:107B10007145F5D151590029F2D02C2202FB03C343
:107B20000833184430BD002030BD7047D44A0120CE
:107B300070080508000001401B4B1C4A03F5727CCD
:107B4000016803E063452BD053F82C2F9142F9D103
:107B500070B593F804E0427996450AD0634505D0A4
:107B600053F82C2F9142F4D06345F9D14FF0FF30F8
:107B700070BD9E46C4680022DEF80C50A54208D0B5
:107B800001320EF10C0E032AE8D0DEF80C50A542AB
:107B9000F6D1DEF810500669B542F1D150B270BD91
:107BA0004FF0FF30704700BF70080508000001402B
:107BB0000120FDF71BBE00BF0220FDF717BE00BF6E
:107BC0000420FDF713BE00BF0820FDF70FBE00BF65
:107BD0001020FDF70BBE00BF4FF47870FDF706BE16
:107BE0004FF47C40FDF702BE70B54FF6FF7C0E4DA2
:107BF0000E4C4FF0010E0E490E4E00234CFA03F2CC
:107C00000EFA03F0013312F0010F03D00C600831BB
:107C100021F8040C102BF1D104F58064B44202D099
:107C200035F802CFE9E770BD501B0508000002409F
:107C3000CC2501200018024010B50409013C052C98
:107C400016D80D4A00F00F0332F8141041FA03F26F
:107C500012F001020ED0012098400138084036F0A1
:107C60005FFE064B064A1B5D184402EBC00010BDC8
:107C7000002010BD104610BD501B0508481B05080C
:107C8000CC250120F0B5104B164602680C460F4F6C
:107C90000546134487B09B0AF85C30F07FFDAA8844
:107CA00004F00303286800926946C4F3810201933B
:107CB000C4F30013C4F3411405960494CDE90223E0
:107CC00033F0EEFF07B0F0BD0000FEBF840D0508E5
:107CD00000B1D7E7704700BFF8B50B4F97F82C30CD
:107CE00083B10A4C0025A66801353079FFF7A4FF5F
:107CF00018B1217D327AFFF7C5FF97F82C30A034F8
:107D0000AB42F0DC0120F8BD301E002090020020C4
:107D100008B10022B6E7704738B50C460546007832
:107D2000FFF78AFF611C0446C9B210B14123C1713B
:107D3000837120466978FFF7EBFFAB7820461BB1D3
:107D4000BDE83840FFF778BABDE83840FFF76EBAB3
:107D5000054B53F8203033B11A689B8851690B42A8
:107D600018BF1B0493617047741B01200E4B012246
:107D700010B40E4C93F800C002FA00F354F820003F
:107D800003EA0C0351B1003B18BF012318B101688D
:107D900082883BB18A615DF8044B7047B3FA83F384
:107DA0005B09F3E71204F5E7721B0120741B012045
:107DB00070B5392086B0FFF73FFF054610B140F29D
:107DC0003E23C380124C4FF4007102220026236B25
:107DD000104843F004032363236B059603F0040368
:107DE00000930323CDE9011201A9009ACDE90363B1
:107DF0002BF0B6FDA36832460E2123F078432846C7
:107E000043F0E043A36006B0BDE8704060E700BF08
:107E1000003802400008024010B5054C23681B6979
:107E200098472368002283F82E201A6310BD00BFF4
:107E30000030002010B5084C236893F82D2012B1B3
:107E4000DB68984700B910BD044A01212368126815
:107E500083F82E101A6310BD00300020C8180120CE
:107E60002DE9F047264F86B0264E01254FF0520AE5
:107E7000DFF89490DFF8948017F8010BFFF7DCFE31
:107E80000446B8B10368C571434480F806A09B0A54
:107E900019F8030030F082FCB4F804C0002301227A
:107EA00020686946CDE900C3CDE90233CDE904235A
:107EB00033F0F6FE16F8010BFFF7BEFE5322044620
:107EC000B0B1036882714344C5719B0A19F803007D
:107ED00030F064FCB4F804C0002302222068694634
:107EE000CDE900C3CDE90233CDE9042333F0D8FE58
:107EF0000135EDB2052DBFD106B0BDE8F08700BF5A
:107F00009453012088530120840D05080000FEBF12
:107F100003681B68184700BF03682DE9F0415F6ADA
:107F20001FB13B46BDE8F0411847002A164611DD57
:107F300004460D460E4400E023689B68204698479F
:107F40000028F9D02368204615F8011B1B689847C4
:107F5000AE42F1D1BDE8F081DEE700BF03685B68A7
:107F6000184700BF03689B68184700BF0368DB68B9
:107F7000184700BF03685B69184700BF03689B6A26
:107F800003B11847704700BF0368DB6A03B11847A5
:107F9000704700BF014B1868F3F79CBE681E0020B5
:107FA000014B5868F3F796BE681E0020014B986895
:107FB000F3F790BE681E0020014BD868F3F78ABE25
:107FC000681E0020014B1869F3F784BE681E00206C
:107FD000014B5869F3F77EBE681E0020154B1B88C5
:107FE00053B9154A154B12781B6882B173B11A68E0
:107FF0009B8878B193617047114BD3F814222AB152
:1080000058B9D3F80022106083F81102704780F04D
:108010000100EBE71B0493617047B3F818C201211C
:10802000084AD3F80002B2FBFCF20A41026083F86E
:1080300011127047AA3B0120B03B0120AC3B01204C
:10804000806F012040420F0030B4EFF31183102203
:1080500082F312880B4C4FF0E0210B480025226878
:10806000DBB2013222608A69C0F81C22C0F82052BB
:108070000A6983F31188054A1368013330BC136021
:10808000704700BFC8180120806F01206C1B0120C1
:1080900010B4EFF31181102383F312884FF0E02224
:1080A0009469136913F4803F0D4B03D00120C3F88A
:1080B000200294690B4AC9B21068D3F8202281F3D8
:1080C0001188094B02444FF47A70196800FB01F3E0
:1080D0001B1B5DF8044BB3FBF1F300FB0230704750
:1080E000806F0120C818012020240120124B5B68FA
:1080F000C3F30803FBB9EFF31183E3B90F4A4FF061
:10810000E02C10B40E4C1368DCF8180011688B4298
:10811000F9D1D4F81C128842F5D80A4A4FF47A7182
:10812000146801FB04F2121AB2FBF4F25DF8044B7E
:1081300001FB03207047ABE700ED00E0C818012009
:10814000806F0120202401202DE9F04FDFF82CA3BF
:108150009AF824322DED028B022B93B0CDE9033037
:1081600036D10FF049FD9AF82630DD0740F1FC8248
:10817000B34BB44A1B78126803F0010322B11168B3
:10818000928803B912048A6100231C468AF82432BB
:10819000AD4B0193019B1B78002B00F03581AB4B5D
:1081A0001B78472B08D10399A94A0AEB8103D3F81E
:1081B00074349B1122F811300AEB8404D4F874044F
:1081C000801113B0BDEC028BBDE8F04F38F0CCB994
:1081D0000125A04AAB42157040F007819AF8293278
:1081E0009FED9D7A07EE903A9AF82630F8EEE77AFE
:1081F00013F0010F994B67EE877A0293FCEEE77A52
:1082000017EE904A40F0B284049B1C44CAF83042F6
:10821000DAF838120029C0F282839AF84032002B33
:1082200000F094838E4B0593029B1B68590700F165
:10823000B4854FF0004300260DF12C0B0F93DAF8B4
:10824000A8320D96B3420B9610960E960C9645DD0D
:108250009FED848A844F854D08E0B9F12B0F40F2E1
:108260000F810136DAF8A8329E4237DA17F8014B4F
:1082700004EB440C630015F81C9060460193012345
:1082800009F01F024FEA591E05EB4C0C03FA02F2EB
:1082900012AB4FEA4008604603EB8E034FEA8E01B3
:1082A00053F80C3C1340D8D00AEB0103D3F8383212
:1082B00012EA030900F014810DAB0DA9013653F841
:1082C0002E3023EA020341F82E305BF82E301343A0
:1082D0004BF82E30DAF8A8329E42C7DBDAF8AC321F
:1082E000002B2DDD624E0024604D4FF0010816F882
:1082F000010B12AF5A460DA900EB4003013405EB08
:10830000430318465B794FEA531C03F01F0307EB46
:108310008C0C08FA03F35CF81C7C5CF814CC3B4230
:1083200003EA0C0C14BF01230023BCF1000F18BF9B
:1083300083F0010311F01EFBDAF8AC329C42D6DB6D
:108340000DF133010DF12B030C4613F8012F11F839
:10835000010F9C4282EA00021A70F6D1454B9BE85D
:10836000030083E80300029BDAF838221B6802F45A
:1083700080109AF89C1203F48003034314BF012376
:1083800000238AF82A32002940F021843A4B1B78D6
:10839000002B00F026842C4B0193950740F1D480EC
:1083A000059B1B689C0740F1D480BAF82C32D80793
:1083B00040F1D085022035F0CDF99AF82630DB0760
:1083C00040F1E080DAF838321F0640F1D680BAF882
:1083D0002C120E0500F1DE804FF4006035F0D0F96C
:1083E000BAF82C12DAF83832D4E010F077F8002816
:1083F0003FF4CAAE144B2C468AF824520193019BD9
:108400001B78002B7FF4CBAEFFF770FE049BC3F10B
:1084100001031D1838F0ECF8039A0AEB820392006E
:10842000D3F87434B0EBA31F01D0830198118542B7
:10843000524440F37A82AD01C2F87454AFE600BFF3
:10844000721B0120741B012094250020542B012055
:10845000582B0120E8510020002474499037012056
:10846000F04001208096984A30720120E8370120C0
:108470004C720120B8710120E8400120806F01207A
:1084800008F1020805EB080115F808204C78A24213
:1084900021D29CF8011040F2833E4FF0190C40F6B7
:1084A00033080AEB8101D1ED957A1CFB02E1FDEE68
:1084B000E77A17EE902A4245A8BF4246B2F5617F9F
:1084C000B8BF4FF461728A4205DD1CFB04E39A4297
:1084D000CCBF002301235A460DA911F04BFAC0E688
:1084E00008F1020805EB080315F808E093F801808D
:1084F000C6451CD29CF801304FF0190C0AEB8303DF
:10850000D3ED957A40F28333FDEEE77A1CFB0E3E05
:1085100040F6330C17EE903A6345A8BF6346B3F5B7
:10852000617FB8BF4FF46173734500F30282C846A0
:108530005144D1F8C4321A4200F0F58043465A46FD
:108540000DA911F017FA8CE6B54BDB78002B7FF400
:1085500027AF012035F0FEF8DAF8383259077FF5F9
:1085600029AF012035F0F6F8BAF82C329A073FF51A
:1085700024AF022035F004F91FE7A94AD278002A77
:1085800040F0ED844FF4006035F0E4F8BAF82C12B6
:10859000DAF83832A34A8D07A3481278406802F00F
:1085A000020200F0AF8120B10468808802B90004A3
:1085B000A0619E4ADFED9E6AB2F8442007EE902A41
:1085C0009C4AF8EEE77A527986EEA77A07EE902A6F
:1085D000994AD2F88001F8EE677A67EE277AFDEEC5
:1085E000E77A17EE902A0A2AB8BF0A220261DC0055
:1085F00007D49AF82620500703D522F004028AF8FF
:108600002620059A126812F00A0F13D01A0740F1BB
:1086100011844F0740F16884DE0640F14082BAF8C9
:108620002C22150500F13B82540640F1D4879A05AF
:1086300000F142829A064FF4807040F12D8235F0AD
:108640009FF87E4B1B780E2B00F03E82082B00F02B
:108650003B82029B1B685B0500F13E829AF826C0B4
:108660001CF0010C40F01382754B1B688BB3DFF8D4
:10867000E8B10020DFF8E49140F6330E9BF8088063
:1086800019264A4640F283351379C7B2547916FB4E
:108690000351A34219D2137816FB04540AEB830347
:1086A000D3ED957AFDEEE77A17EE903A7345A8BFC1
:1086B0007346B3F5617FB8BF4FF461738B4204DD3D
:1086C000A34202DCB84540F02084013006320A287B
:1086D000DAD1DAF83C329F0600F12382594B93F845
:1086E0004C33002B40F0C281BCF1000F40F0C6813A
:1086F000029BDAF838221B6802F48072514903F0B9
:108700008053134391F89C2114BF012300239A4204
:1087100002D00022C1F8B4214A4A022482F89C31D6
:108720008AF8244236E5FFF7E1FC07EE900AF8EEFE
:10873000677AF4EEC87AF1EE10FA3FF592ADB8F12F
:10874000000F7FF48EAD630001223F48234415F8EB
:108750001330590903F01F0302FA03F350F82120E4
:10876000134340F821307CE510F03CFC9AF82630A9
:10877000DC073FF509ADDAED917A0DF13C09334D97
:1087800011ACFDEEE77A324817EE903AB3F5FA6F86
:10879000A8BF4FF4FA63B3F57A7FB8BF4FF47A738A
:1087A000A3F57A73C3EBC3135B00A5FB03230DF1A1
:1087B0003D029B097F3B8DF83C3025E010F8011B02
:1087C00001320AEB8103D3ED917AFDEEE77A17EEE1
:1087D000903AB3F5FA6FA8BF4FF4FA63B3F57A7F16
:1087E000B8BF4FF47A730129A3F57A73C3EBC313AF
:1087F0004FEA4303A5FB03634FEA9313A3F17F03FF
:1088000008BF5B4202F8013C9442D7D100241149D1
:1088100008230125204622468DF8444022E000BF6F
:10882000283A0120721B0120741B01200430002013
:10883000002474495C3A0120F44001206036012094
:10884000283C0120E851002044720120D34D6210E1
:108850009D520508A5520508580401202C3C012012
:1088600011F8013B0AEB8303D3ED917A05FA02F389
:108870000132FDEEE77A40EA030617EE903AB3F5CF
:10888000FA6FA8BF4FF4FA63B3F57A7FB8BF4FF41D
:108890007A73A3F57A73C3EBC3135B00B3F5FA3FA6
:1088A00001DB70B20124082ADAD10CB18DF8440042
:1088B000A44B93F87422D3F89812032A7FF464AC83
:1088C00000293FF461AC0A7B002A7FF45DAC0120F3
:1088D0000873D3F8A832C3F8A820092203F1900145
:1088E000C3F89C90C3F8A42040F20312A3F8902090
:1088F0001A698242D2B2186808BFC3F8A09031F05A
:108900006BFB41E420B10468808802B10004A061DF
:108910008D4A42F21070D2F88021106167E69AF811
:108920002630DD073FF579AC7CE4013BC2F87434B6
:1089300035E440F2833E4FF0190C1CFB08E8434538
:10894000CCBF4FF000084FF00108F1E57F48804AA6
:10895000848AC08A06EE904A02F1100407EE100ADB
:10896000F8EEE66AB8EEC77AF2EC017A9B08F4EE0C
:10897000E67A63F07F00F1EE10FAF4EEC77AC8BF32
:10898000C3B2F1EE10FA48BF43F040039442EBD17A
:108990009AF88C229A4200F036860022AAF88E229B
:1089A0008AF890226B4A8AF88C321278002A00F0FA
:1089B00017865F2B00F050836F2B00F03C8600235E
:1089C000CAF894329AF82630DF073FF52BAC9AF8B4
:1089D0009032002B7FF426ACBAF98E32322B7FF71F
:1089E00021AC5D4B1B6813F0600F7FF41BAC5B4B3D
:1089F00001221B788AF89022934201F00381DAF871
:108A00003C3213F400727FF40DAC9AF88C32572B81
:108A100001F0C481029909684C0702D55A2B00F075
:108A2000B0815D2B01F03D825E2B01F033825B2B28
:108A300001F02982562B01F0F3829AF88C32972BA1
:108A400001F0D782BAF82C22900741F07A82A3F184
:108A5000B702072A01F25E82DFE812F0550A5C0ACB
:108A60005C0A5C0A9F0C5C0A980C670C00233C4A69
:108A700082F84C33BCF1000F3FF43AAE394B1B780F
:108A8000002B7FF435AE17200BF018FA30E64FF0CC
:108A9000010C8AF873C4E7E534F05CFED1E54020B0
:108AA00034F058FEDAF8383298057FF5C3ADBAF8DD
:108AB0002C2211053FF5BEAD14F064FE002840F0F5
:108AC0005786DAF83832B5E5402034F043FE029B91
:108AD0001B685B057FF5C2AD234A02F1780013469F
:108AE00003E00633984200F0C78119780F29F8D1C6
:108AF0009C78D9788C4210D359790029F1D00CE0B8
:108B00009178D3789942C0F09C825379002B40F041
:108B100098820632904200F0C98113780F2BF8D169
:108B2000EEE7059B1B689E077FF5D8AD0C4B93F8CD
:108B30004C33002B7FF4D8AD094AC2E9D43301236A
:108B400095E700BF3C2F0120F4400120683601204A
:108B5000C471012090030120B43A0120342F012078
:108B6000E851002060300020E83701201D68EB0646
:108B70007FF54AABB34B187816F02EF900287FF436
:108B800043ABEF043FF540AB9AF82A32002B7FF459
:108B90003BABBAF82C321E053FF536AB0FF054FB59
:108BA000A94B1B78002B01F06181002841F0518115
:108BB0002CB1DAF83032049A9A4201F24F82102036
:108BC0000BF07CF901238AF83432FFF721BB142023
:108BD0000BF074F99D4BDAF838221B78002B7FF4E8
:108BE000DAAB002A04DA9AF82630DF077FF5D3AB38
:108BF0009AF8E032964A0693964B12681B680892E0
:108C00005E1C00F03C85944A0192944A002B126845
:108C1000079240F3FC80924C0025DFF858922179AE
:108C20000A234FF0010C13FB01C309EB030219F8EF
:108C300003005678B04280F0E18001EB810240F6FB
:108C4000330B192740F2833E19F812304FEA81089E
:108C500017FB00E009EB42020AEB8303D3ED957AA0
:108C6000FDEEE77A17EE903A5B45A8BF5B46B3F599
:108C7000617FB8BF4FF46173834240F3BF80D27805
:108C800017FB06E7774E013ABB4202EB4200304445
:108C900090F8406302FA0CF000F3B080002E00F070
:108CA000AD802368079FFB1A002B04DB07F5FA73DE
:108CB00084F805C02360069B002B00F0A180694B5F
:108CC00002441A4492F84133002B40F09980414409
:108CD00009EB41010B790433DBB20AEB830393ED1B
:108CE000917A614B5B8A03F1C80107EE901AF8EEA6
:108CF000E77AB4EEE77AF1EE10FA00F31C81C83B94
:108D000007EE903AF8EEE77AB4EEE77AF1EE10FA71
:108D100040F1FE84637992F84283002B70D041F2D7
:108D20000242524BC8F100081A800222FF210E2095
:108D300099540BF0C3F8731E1F2B00F2FB82DFE87F
:108D400013F0D102A70262038D020703630235020A
:108D5000EA0148032A03D303F9028D0213046302D4
:108D60003502EA01CD03C703C103A703AF017F03A7
:108D7000F902D1021704A7021504F902AF010D048C
:108D8000EF039AF89D32002B01F0AF8201238AF89D
:108D90009D228AF89E32364B05939AF89F32DBB1BA
:108DA0009AF82630DA0717D52F4B9AED947A9B8ADA
:108DB00007EE903AF8EEE77AB4EEE77AF1EE10FAC1
:108DC0000ADDDAF8383213F0010207D18AF89F225F
:108DD0003222AAF8A22201E0DAF838329B0471D5D7
:108DE0009AF8A4322BB99AF89D3213B93223AAF813
:108DF000A23201238AF8A432FFF71BBA00232360B2
:108E0000144B013508341B689D42FFF608AF069BE2
:108E1000002B40F0B880114BDAF854241B689B1AE1
:108E2000B3F5FA6F02D40023CAF85834DAF83822BE
:108E3000FFF7B3BA042034F08DFCDAF83832FFF7CC
:108E4000EBBB00BF1A3B012090030120E84001204A
:108E5000583601208C03012094250020C8180120D9
:108E600068720120F44E050868360120703A01202E
:108E7000F0400120684801209AF82630D9077FF594
:108E80004CAE9AF87234002B7FF401AEB74C04F567
:108E9000287594F8DA30002B40F0AC83E034A5421A
:108EA000F7D101238AF87234FFF7D8BB9AF87234ED
:108EB000002B3FF4D3AB0CF0DBF900238AF87234BB
:108EC000FFF7CCBB9AF89D32002B3FF4B2A99AF879
:108ED000263013F001037FF4ACA98AF89D320123F8
:108EE0008AF89E32FFF7A5B9042034F049FCBAF99C
:108EF00070349F4A82FB0312DB17C3EBA203AAF86C
:108F00006834DAF83832FFF787BB9AF873348BF895
:108F100008705BBB00EB400309EB43035A78430046
:108F20000AB194490A701A1809EB42029278F2B118
:108F300090494A701BE0637992F84283002B3FF41A
:108F40005FAF8D4BB8F1000F00F094878B4A1A6029
:108F50000422EBE6012034F013FCFFF72BBA884A19
:108F6000D279022A7FF40EABFFF731BA43000344F3
:108F700009EB430999F80330002B3FF4AAAB7D4A73
:108F80009370FFF7A6BBDAF8E432002B7FF743AF0C
:108F9000DFED7C8A00269FED7C8ADFF80892DFF8FF
:108FA000EC817A4B012213F826500A2313FB052388
:108FB00009EB030119F803204878824236D205EB09
:108FC000850340F633014FF0190C40F2833719F84E
:108FD000134009EB43031CFB02720AEB8404D4ED3B
:108FE000957AAC00FDEEE77A069417EE904A8C4233
:108FF000A8BF0C46B4F5617FB8BF4FF461749442CA
:1090000014DDDA781CFB0070614F013A844202EBF8
:109010004202CCBF002401243A4492F840B3BBF191
:10902000000F08BF0024002C40F0A4820023A8F801
:1090300002300136DAF8E43208F104089E42B0DB6F
:10904000E9E6DAF8383218047FF530AF9AF872346E
:10905000002B7FF403AB19E7BAF98E32B3F5FA7F30
:10906000FFF6E0A89AF89032002B7FF4DBA8CAF84C
:10907000943201238AF890329AF8263013F00104D2
:1090800000F0D7859AF89C221AB943F002038AF8B7
:10909000263003200EF0A0FC3E4B0593FFF7C4B82A
:1090A000DFF804B13C4BDBF800005A79478A4744AB
:1090B000B7F5FA6FA8BF4FF4FA6727EAE777478258
:1090C000002A40F0E1851E2E00F04F8187895B79F0
:1090D0004744B7F5FA6FA8BF4FF4FA6727EAE77776
:1090E0008781002B40F0C48501232C4A137015F0B2
:1090F00081FE00230C2E6371294B1B6840F04081D8
:10910000DAF854249B1AB3F5FA6F3FF579AE0023D1
:10911000CAF8583474E6DFF890B01F4BDBF8000053
:109120005A79077C4744C82FA8BFC82727EAE777A2
:109130000774002A40F06786112E00F01681877AA6
:109140005B794744C82FA8BFC82727EAE77787720B
:10915000002BC9D09AF8503414220F970A3BADF86F
:109160004420012B4BD9DBF80000BDE7883C0120EF
:1091700067666666FC380120703A0120021402140A
:10918000DC3701200080BB446F12033B5873012081
:10919000F44E0508F0400120E8310120D53A0120C5
:1091A000C8180120684801205C360120DFF8DCB2D5
:1091B000B24BDBF800005A79C77B4744C82FA8BFE1
:1091C000C82727EAE777C773002A40F02F86102EBA
:1091D00000F0CB80477A5B794744C82FA8BFC827E7
:1091E00027EAE7774772002B3FF47EAF9AF85034B6
:1091F00013220F970A3BADF84420012BB3D80FA9D7
:109200000D2018F04FFCAEE7DFF880B29B4BDBF887
